:100000000C94801A0C94B11A0C94B11A0C94B11A75
:100010000C94B11A0C94B11A0C94B11A0C94B11A34
:100020000C94B11A0C94B11A0C94B11A0C94B11A24
:100030000C94B11A0C94B11A0C94B11A0C94B11A14
:100040000C94B11A0C945FD10C94B11A0C94B11A9F
:100050000C94B11A0C94B11A0C945CBE0C94FCA9CB
:100060000C94B11A0C942F560C9425560C94B11A7A
:100070000C94B11A0C94B11A0C94B11A0C94B11AD4
:100080000C9408340C94B11A0C94B11A0C94B11A53
:100090000C94B11A0C94B11A0C94B11A0C94B11AB4
:1000A0000C94B11A0C94B11A0C94DA330C94B11A62
:1000B0000C94B11A0C94B11A0C94B11A0C94B11A94
:1000C0000C94B11A0C94B11A0C94B11A0C942337F5
:1000D0000C94ED360C94B11A0C94B11A0C94B11A1C
:1000E0000C94B11A084AD73B3BCE016E84BCBFFDCD
:1000F000C12F3D6C74319ABD56833DDA3D00C77FF8
:1001000011BED9E4BB4C3E916BAAAABE0000008090
:100110003F05A84CCDB2D44EB93836A9020C50B91F
:10012000918688083CA6AAAA2ABE000000803F004B
:100130000C946FFC0D94590B0C94A4FC0C9453FC80
:100140000C94D5FB0C94F3A70C9467FC0C949F378C
:100150000D94F20C0C94D9A90C9449FC0D942E0C1E
:100160000C94C1560C94AEFC0C9463440C9495FC16
:100170000D94750F0C94C9370C94CCFB0C94F1FBC7
:100180000C94AEFB0D9439090D94DC1E0D94890975
:100190000C94E7370C94FFFB0C94BA560C940FA9FF
:1001A0000D9437110D94480F0D9426050C946B4255
:1001B0000D94570F0C943FFF0D942F0F0D94FF0ECD
:1001C0000C94CD560D94820B0C94CFFB0C948BFCAD
:1001D0000D94820F0D946F010C94D9560D94171441
:1001E0000C94BD370D94C0070C94D4370C94B8FC14
:1001F0000C94DF370D94410C0D9474100D94550937
:100200000C94C5560D94BE1E0C943CFC0C94AB563D
:100210000C94D9FB0C94C0FB0C94CD370C94E3FBED
:100220000C94D2A70C949C560C94D5560C94FBFBC2
:100230000D94B90B0C94F5FB0C9461370C94B93701
:100240000C94A9FB0C94C2FC0C94C1370D94631060
:100250000C94D0A80C94C8FB0C94A4440C946EA4E9
:100260000C941C420C9444FC0C94E0560C94CCFC72
:100270000C94B5370D94EC0B0D94960B0C943DA794
:100280000D9445010D94610F0C946D560C94AE378E
:100290000C94C4FB0D94EB0A0C9477FC0C94D6FCE4
:1002A0000C94F3560D94D7020D94260F0D94250A45
:1002B0000D94A8030D9406090C94C5370D94B50A46
:1002C0000C94EB560D94CD0B0C9437A80C94E7FBD3
:1002D0000C9437440C9481FC0C94EDFB0C94F1A429
:1002E0000C94F0A40C945DFC0C94DC440C94E2A8F7
:1002F0000D942C0F0C946F420D9460000C94C95611
:100300000C94D1560C94DFFB0C9452A80C945AA771
:100310000C9490374E414E494E495459494E46CD62
:10032000CCCC3D0AD7233C17B7D13877CC2B3295AC
:1003300095E6241FB14F0A000020410000C842008A
:10034000401C4620BCBE4CCA1B0E5AAEC59D740054
:10035000407A10F35A00A0724E18090010A5D4E894
:100360000000E87648170000E40B54020000CA9A27
:100370003B000000E1F50500008096980000004079
:10038000420F000000A086010000001027000000BE
:1003900000E803000000006400000000000A000004
:1003A0000000000100000000002C76D888DC674FB8
:1003B0000823DFC1DFAE59E1B1B796E5E3E453C6E8
:1003C0003AE651997696E8E6C28426EB898C9B62E0
:1003D000ED407C6FFCEFBC9C9F40F2BAA56FA5F48A
:1003E00090055A2AF75C936B6CF9676DC11BFCE0B2
:1003F000E40D47FEF520E6B500D0ED902E03009405
:100400003577050080841E080000204E0A00000099
:10041000C80C333333330F986E12831141EF8D21A3
:1004200014893BE65516CFFEE6DB18D1844B381B0A
:10043000F77C1D901DA4BBE424203284725E2281CF
:1004400000C9F124ECA1E53D27434F4D4D554E49E0
:10045000434154494F4E0044525952554E00455263
:10046000524F525300494E464F004543484F0045B6
:1004700072726F722077726974696E6720746F2070
:10048000454550524F4D210A0053544F505045445A
:100490002E20005072696E7465722073746F7070D4
:1004A00065642064756520746F206572726F727365
:1004B0002E2046697820746865206572726F7220FC
:1004C000616E6420757365204D39393920746F2051
:1004D000726573746172742E202854656D70657234
:1004E00061747572652069732072657365742E205E
:1004F0005365742069742061667465722072657337
:1005000074617274696E67290A004E6F20436865D2
:10051000636B73756D2077697468206C696E6520F4
:100520006E756D6265722C204C617374204C696E1F
:10053000653A20004E6F20436865636B73756D20CC
:1005400077697468206C696E65206E756D6265727E
:100550002C204C617374204C696E653A20006368EE
:1005600065636B73756D206D69736D617463682C61
:10057000204C617374204C696E653A20004C696EA2
:1005800065204E756D626572206973206E6F7420F0
:100590004C617374204C696E65204E756D62657296
:1005A0002B312C204C617374204C696E653A20000D
:1005B0004D3131300053657269616C207374617420
:1005C0007573206D69736D617463680A0077616982
:1005D000740A0053442072656164206572726F7200
:1005E0000A002121204B494C4C20636175736564DE
:1005F00020627920746F6F206D75636820696E6169
:1006000063746976652074696D65202D2063757249
:1006100072656E7420636F6D6D616E643A20004880
:100620006F74656E642049646C652054696D656FF4
:10063000757400486F74656E642049646C6520545D
:10064000696D656F75740A003D3D6F6E46696C613A
:100650006D656E7452756E6F75743D3D0070617599
:100660007365004D363030002066696C616D656ED3
:10067000745F72756E6F7574200066696C616D656C
:100680006E745F72756E6F757420540046696C618C
:100690006D656E7452756E6F75742054002A2A2A27
:1006A000496E6974696E67206361726420697320A2
:1006B0004F4B2A2A2A004D6564696120496E736593
:1006C00072746564004D656469612052656D6F7672
:1006D0006564004D313030305300627573793A20D3
:1006E00070617573656420666F7220696E707574D1
:1006F0000A00627573793A207061757365642066CB
:100700006F7220757365720A00627573793A207092
:10071000726F63657373696E670A002A2A2A6B69B0
:100720006C6C2A2A2A00706F7765726F6666004BC0
:10073000494C4C45442E20005072696E74657220FD
:1007400068616C7465642E206B696C6C2829206369
:10075000616C6C6564210A0053544F505045442E1F
:1007600020005072696E7465722073746F707065CA
:10077000642064756520746F206572726F72732EC9
:100780002046697820746865206572726F722061F6
:100790006E6420757365204D39393920746F20726D
:1007A0006573746172742E202854656D7065726172
:1007B000747572652069732072657365742E205399
:1007C0006574206974206166746572207265737443
:1007D000617274696E67290A006563686F3A004543
:1007E00072726F723A0042696C696E656172204C78
:1007F0006576656C696E6720477269643A0A002104
:10080000212053544F502063616C6C6564206265F5
:100810006361757365206F6620424C546F75636821
:10082000206572726F72202D20726573746172740C
:100830002077697468204D3939390A002121205305
:10084000544F502063616C6C656420626563617510
:100850007365206F6620424C546F75636820657223
:10086000726F72202D2072657374617274207769C3
:100870007468204D3939390A002F2F616374696F0C
:100880006E3A0070726F6D70745F00656E64005335
:10089000656E64204D31303820746F207265737539
:1008A0006D650A00496E736572742066696C616DCE
:1008B000656E7420616E642073656E64204D313006
:1008C000380A005265686561742066696E697368EC
:1008D00065642E0052656865617420446F6E650022
:1008E000526568656174696E672E2E2E00526568C8
:1008F000656174004865617465722054696D656F47
:1009000075740053656E64204D31303820746F204B
:1009100068656174206E6F7A7A6C650A004E6F7A32
:100920007A6C65205061726B656400486F74656E07
:100930006420746F6F20636F6C640A00706175735C
:1009400065640050617573650044697361626C652C
:1009500052756E6F75740050757267654D6F726574
:10096000005061757365640073686F770062757419
:10097000746F6E00626567696E004C6F616420463B
:10098000696C616D656E74004C6F61642046696CC2
:10099000616D656E74205400496E736572742066D3
:1009A000696C616D656E7420616E642073656E6440
:1009B000204D3130380A00726573756D65640052E0
:1009C0006573756D696E670057616974696E67203C
:1009D000666F72206865617475702E0A004C6561DF
:1009E00076696E6720473236003F537065636966EB
:1009F00069656420582C5920636F6F7264696E6159
:100A00007465206F7574206F6620626F756E6473F5
:100A10002E0A003F28522965706561742076616C4A
:100A20007565206E6F7420706C61757369626C659A
:100A30003B206D757374206265206174206C656164
:100A4000737420312E0A003F285229657065617445
:100A5000206D7573742062652073706563696669C3
:100A60006564207768656E206E6F74207573696E9B
:100A70006720616E204C43442E0A003F537065632B
:100A80006966696564206E6F7A7A6C652074656D3D
:100A90007065726174757265206E6F7420706C6120
:100AA000757369626C652E0A003F537065636966F1
:100AB0006965642066696C616D656E742073697A1E
:100AC00065206E6F7420706C61757369626C652E41
:100AD0000A003F53706563696669656420707269D6
:100AE0006D65206C656E677468206E6F7420706C25
:100AF00061757369626C652E0A003F5072696D659D
:100B0000206C656E677468206D7573742062652053
:100B1000737065636966696564207768656E206EC9
:100B20006F74207573696E6720616E204C43442E8C
:100B30000A003F537065636966696564206E6F7A69
:100B40007A6C652073697A65206E6F7420706C61B1
:100B5000757369626C652E0A003F52657472616339
:100B600074696F6E204D756C7469706C6965722064
:100B70006D7573742062652073706563696669655D
:100B8000642E0A003F53706563696669656420528C
:100B9000657472616374696F6E204D756C746970F1
:100BA0006C696572206E6F7420706C617573696218
:100BB0006C652E0A003F5370656369666965642041
:100BC0006C6179657220686569676874206E6F74FE
:100BD00020706C61757369626C652E0A0043292E62
:100BE0000A003F53706563696669656420626564E5
:100BF0002074656D7065726174757265206E6F74B6
:100C000020706C61757369626C65202834302D002A
:100C1000473236207374617274696E672E2E2E0A05
:100C2000004F46460A00466164652048656967686A
:100C3000742000426564204C6576656C696E67209F
:100C4000004661696C656420746F20656E61626C3A
:100C50006520426564204C6576656C696E670A00A4
:100C6000496E76616C6964206D6573682E0A005068
:100C7000726F62696E6720506F696E740025532031
:100C800025692F2569002E0A002F0050726F6269B6
:100C90006E67206D65736820706F696E7420002028
:100CA0002844525952554E29004732392041757413
:100CB0006F20426564204C6576656C696E67003F05
:100CC00020284C2C522C462C4229206F7574206F02
:100CD0006620626F756E64732E0A003F2856296580
:100CE00072626F7365206C6576656C20696D706CDF
:100CF00061757369626C652028302D34292E0A00D5
:100D0000426164205A2076616C75650A004E6F203E
:100D100062696C696E65617220677269640A004479
:100D20006576696174696F6E0025533A20257300FA
:100D300046696E6973686564210A003A207A3A2030
:100D400000206F662000476F696E6720746F3A203D
:100D5000580043570A00206469723A0020616E67A8
:100D60006C653A00537461727420726164697573C2
:100D70003A004D343820506F696E740025533A2084
:100D800025642F256400506F736974696F6E696EF6
:100D900067207468652070726F62652E2E2E0A00BF
:100DA0003F4C656773206F66206D6F76656D656E6D
:100DB0007420696D706C61757369626C6520283090
:100DC0002D3135292E0A003F2028582C5929206F13
:100DD0007574206F6620626F756E64732E0A005002
:100DE000726F6265206F7574206F6620626F756E1A
:100DF0006473003F53616D706C652073697A652080
:100E00006E6F7420706C61757369626C6520283434
:100E10002D3530292E0A004D3438205A2D50726F4E
:100E20006265205265706561746162696C6974798C
:100E300020546573740A003F2856296572626F73E7
:100E400065206C6576656C20696D706C6175736981
:100E5000626C652028302D34292E0A005374616E8F
:100E60006461726420446576696174696F6E3A20CA
:100E7000002052616E67653A2000204D61783A206B
:100E800000204D696E3A2000205369676D613A2059
:100E9000004D65616E3A20005741524E494E472140
:100EA000204C6F77205A204A65726B206D61792043
:100EB0006C65616420746F20756E77616E74656413
:100EC000207061757365732E0A004F4646004F4EC1
:100ED0000020204D61783A2000200020204D696ECE
:100EE0003A2000536F667420656E6473746F70737C
:100EF0003A20003D3D4F6E506F7765724C6F7373B3
:100F0000526573756D653D3D004D32342053256C3F
:100F1000642054256C64004739322E3920452573EE
:100F200000473120462564004739322E39205A25A2
:100F300073004731205A302046323030004731208C
:100F400058257320592573204633303030004D34F6
:100F5000323020532569205A2573004D3130362018
:100F600050256920532569004D32303020442573C7
:100F70000047323852305859004739322E3920450F
:100F800030205A300A47315A2573004D313039200C
:100F9000532569004D31393020532569004D3432D5
:100FA00030205330205A300020496E76616C6964DD
:100FB000206578747275646572200047322F47335C
:100FC0002062616420706172616D65746572730A7C
:100FD00000536C6565702E2E2E005A2050726F6281
:100FE000652050617374204265640A005A20507273
:100FF0006F62652050617374204265640047323827
:101000004C30004D3131372050726F62652066617F
:10101000696C65642E0A4732380A0070726F626527
:101020005F72657769706500473239205265747266
:1010300079696E670050726F62696E6720466169F8
:101040006C6564004D31313720426564206C6576F3
:10105000656C696E67206661696C65642E0A47304D
:10106000205A31300A4D3330302050323520533839
:1010700038300A4D333030205035302053300A4D4F
:101080003330302050323520533838300A4D333029
:1010900030205035302053300A4D3330302050321C
:1010A0003520533838300A4D333030205035302019
:1010B00053300A47342053310070726F62655F66A7
:1010C00061696C6564004D31313720426564206C84
:1010D0006576656C696E6720646F6E652E00205AB8
:1010E0003A200020593A200042656420583A2000F6
:1010F0004D65736820706F696E74206F7574206F12
:10110000662072616E67650A004D302053746F70FF
:10111000004D312053746F7000436F6E74696E75AB
:101120006500436C69636B20746F20526573756D45
:10113000652E2E2E004E6F204D6F76652E00456E6B
:10114000642066696C65206C6973740A0042656787
:10115000696E2066696C65206C6973740A004E6F55
:10116000206D656469610A00526573756D696E670B
:1011700020534400286E6F2066696C652900437512
:101180007272656E742066696C653A2000507269EF
:101190006E742074696D653A20000A53746174732B
:1011A0003A2046696C616D656E7420757365643AAA
:1011B00020002C204C6F6E67657374206A6F623A52
:1011C0002000546F74616C2074696D653A2000537F
:1011D000746174733A20002C204661696C65643A2E
:1011E00020002C2046696E69736865643A200050BF
:1011F00072696E74733A200053746174733A2000FC
:10120000436F6F6C696E672E2E2E0048656174699E
:101210006E672E2E2E0045202553006F6B006F66E3
:1012200066006A0465045E04570449044445425557
:10123000473A004D31313320530042656420436FFB
:101240006F6C696E672E2E2E0042656420486561C2
:1012500074696E672E2E2E0044445820313053207E
:1012600050726F204F46462E002F2F002052004113
:101270006363656C65726174696F6E3A2050004DEE
:1012800032303620580046523A0020466C6F773A8A
:1012900020003A200020536572766F2000206F7581
:1012A00074206F662072616E67650A0053657276FE
:1012B0006F200020643A0020693A0020703A00490B
:1012C0006E76616C69642065787472756465720A03
:1012D0000020643A0020693A0020703A0064697383
:1012E00000656E0043290A0061626C656420286D08
:1012F000696E2074656D702000436F6C64206578A2
:1013000074727564657320617265200050494420D1
:101310004175746F74756E65005049442041757451
:101320006F74756E65206661696C65642120426129
:1013300064206865617465722069640A0046696C9E
:10134000616D656E742072756E6F7574206469735B
:1013500074616E636520286D6D293A200046696CC2
:10136000616D656E742072756E6F757420004D34FA
:10137000323120696E636F727265637420706172BE
:10138000616D657465722075736167650A004D65EE
:10139000736820706F696E74206F7574206F66209B
:1013A00072616E67650A004F6666736574732041EB
:1013B00070706C696564004572723A20546F6F20DA
:1013C0006661722100546F6F206661722066726FD1
:1013D0006D207265666572656E636520706F696EFB
:1013E000740A00454550524F4D204F4B0A00506F34
:1013F0007765722D6C6F7373207265636F7665729B
:101400007920004D383400446F6E65207072696E2B
:1014100074696E672066696C650A004D3737004D48
:101420003331004361703A004D4541545041434BC4
:1014300000434F4F4C45525F54454D504552415427
:10144000555245004348414D4245525F54454D5029
:10145000455241545552450042414259535445501A
:1014600050494E470041524353004D4F54494F4E4F
:101470005F4D4F44455300544845524D414C5F50D9
:10148000524F54454354494F4E004C4F4E475F46D0
:10149000494C454E414D45004155544F5245504FE2
:1014A00052545F53445F5354415455530053445F67
:1014B0005752495445005245504541540053444306
:1014C0004152440050524F4D50545F535550504F6D
:1014D000525400454D455247454E43595F50415285
:1014E00053455200434153455F4C494748545F427E
:1014F00052494748544E45535300544F47474C4573
:101500005F4C494748545300534F46545741524546
:101510005F504F574552004255494C445F50455229
:1015200043454E54004C4556454C494E475F444157
:101530005441005A5F50524F42450052554E4F554C
:1015400054004155544F4C4556454C005052494E5D
:10155000545F4A4F420050524F4752455353004147
:1015600055544F5245504F52545F54454D500056BC
:101570004F4C554D455452494300454550524F4DEF
:101580000042494E4152595F46494C455F545241D1
:101590004E534645520053455249414C5F584F4EB9
:1015A0005F584F4646004649524D574152455F4E9F
:1015B000414D453A4D61726C696E20322E302E37A6
:1015C0005F4457372E3320426F6E64746563682022
:1015D00053534D444242202841707220323420320D
:1015E0003032312032333A30313A34392920534FB6
:1015F000555243455F434F44455F55524C3A6874DA
:101600007470733A2F2F6769746875622E636F6DFB
:101610002F496E73616E6974794175746F6D617471
:10162000696F6E2F4D61726C696E2F747265652FD4
:10163000437265616C6974794477696E5F322E30EC
:101640002050524F544F434F4C5F56455253494FD1
:101650004E3A312E30204D414348494E455F545952
:1016600050453A444458203130532050726F204541
:10167000585452554445525F434F554E543A3120C9
:10168000555549443A63656465326132662D34319B
:1016900061322D343734382D396231322D6335358E
:1016A0006336326633363766660A0050726F62659B
:1016B000204F6666736574205A0050726F62652011
:1016C0004F6666736574205A00290A0020746F20E3
:1016D000003F5A206F7574206F662072616E6765D7
:1016E000202800290A0020746F20003F59206F75C0
:1016F00074206F662072616E676520282D00290AAC
:101700000020746F20003F58206F7574206F662092
:1017100072616E676520282D0050726F6265204FE0
:10172000666673657420580043616E6E6F74206F37
:1017300070656E207375626469722000256973009C
:1017400025696D20256973002569682025696D204C
:1017500025697300256964202569682025696D2045
:101760002569730025697920256964202569682029
:1017700025696D20256973003D3D4477696E2049D8
:101780006E697420436F6D706C6574653D3D002A11
:101790002A2A4E6F7A7A6C6554656D705374617441
:1017A00075735B325D203D003D3D48656174696E37
:1017B0006720446F6E65204368616E6765204669E7
:1017C0006C616D656E743D3D0020207374617274B0
:1017D00070726F677265737320003D3D7761697445
:1017E00077617920353D3D003D3D776169747761D2
:1017F0007920343D3D003D3D776169747761792002
:10180000333D3D003D3D7761697477617920313D1D
:101810003D003D3D6F6E5072696E7454696D657226
:1018200053746F707065643D3D003D3D6F6E466161
:1018300063746F727952657365743D3D00270A0ABF
:101840000000272027002027002D006E6F74696696
:1018500069636174696F6E200063616E63656C001B
:101860005072696E742041626F72746564004469DD
:10187000736D6973730055492041626F72746564BA
:1018800000726573756D65004D3234002A2A2A4353
:10189000506C617920546F6E652A2A2A003D3D6F95
:1018A0006E5072696E7454696D65725061757365BE
:1018B000643D3D00486F6D696E67204661696C65E7
:1018C00064006F70656E0054524947474552454465
:1018D000003A200066696C616D656E74007A5F6D18
:1018E000696E00795F6D696E00785F6D696E005298
:1018F00065706F7274696E6720656E6473746F7063
:10190000207374617475730A0020746F6F206C6F9C
:101910006E6720657874727573696F6E207072657A
:1019200076656E7465640A0020636F6C6420657868
:1019300074727573696F6E2070726576656E74650A
:10194000640A00486F6D6520257325732573204652
:1019500069727374005761726E696E673A20486FDE
:101960006D696E672042756D702044697669736F8A
:1019700072203C20310A0002020400000000000036
:1019800000000000000000809D4300009B43000019
:10199000C843000000410000004100000040FFFF7C
:1019A000FF000000010000000100008000555555B7
:1019B000000000400033333300AAAA2A00499224D1
:1019C0000000002000C7711C0099991900D145172B
:1019D00000555515003BB113002449120011111197
:1019E00000000010000F0F0F00E3380E0043790DC8
:1019F00000CCCC0C00C3300C00E8A20B0064210B1F
:101A000000AAAA0A00703D0A009DD80900427B097D
:101A10000092240900DCD3080088880800104208DE
:101A20000000000800F0C107008787070075500715
:101A300000711C07003EEB0600A1BC060069900681
:101A40000066660600703E06006118060017F40581
:101A50000074D105005BB00500B29005006272050C
:101A6000005555050078390500B81E050005050527
:101A7000004EEC040087D40400A1BD040090A7042C
:101A80000049920400C17D0400EE690400C75604B9
:101A900000444404005C32040008210400411004A6
:101AA00000000004003FF00300F8E0030026D2032A
:101AB00000C3C30300CCB503003AA803000A9B038C
:101AC00000388E0300C08103009F750300D06903B6
:101AD00000505E03001D53030034480300913D0392
:101AE000003333030016290300381F030097150342
:101AF00000300C0300030303000BFA020049F1025B
:101B000000BAE802005CE002002DD802002DD002ED
:101B10000059C80200B0C0020031B90200DAB102B7
:101B200000AAAA0200A0A30200BC9C0200FA95022F
:101B3000005C8F0200DF88020082820200457C0286
:101B4000002776020027700200436A02007C6402CC
:101B500000D05E02003F590200C8530200FFFDFCA6
:101B6000FAF8F6F4F2F0EEECEAE9E7E5E3E1E0DEBC
:101B7000DCDAD9D7D5D4D2D0CFCDCBCAC8C7C5C36C
:101B8000C2C0BFBDBCBAB9B7B6B4B3B2B0AFADACEA
:101B9000AAA9A8A6A5A4A2A1A09E9D9C9A9998973F
:101BA00095949392908F8E8D8B8A89888786848373
:101BB0008281807F7E7D7B7A797877767574737287
:101BC00071706F6E6D6C6B6A69686766656463627D
:101BD00061605F5E5D5C5B5A595858575655545367
:101BE000525150504F4E4D4C4B4A4A494847464639
:101BF000454443424241403F3E3E3D3C3B3B3A39F7
:101C0000383837363535343332323130302F2E2EA6
:101C10002D2C2B2B2A292928272726252524232349
:101C200022212120201F1E1E1D1C1C1B1B1A1919DE
:101C30001818171616151514131312121111100F68
:101C40000F0E0E0D0D0C0C0B0A0A090908080707E8
:101C5000060605050404030302020100003D3D6F72
:101C60006E5072696E7454696D65725374617274EA
:101C700065643D3D0000809D4300009B430000C81B
:101C8000430000000000000000000000003D3D6F28
:101C90006E53746F726553657474696E67733D3DFE
:101CA000003D3D6F6E436F6E666967757261746962
:101CB0006F6E53746F72655772697474656E3D3DD3
:101CC0000053657474696E67732053746F72656432
:101CD000000A20696E6974207A70726F62655F7A9B
:101CE0006F6666736574203D20003D3D6F6E436FE7
:101CF0006E66696775726174696F6E53746F726531
:101D0000526561643D3D00454550524F4D20496E3E
:101D1000697469616C697A65640A003B20003A0A5B
:101D20000020204D363033200020440020204D3448
:101D3000313220530046696C616D656E7420727596
:101D40006E6F75742073656E736F723A0020550064
:101D50004C0046696C616D656E74206C6F61642F18
:101D6000756E6C6F6164206C656E677468733A00A1
:101D700020204D3835312058005A2D50726F626541
:101D8000204F66667365740020204D343133205334
:101D900000506F7765722D4C6F7373205265636FBF
:101DA000766572793A0020440020490020204D33A6
:101DB000303420500020440020490020204D333092
:101DC000312050005049442073657474696E677304
:101DD0003A00204A0020204732392057204900206D
:101DE000204D3432302053004175746F20426564B9
:101DF000204C6576656C696E673A0020204D323064
:101E000036205800486F6D65206F66667365743ABA
:101E10000020580020530020204D32303520420051
:101E2000416476616E6365643A20423C6D696E5F21
:101E30007365676D656E745F74696D655F75733E1C
:101E400020533C6D696E5F66656564726174653EC2
:101E500020543C6D696E5F74726176656C5F666577
:101E60006564726174653E20583C6D61785F785F8F
:101E70006A65726B3E20593C6D61785F795F6A6577
:101E8000726B3E205A3C6D61785F7A5F6A65726B57
:101E90003E20453C6D61785F655F6A65726B3E0010
:101EA00020540020520020204D3230342050004178
:101EB0006363656C65726174696F6E2028756E6905
:101EC00074732F7332293A20503C7072696E745FBC
:101ED000616363656C3E20523C7265747261637429
:101EE0005F616363656C3E20543C74726176656C1F
:101EF0005F616363656C3E0020204D3230312058B5
:101F0000004D6178696D756D20416363656C657224
:101F10006174696F6E2028756E6974732F7332292E
:101F20003A0020204D3230332058004D6178696DE1
:101F3000756D206665656472617465732028756EC1
:101F40006974732F73293A00537465707320706538
:101F50007220756E69743A0020440020204D3230A2
:101F6000302053002044697361626C65640A004646
:101F7000696C616D656E742073657474696E6773E6
:101F80003A0020286D6D2900202047323120202082
:101F9000203B20556E69747320696E206D6D003D85
:101FA0003D6F6E4C6F616453657474696E67733D09
:101FB0003D000000FA430000FA4300002041000009
:101FC0008C420000A0420000A0420000C8430080F4
:101FD000CF43EE020000EE020000640000003C006F
:101FE000000024F4D43050C38E20C2A24017828B4C
:101FF0007011127A910D816CD90AA861E108C75855
:102000006607615143061E4B5D05C145A7041A4191
:102010001104093D9803713931034036DB02653301
:102020009102D4305402802E1D02632CEE01752AD9
:10203000C501B028A001102781018F2564012B2440
:102040004B01E0223401AC211F018D200D01801FC6
:10205000FC00841EED00971DDF00B81CD200E61BBB
:10206000C600201BBC00641AB200B219A8000A19ED
:10207000A0006A189900D117910040178B00B5167F
:10208000840031167E00B31579003A157300C71429
:102090006F0058146A00EE1366008813630025135E
:1020A0005E00C7125B006C12570015125400C1117C
:1020B000510070114F0021114B00D61049008D10B6
:1020C00047004610440002104200C00F4000800F3D
:1020D0003E00420F3C00060F3B00CB0E3800930E33
:1020E00037005C0E3500270E3400F30D3200C10DB1
:1020F0003100900D3000600D2E00320D2D00050DC9
:102100002C00D90C2B00AE0C2900850C29005C0C8E
:102110002700350C27000E0C2600E80B2400C40B0A
:102120002400A00B23007D0B23005A0B2100390B48
:102130002100180B2000F80A1F00D90A1E00BB0A54
:102140001E009D0A1D00800A1D00630A1C00470A2C
:102150001B002C0A1B00110A1A00F7091A00DD09DE
:102160001900C4091900AB091900920917007B096D
:102170001800630917004C091600360916002009DB
:1021800016000A091500F5081500E0081400CC082F
:102190001400B8081400A4081400900813007D0867
:1021A00012006B0813005808120046081200340889
:1021B0001100230811001208110001081100F00796
:1021C0001000E0071000D0071000C0071000B00793
:1021D0000F00A107100091070E0083070F0074077E
:1021E0000F0065070E0057070E0049070E003B075A
:1021F0000D002E070E0020070D0013070D00060727
:102200000D00F9060C00ED060D00E0060C00D406EA
:102210000C00C8060C00BC060C00B0060C00A4069E
:102220000B0099060C008D060B0082060B0077064A
:102230000B006C060B0061060A0057060B004C06EB
:102240000A0042060A0038060A002E060A00240682
:102250000A001A060A001006090007060A00FD0512
:102260000900F4050900EB050900E2050900D9059C
:102270000900D0050900C7050900BE050900B5051C
:102280000800AD050800A50509009C050800940597
:1022900008008C050800840508007C05080074050A
:1022A00008006C050700650508005D050700560578
:1022B00008004E05070047050700400508003805DF
:1022C0000700310507002A050700230507001C0544
:1022D0000600160507000F050700080506000205A1
:1022E0000700FB040600F5040700EE040600E804FE
:1022F0000600E2040700DB040600D5040600CF0454
:102300000600C9040600C3040600BD040600B704A5
:102310000600B1040500AC040600A6040600A004F3
:1023200005009B04060095040500900406008A043D
:10233000050085040500800406007A040500750484
:102340000500700405006B040500660405006104C7
:1023500005005C04050057040500520405004D0407
:10236000050048040500430405003E0404003A0447
:10237000050035040500300404002C040500270482
:102380000400230405001E0404001A0404001604BB
:102390000500110404000D040400090405000404F0
:1023A000040000040400FC030400F8030400F40328
:1023B0000400F0030400EC030400E8030400E40359
:1023C0000400E0030400DC030400D8030400D40389
:1023D0000400D0030400CC030400C8030300C503B9
:1023E000030024F404D9201BC40C5C0E9804C40917
:1023F0005F0265077101F405F900FB04B3004804AE
:102400008700C10369005803550003034500BE025D
:102410003A008402310053022A00290225000402F6
:102420002000E4011C00C8011900AF011700980149
:1024300014008401130071011000610110005101AA
:102440000E0043010D0036010B002B010B00200193
:102450000B00150109000C01090003010800FB0035
:102460000800F3000800EB000700E4000600DE00AF
:102470000600D8000600D2000600CC000500C70008
:102480000500C2000500BD000400B9000400B5004D
:102490000400B1000400AD000400A9000400A50080
:1024A0000300A20003009F0004009B0003009800AB
:1024B00003009500020093000300900003008D00CC
:1024C00002008B00030088000200860002008400E6
:1024D0000300810002007F0002007D0002007B00FB
:1024E000020079000200770001007600020074000B
:1024F000020072000100710002006F0002006D0016
:1025000001006C0002006A0001006900020067001F
:102510000100660001006500010064000200620025
:10252000010061000100600001005F0002005D0029
:1025300001005C0001005B0001005A00010059002D
:10254000010058000100570001005600010055002D
:10255000010054000100530000005300010052002C
:10256000010051000100500001004F0001004E0029
:1025700000004E0001004D0001004C0001004B0026
:1025800000004B0001004A00010049000100480022
:10259000000048000100470001004600000046001E
:1025A0000100450000004500010044000100430017
:1025B0000000430001004200000042000100410011
:1025C000000041000100400001003F0000003F000A
:1025D00001003E0000003E0001003D0000003D0003
:1025E00001003C0000003C0000003C0001003B00FA
:1025F00000003B0001003A0000003A0001003900F1
:1026000000003900010038000000380000003800E8
:1026100001003700000037000100360000003600DE
:1026200000003600010035000000350000003500D4
:1026300001003400000034000000340001003300C9
:1026400000003300000033000100320000003200BF
:1026500000003200010031000000310000003100B4
:1026600001003000000030000000300001002F00A9
:1026700000002F0000002F0000002F0001002E009E
:1026800000002E0000002E0001002D0000002D0093
:1026900000002D0000002D0001002C0000002C0087
:1026A00000002C0000002C0001002B0000002B007B
:1026B00000002B0000002B0001002A0000002A006F
:1026C00000002A0000002A00010029000000290063
:1026D0000000290000002900000029000100280056
:1026E000000028000000280000002800000028004A
:1026F000010027000000270000002700000027003D
:10270000000027000100260000002600000026002F
:102710000000260000002600010025000000250022
:102720000000250000002500000025000000250015
:102730000100240000002400000024000000240008
:1027400000002400010023000000230000002300FB
:1027500000002300000023000000230000002300ED
:1027600001002200000022000000220000002200E0
:1027700000002200000022000100210000002100D2
:1027800000002100000021000000210000002100C5
:1027900000002100010020000000200000002000B7
:1027A00000002000000020000000200000002000A9
:1027B0000000200001001F0000001F0000001F009B
:1027C00000001F0000001F0000001F0000001F008D
:1027D00001001E0000001E0000001E0000001E0080
:1027E0000000393000003325000087190000B00FC9
:1027F0000000DB080000BD040000740200003F017F
:10280000000020436F756E7420583A00236465669B
:10281000696E652044454641554C545F0000626531
:1028200064004B6420004B6920004B70200050492D
:1028300044204175746F74756E652066696E6973A6
:10284000686564212050757420746865206C61731C
:1028500074204B702C204B6920616E64204B6420E7
:10286000636F6E7374616E74732066726F6D206235
:10287000656C6F7720696E746F20436F6E66696751
:1028800075726174696F6E2E680A00504944204168
:1028900075746F74756E65206661696C656421205E
:1028A00074696D656F75740A0050494420417574F0
:1028B0006F74756E65206661696C6564212054656E
:1028C0006D706572617475726520746F6F206869D0
:1028D00067680A00204B643A2000204B693A2000C8
:1028E000204B703A200020436C6173736963205061
:1028F0004944200A00204E6F206F76657273686F1E
:102900006F740A002054753A2000204B753A20005D
:10291000206D61783A2000206D696E3A20002064B5
:102920003A200020626961733A20005049442041F6
:1029300075746F74756E652073746172740A0050DB
:102940004944204175746F74756E65206661696CC9
:102950006564212054656D706572617475726520BF
:10296000746F6F20686967680A00426564004531CA
:1029700000626564002C2073797374656D20737434
:102980006F7070656421204865617465725F4944A9
:102990003A200048656174696E67204661696C651C
:1029A000640048656174696E67206661696C65647E
:1029B000004D3131322053687574646F776E0010AA
:1029C00000C90210012C014001220170011801B060
:1029D000010E01F00104015002FA00B002F00030D3
:1029E00003E600D003DC009004D2007005C800A00C
:1029F00006BE000008B400B009AA00D00BA0006019
:102A00000E960060118C000015820020197800C01D
:102A10001D6E00A0226400B0275A00902C500000C8
:102A2000314600E0343C0010383200903A28006013
:102A30003C1E00A03D1400803E0A00203F000054D0
:102A40004845524D414C2052554E41574159005432
:102A50006865726D616C2052756E617761790045B1
:102A600072723A204D415854454D50004D415854D2
:102A7000454D5020747269676765726564004572E0
:102A8000723A204D494E54454D50004D494E5445E3
:102A90004D502074726967676572656400202F006D
:102AA0002042403A0020403A0020573A0020573A4E
:102AB00000496E76616C696420657874727564652E
:102AC000720A007C3C3E5E2B3D3F2F5B5D3B2C2A17
:102AD000225C0043616E6E6F74206F70656E2073B0
:102AE00075626469722000534420496E69742046FF
:102AF00061696C0053442063617264206F6B0A004B
:102B00006F70656E526F6F74206661696C65640AE0
:102B100000766F6C756D652E696E697420666169EB
:102B20006C65640A004E6F20534420636172640A2E
:102B3000000A4D3234004D3233202573002E0A0036
:102B40006F70656E206661696C65642C2046696CE7
:102B5000653A200046696C652073656C6563746531
:102B6000640A002053697A653A200046696C652042
:102B70006F70656E65643A2000454E44205355429F
:102B8000524F5554494E450A002220706F7300225F
:102B900020706172656E743A2200535542524F554F
:102BA00054494E452043414C4C2074617267657412
:102BB0003A220053756263616C6C204F76657266D1
:102BC0006C6F77004578636565646564206D617836
:102BD00020535542524F5554494E452064657074F8
:102BE000683A002E0A0044656C6574696F6E206651
:102BF00061696C65642C2046696C653A2000466901
:102C00006C652064656C657465643A00534420709B
:102C100072696E74696E67206279746520004E6F08
:102C200074205344207072696E74696E670A00578D
:102C3000726974696E6720746F2066696C653A20EA
:102C400000667265736800646F696E67002066696C
:102C50006C653A20004E6F7720002F6175746F25E8
:102C6000632E67002020506C616E6E65724275663F
:102C700066657242797465733A2000204672656514
:102C8000204D656D6F72793A2000436F6D70696CED
:102C900065643A2041707220323420323032310A79
:102CA00000204C61737420557064617465643A202F
:102CB000323032312D30342D3138207C2041757442
:102CC000686F723A20426F6E6474656368202F20CB
:102CD000496E73616E6974794175746F6D61746961
:102CE0006F6E0A00322E302E375F4457372E330A6C
:102CF000004D61726C696E0020536F66747761726B
:102D0000652052657365740A0020576174636864B6
:102D10006F672052657365740A002042726F776E88
:102D2000206F75742052657365740A0020457874AD
:102D300065726E616C2052657365740A00506F771E
:102D4000657255700A0073746172740A00473238F4
:102D50005859004D31303031006572726F722077F2
:102D6000726974696E6720746F2066696C650A0009
:102D7000446F6E6520736176696E672066696C6565
:102D80002E0A004D323900456E6473746F70730003
:102D900025532025632025632025632025630020FB
:102DA0005A3A0020593A0020583A00656E6473740C
:102DB0006F7073206869743A200070012C019001D3
:102DC0002701B0012201C0011D01F001180110020C
:102DD000130130020E016002090190020401C002D9
:102DE000FF000003FA004003F5008003F000D00369
:102DF000EB002004E6007004E100E004DC00400584
:102E0000D700C005D2004006CD00D006C80080071C
:102E1000C3003008BE00F008B900C009B400B00A11
:102E2000AF00B00BAA00D00CA500000EA000500F00
:102E30009B00C01096005012910000148C00C01529
:102E40008700B0178200B0197D00D01B7800001EEB
:102E5000730040206E0090226900F0246400402737
:102E60005F0090295A00E02B5500102E50002030B2
:102E70004B0010324600E033410090353C001037E3
:102E8000370070383200A0392D00B03A2800A03B3E
:102E90002300603C1E00103D1900903D1400103EC0
:102EA0000F00703E0A00C03E0500003F0000403F9A
:102EB000FBFF803FF6FFC03FF1FF00000A0B020955
:102EC0000C0D0E08070304010000000000000000C4
:102ED00000000000000000000000000000000000F2
:102EE00000000000000012111000000000000000AF
:102EF00000000000000000000000000000000000D2
:102F000050726F62696E67204661696C656400206B
:102F10005A3A200020593A200042656420583A204D
:102F2000003D3D6F6E55736572436F6E6669726DDD
:102F300052657175697265643D3D00220A00556EE7
:102F40006B6E6F776E20636F6D6D616E643A2022D9
:102F5000002042002050006F6B00204500205A00E6
:102F6000205900204D393220580020453A00205A7F
:102F70003A0020593A00583A0020746F6F206C6F65
:102F80006E6720657874727573696F6E20707265F4
:102F900076656E7465640A0020636F6C64206578E2
:102FA00074727573696F6E2070726576656E746584
:102FB000640A0043616E6E6F7420656E74657220E2
:102FC0007375626469723A20004D323520500A4DA3
:102FD000323400526573756D650055492050617536
:102FE0007365004E6F204D61746368203A0050672E
:102FF0005570005067446F776E0049732046696CC6
:103000006520004973204469722000476F55704461
:10301000697200486173204D656469610046696C9E
:10302000656E616D652053656C6563746564004D04
:103030003130303043004D313030300046696C6102
:103040006D656E7420537461742030202D20330020
:1030500046696C616D656E74205374617420302014
:103060002D20320046696C616D656E742053746169
:10307000742030202D2031002046696C616D656E12
:103080007420526573706F6E7365204E6F005265C9
:1030900073756D652059657320647572696E67205C
:1030A0007072696E74000A204E6F2046696C616D03
:1030B000656E7400496E76616C6964204F70746946
:1030C0006F6E004D3530300053746F72652053655C
:1030D0007474696E677300426564205049442053DC
:1030E000746172746564004D3939390A4D32383073
:1030F00050305331363000424C546F756368205263
:1031000065736574004D3530320A4D3530300049F5
:103110006E697420454550524F4D00486F74656E7E
:103120006420504944205374617274656400456E94
:10313000676C69736820416C7265616479205365BE
:1031400074004368696E657365204E6F7420537513
:1031500070706F7274656400496E4C616E6743688D
:103160006F696365000A202A2A2A726563646174A4
:103170002E646174615B305D203D004732380A4740
:1031800031204631303030205A313000556E737561
:1031900070706F72746564204F7074696F6E205325
:1031A000656C6563746564004732365232353500AC
:1031B0004D3139305335350A4732380A4732390AEA
:1031C0004D3430300A4D313034533231350A4732C4
:1031D000380A4D313039533231350A4D343230539B
:1031E000310A47315831303059313030463530307E
:1031F000300A47315A300A4D3530300A4D313137B7
:1032000020536574205A204F6666736574004731F9
:10321000204631303030205A302E30004732380AC4
:103220004731204631303030205A302E30004D3575
:103230003030005A204F6666736574203A2025733B
:10324000004D353030005A204F6666736574203A61
:10325000202573004732380A473146313530305A1D
:10326000302E30004732385A0A4731463135303037
:103270005A302E30004D383400473146313030302E
:103280005A302E30004732380A473146313030301C
:103290005A302E30004D616E75616C536574546503
:1032A0006D70005A204F6666736574203A2025734E
:1032B0000053746F702054726967676572656400AB
:1032C00053746F70204E6F0053746F705072696E3C
:1032D000740048616E646C652044617461204164CF
:1032E0006A75737420322053657474696E67205355
:1032F000637265656E200048616E646C6520446190
:103300007461205072696E7446696C652033205375
:10331000657474696E672053637265656E2000483A
:10332000616E646C652044617461205072696E74D2
:1033300046696C6520322053657474696E6720534A
:10334000637265656E20004D38340048616E646CB0
:10335000652044617461205072696E7446696C65C1
:1033600020506F73740048616E646C652044617412
:1033700061205072696E7446696C652050726500F8
:10338000426567696E537769746368003D3D204309
:103390006865636B6B65793D3D007265636461745C
:1033A0002E61646472203D3D007265636461742E19
:1033B000646174615B305D203D3D007761697477C5
:1033C0006179203D3D0020202A2A2A2A2A2A2A52D1
:1033D00054535F48616E646C65446174612A2A2AA3
:1033E0002A2A2A2A2A2000526573656E643A200030
:1033F00000002200250028002B002E0031003400A0
:1034000002010000050108010B0100002100240059
:1034100027002A002D0030003300010100000401C4
:1034200007010A0105050505070508080808020245
:1034300002020A0A0808040404040101010101014E
:1034400001010303030303030303040707070C0C31
:103450000C0C0C0C0C0C02020202060606060606F8
:1034600006060B0B0B0B0B0B0B0B0102102020089D
:1034700008102040102040800201020108040201CF
:10348000010204081020408080402010080402013E
:103490008004020180402010080402010804020197
:1034A000010204081020408001020408102040801E
:1034B000444458203130532050726F20526561646B
:1034C000792E005072696E74696E672E2E2E005030
:1034D00072696E7420506175736564006E6F7469F3
:1034E0006669636174696F6E2000504944205475A9
:1034F0006E652046696E697368656400C4000201E8
:1035000011241FBECFEFD1E2DEBFCDBF00E00CBF64
:1035100014E0A0E0B2E0EEE9FFE502E00BBF02C07C
:1035200007900D92A430B107D9F726E1A4E0B4E0EA
:1035300001C01D92A033B207E1F71AE1CFE7DAE14B
:1035400000E006C021970109802FFE010F94FC2B9B
:10355000CE37D10780E00807A9F70F9473190D94AF
:10356000BD2F0C9400009F92AF92BF92CF92DF923A
:10357000EF92FF920F931F93CF93DF9300D01F9290
:103580001F92CDB7DEB7EDE5FBE10027BB27462F45
:10359000572FA82FAA2341F4A52F542FB85FAA2391
:1035A00019F4A52F5527B85FA03138F45295A2958C
:1035B000452F4F70507FA42BBC5FA03428F4550FCB
:1035C000AA1F550FAA1FBE5FA03818F4550FAA1FD7
:1035D000B395550FAA1FEA0FF01F449151E0AA2797
:1035E000B85081F1C8F0B0FF02C0440F551FB1FFC1
:1035F00004C0440F551F440F551FB2FF06C052951B
:103600004295142F1F70407F512BB3FF1BC0A52F75
:10361000542F44270C94221BB195B0FF02C055953E
:103620004795B1FF04C05595479555954795B2FF0D
:1036300005C05295407F4295452B5F70B3FF02C095
:10364000452F5527DD24CC24BB24B2E0649FD0183D
:10365000C108B00AB00B749FC018B108B00B849FAA
:10366000B018B109659FC018B108B00B759FB018AC
:10367000B109859FB0196A9FB018B1097A9FB01936
:103680004D9DA12C99243327992722275D9DA00CBD
:10369000911C301F901F201FAD9D900C311D901F5D
:1036A000201F4C9DA00C911C301F901F201F5C9D63
:1036B000900C311D901F201FAC9D300D911D201FBF
:1036C0004B9D900C311D901F201F5B9D300D911D57
:1036D000201FAB9D900D211D4B9F300D911D201F74
:1036E0005B9F900D211DAB9F200DB1E0BB24CC242E
:1036F000DD24639FD018C108B00AB00B739FC018B7
:10370000B108B00B839FB018B109699FC018B10808
:10371000B00B799FB018B109899FB019629FB0189A
:10372000B109729FB019D61AC70AB80A20F0B1E0E1
:103730003B0F901F201F1124792F632F90E0822FC1
:103740000F900F900F900F900F90DF91CF911F91DE
:103750000F91FF90EF90DF90CF90BF90AF909F9030
:103760000895AF92BF92CF92DF92EF92FF920F93A4
:103770001F93CF93DF93CEE3DCE00DEE18E08EE4F1
:10378000A82E8CE0B82EC12CD12C7601C39469915F
:103790007991899199910F943A25288939894A8993
:1037A0005B890F949B250F94782DF8016193719399
:1037B000819391938F01C616D706E806F90610F497
:1037C0006B017C01AC16BD0611F76FEF7FEFCB01EB
:1037D000A70196010F94792B2093FD083093FE08E2
:1037E0004093FF0850930009DF91CF911F910F91F3
:1037F000FF90EF90DF90CF90BF90AF900895CF9261
:10380000DF92EF92FF928091F907882309F457C065
:10381000C090F507D090F607E090F707F090F80712
:1038200020E030E0A901C701B6010F9435258823B7
:1038300009F445C020E030E040E05FE3C701B60195
:103840000F949B259B01AC010F949B252BED3FE032
:1038500049E450E40F949B259B01AC0160E070E0CB
:1038600080E89FE30F94FF2C6B017C01C0923A0C1F
:10387000D0923B0CE0923C0CF0923D0C60916502C2
:1038800070916602072E000C880B990B0F943C2553
:103890002AE037ED43E25CE30F949B25A7019601F4
:1038A0000F949B2560936102709362028093630280
:1038B00090936402FF90EF90DF90CF900895C12C19
:1038C000D12C80E8E82E8FE3F82ED0CF0F931F93F2
:1038D000CF93DF9350E0FC01E40FF51F8081440F8C
:1038E000551F440F551F41565A4FEA01882329F1AD
:1038F00088819981AA81BB81EB01088119812A8184
:103900003B810097A105B10569F40C591F4F2F4F5A
:103910003F4FDA010D931D932D933C9313978FEF37
:10392000808306C0081B190B2A0B3B0B37FDF7CF12
:10393000DF91CF911F910F910895188219821A82F9
:103940001B82F6CFCF93DF9324E0829FC001112426
:10395000EC01C053D74FFC01EA5FF74F8650984FF8
:10396000DC012D913D914D915C916081718182814D
:1039700093810F94052C688379838A839B83DF91DD
:10398000CF91089580919A0590919B05A0919C05F7
:10399000B0919D058093410290934202A09343020F
:1039A000B093440280919805909199059093680294
:1039B0008093670208958091410290914202A09104
:1039C0004302B091440280939A0590939B05A09383
:1039D0009C05B0939D058091670290916802909339
:1039E00099058093980584E690E09093680280930F
:1039F000670208958091891290918A12891B8770BD
:103A000089F48091910D81110DC08091860C909167
:103A1000870C892B39F481E09091A806911103C09D
:103A200080E0089581E00895CF93DF93DB01F901F1
:103A30009C919130C1F0943080F094509C938830E8
:103A4000D1F480819181009771F0019791838083F7
:103A5000480F591FEA01188206C08C3539F49C5F63
:103A60009C93943041F4DF91CF9108958B3339F7D3
:103A700081E08C93F8CF20813181B9016F5F7F4F56
:103A800071836083420F531FEA0188838081918193
:103A90008F3591056CF7E7CF0F931F9381E000916D
:103AA0002D1410912E1420912F1430913014409128
:103AB000291450912A1460912B1470912C1404171E
:103AC00015072607370708F480E01F910F91089526
:103AD00090E080E00895282F9091F407833021F43E
:103AE00095FD0FC094FD0FC0892F90E0B0E0A0E0DD
:103AF00004C0B695A795979587952A95D2F78170BA
:103B0000089581E0089580E00895FC016591759124
:103B10008591949108958F929F92AF92BF92CF9288
:103B2000DF92EF92FF92CF93DF93EC018090CC086D
:103B30009090CD08A090CE08B090CF0820E030E063
:103B4000A901C501B4010F943525882309F454C097
:103B5000C880D980EA80FB80A7019601C501B40125
:103B60000F94352518160CF04CC02091C4083091E4
:103B7000C5084091C6085091C708C701B6010F9407
:103B80003525882331F1C092C408D092C508E0924F
:103B9000C608F092C7082091C8083091C908409122
:103BA000CA085091CB08688179818A819B810F94E2
:103BB0009B259B01AC0160E070E080E89FE30F94DF
:103BC000042C60930F027093100280931102909363
:103BD000120260910F027091100280911102909177
:103BE0001202DF91CF91FF90EF90DF90CF90BF90C6
:103BF000AF909F908F90089560E070E080E89FE321
:103C0000F0CF60E070E0CB01ECCFCF92DF92EF928B
:103C1000FF92CF93DF93EC01CC80DD80EE80FF80BC
:103C200027E137EB41ED58EBC701B6010F94652E44
:103C300087FD23C023E030E04BE953E4C701B60120
:103C40000F9435251816CCF0C880D980EA80FB8007
:103C500027E137EB41ED58EBC701B6010F94652E14
:103C600087FD0BC0C1E023E030E84DE953E4C70114
:103C7000B6010F94352518160CF4C0E08C2FDF9197
:103C8000CF91FF90EF90DF90CF9008952FEB280F0A
:103C90002A3108F047C0E22FF0E08091370590917B
:103CA0003805A0913905B0913A0504C0B695A7959D
:103CB000979587952A95D2F780FD02C08170089567
:103CC000E75EFA4FE081EE2341F180918607909103
:103CD0008707E80FF92FF11D808190ED980F9A303A
:103CE00030F08E3251F4818180538A3098F4F09311
:103CF0000805E093070581E008958D3211F08B32BD
:103D000049F4818190ED980F9A3088F38E3211F446
:103D10008281EACFF0E0E0E0EACF1092080510924D
:103D20000705E9CF80E008950E94461E882341F0F0
:103D300081E02091070530910805232B09F480E0EC
:103D400008958F929F92AF92BF92CF92DF92EF929F
:103D5000FF92C090D605D090D705E090D805F0909E
:103D6000D90520E030E0A901C701B6010F9435253F
:103D70008823E1F1A701960160E070E080E89FE30D
:103D80000F94FF2C6B017C018090DA059090DB058D
:103D9000A090DC05B090DD0520E030E0A901C50170
:103DA000B4010F943525882329F1A501940160E021
:103DB00070E080E89FE30F94FF2CC092E004D09263
:103DC000E104E092E204F092E3046093E40470936F
:103DD000E5048093E6049093E704FF90EF90DF9072
:103DE000CF90BF90AF909F908F900895C12CD12C11
:103DF0007601CACF60E070E0CB01DFCF129A089560
:103E00005F9A8091380C8E7F8093380C8A9A8091CB
:103E1000380C8D7F8093380C8091080180958170DB
:103E2000809306018091380C8B7F8093380C0C9422
:103E3000FE1E269A2E9A08958C3221E0920714F0E5
:103E40008CE291E09093EE118093ED110C941AFDA9
:103E5000E2E1F6E0108211821282138214820C9445
:103E60001AFD4F925F926F927F928F929F92AF92C4
:103E7000BF92CF92DF92EF92FF920F931F93CF9357
:103E8000DF93EC012091CE053091CF054091D00514
:103E90005091D105688179818A819B810F94042C8E
:103EA0006B017C012091D2053091D3054091D4055E
:103EB0005091D5056C817D818E819F810F94042C5A
:103EC0004B015C01A701960160910302709104020D
:103ED00080910502909106020F943525882309F4FC
:103EE00050C0C0920302D0920402E0920502F09208
:103EF00006022091E0043091E1044091E2045091E7
:103F0000E304C701B6010F949B252B013C010F94DC
:103F1000A72D6B017C0120E030E0A9010F9435252D
:103F200087FD70C020E030E040E450E4C701B601F6
:103F30000F94652E18162CF4C12CD12CC0E4EC2E55
:103F4000FE2CA7019601C301B2010F94042C6093CB
:103F5000D8047093D9048093DA049093DB04C701EA
:103F6000B6010F94712D6093D604062E000C770BCA
:103F70006F5F7F4F6430710514F064E070E0609310
:103F8000D404D09101021091D604A501940160914E
:103F90000702709108028091090290910A020F9421
:103FA0003525811133C0D11381C02091BC043091DB
:103FB000BD044091BE045091BF046091D80470913B
:103FC000D9048091DA049091DB040F949B25209111
:103FD000C0043091C1044091C2045091C3040F94B5
:103FE000052CDF91CF911F910F91FF90EF90DF9003
:103FF000CF90BF90AF909F908F907F906F905F9089
:104000004F900895C12CD12C76019BCF809207024E
:1040100090920802A0920902B0920A022091E40450
:104020003091E5044091E6045091E704C501B401E4
:104030000F949B254B015C010F94A72D6B017C0114
:1040400020E030E0A9010F94352587FDF3C020E082
:1040500030E040E450E4C701B6010F94652E181615
:104060002CF4C12CD12CB0E4EB2EFE2CA701960130
:10407000C501B4010F94042C6093DC047093DD043B
:104080008093DE049093DF04C701B6010F94712D75
:104090006093D704062E000C770B6F5F7F4F643060
:1040A000710514F064E070E06093D504C091D7040A
:1040B000D11305C0809102028C1709F470C0809161
:1040C000D6049091D70490930202809301020C2EA3
:1040D000000CDD0B25E01203C0011124FC01EC0FE4
:1040E000FD1FEE0FFF1FEE0FFF1FE057F84F20815F
:1040F0003181428153812093D0043093D104409385
:10410000D2045093D3040091D504002E000C110B5F
:10411000FC01E00FF11FEE0FFF1FEE0FFF1FE05736
:10412000F84F60817181828193810F94042C609398
:10413000CC047093CD048093CE049093CF0420914F
:10414000D40435E02303F0011124CE0FDF1FCC0F80
:10415000DD1FCC0FDD1FC057D84F288139814A8120
:104160005B812093C8043093C9044093CA045093E0
:10417000CB04E00FF11FEE0FFF1FEE0FFF1FE05704
:10418000F84F60817181828193810F94042C609338
:10419000C4047093C5048093C6049093C7048090B0
:1041A000DC049090DD04A090DE04B090DF04209148
:1041B000CC043091CD044091CE045091CF04C50180
:1041C000B4010F949B252091D0043091D1044091EB
:1041D000D2045091D3040F94052C6B017C01C09242
:1041E000C004D092C104E092C204F092C3042091B2
:1041F000C4043091C5044091C6045091C704C50160
:10420000B4010F949B252091C8043091C9044091BA
:10421000CA045091CB040F94052CA70196010F946A
:10422000042C6093BC047093BD048093BE049093EF
:10423000BF04BBCEC12CD12C760118CFCF92DF9218
:10424000EF92FF92CF93DF93EC0108960E948B1DB3
:104250006B017C0120E030E0A9010F94352520E0BE
:1042600030E0A901882359F0CE010E94311F9B0143
:10427000AC01C701B6010F949B259B01AC01688579
:1042800079858A859B850F94042C688779878A872E
:104290009B87DF91CF91FF90EF90DF90CF900895B3
:1042A0002F923F924F925F926F927F928F929F9246
:1042B000AF92BF92CF92DF92EF92FF920F931F9334
:1042C000CF93DF93D62FC72FFC0180809180A280EF
:1042D000B380C501B40120E831E541E050E00F941E
:1042E000792BC9016DE671E00F94E82B6B017C011D
:1042F000C501B40120E13EE040E050E00F94792B8D
:10430000CA01B90128E130E040E050E00F94792B78
:10431000362E272E062F172F8CE3482E512C612C7A
:10432000712CC501B401A30192010F94792BB62E13
:10433000A72ECA01B901A30192010F94792BCB01D9
:10434000C114D10479F1AF92BF927F936F932F92F2
:104350003F92FF92EF92DF92CF9284E697E19F9394
:104360008F93CF93DF930F94CC248DB79EB70E9687
:104370000FB6F8949EBF0FBE8DBF8D2F9C2FDF917F
:10438000CF911F910F91FF90EF90DF90CF90BF9052
:10439000AF909F908F907F906F905F904F903F90E5
:1043A0002F900895E114F104C9F0AF92BF927F936A
:1043B0006F932F923F92FF92EF9284E597E19F9344
:1043C0008F93CF93DF930F94CC24EDB7FEB73C9639
:1043D0000FB6F894FEBF0FBEEDBFCFCF012BB9F0E3
:1043E000AF92BF927F936F932F923F9288E497E1B1
:1043F0009F938F93CF93DF930F94CC248DB79EB769
:104400000A960FB6F8949EBF0FBE8DBFB6CF892B0C
:10441000A9F0AF92BF927F936F9380E497E19F934F
:104420008F93CF93DF930F94CC24EDB7FEB73896DC
:104430000FB6F894FEBF0FBEEDBF9FCFAF92BF92F5
:104440008CE397E19F938F93CF93DF930F94CC24CA
:104450000F900F900F900F900F900F908ECFEF92C4
:10446000FF920F931F93CF93DF93CDB7DEB78C01ED
:10447000EDB6FEB60F94822401962DB73EB7281BE9
:10448000390B0FB6F8943EBF0FBE2DBF8DB79EB748
:104490000196B8010F947B240E943DF90FB6F89461
:1044A000FEBE0FBEEDBEDF91CF911F910F91FF9029
:1044B000EF9008958C38910514F08CE890E090937B
:1044C0008311809382110C9494BEAB01BC01409384
:1044D0002D1450932E1460932F147093301485E98B
:1044E00095E10C944CAF2F923F924F925F926F9256
:1044F0007F928F929F92AF92BF92CF92DF92EF9274
:10450000FF920F931F93CF93DF93CDB7DEB76097E2
:104510000FB6F894DEBF0FBECDBF8B876C87042F1C
:10452000122F282F30E03E872D87462F50E05A87E4
:10453000498785E0982E929EC001939E900D11248C
:10454000988B8F87FA01E80FF91FEE0FFF1FEE0F10
:10455000FF1FE057F84F60817181828193819B0139
:10456000AC010F94F72E882309F445C14B85400F09
:104570006C85610F949EC0011124E985FA85E80FCE
:10458000F91FEE0FFF1FEE0FFF1FE057F84FC0801F
:10459000D180E280F380040F909EA0011124E98570
:1045A000FA85E40FF51FEE0FFF1FEE0FFF1FE05718
:1045B000F84F0081918082807380262F30E0EF8554
:1045C000F889E20FF31FEE0FFF1FEE0FFF1FE057FA
:1045D000F84F20807181798372817A8373817B8324
:1045E000610F70E0EF85F889E60FF71FEE0FFF1FF0
:1045F000EE0FFF1FE057F84FF88BEF87F081FC8339
:10460000EF85F889F181FD83EF85F889F281FE83DA
:10461000EF85F889F381FF83FC01E20FF31FEE0FB2
:10462000FF1FEE0FFF1FE057F84F20812887A18062
:10463000B2806380FA01E60FF71FEE0FFF1FEE0F47
:10464000FF1FE057F84F4080518032801381202FA8
:10465000392D482D572D602F792D882D972D0F94AA
:10466000F72E882321F000E0912C812C712C9601EB
:10467000A701B601C7010F94F72E882321F0C02EA1
:10468000D92CE82CF72C2C813D814E815F816C81E7
:104690007D818E819F810F94F72E882321F01C82CB
:1046A0001D821E821F82222D39814A815B81622DEB
:1046B00079818A819B810F94F72E882339F02C8091
:1046C0003D8139834E814A835F815B839201432D13
:1046D000512FB201832D912F0F94F72E882321F0B3
:1046E000412C512C312C10E028853A2D4B2D562D84
:1046F00068857A2D8B2D962D0F94F72E882321F027
:104700004886A52CB32C612E85E02D853E85829FA1
:10471000F001839FF00D112449855A85E40FF51FA0
:10472000EE0FFF1FEE0FFF1FE057F84FFA87E987E4
:104730009601A701B601C7010F94052C202F392D32
:10474000482D572D0F94042C6B017C01222D3981AB
:104750004A815B81622D79818A819B810F94052C2E
:104760002C813D814E815F810F94042C9B01AC0113
:10477000C701B6010F94052C6B017C0128853A2DE9
:104780004B2D562D68857A2D8B2D962D0F94052C4B
:104790009201432D512F0F94042C9B01AC01C701B2
:1047A000B6010F94052C20E030E040E450E40F9473
:1047B000FF2CE985FA8560837183828393836C85FE
:1047C0008B8560960FB6F894DEBF0FBECDBFDF912C
:1047D000CF911F910F91FF90EF90DF90CF90BF90FE
:1047E000AF909F908F907F906F905F904F903F9091
:1047F0002F900C94D0F760960FB6F894DEBF0FBEE2
:10480000CDBFDF91CF911F910F91FF90EF90DF907F
:10481000CF90BF90AF909F908F907F906F905F9060
:104820004F903F902F900895809107059091080533
:10483000009731F04AE050E070E060E00D945023C2
:1048400060E070E0CB010895809107059091080524
:10485000009731F04AE050E070E060E00D942222D1
:1048600060E070E0CB010895CF93DF93EB010E94ED
:10487000941E882319F00E942424EB01CE01DF91BD
:10488000CF9108950E94242497FD0CC00E942424F7
:104890006F3F71058105910509F034F40E942424CD
:1048A000862F089580E008958FEF0895CF93C62F47
:1048B0000E94941E882319F0CF910C9442248C2FCF
:1048C000CF9108958091070590910805892B41F0BB
:1048D0000E94422491E0811101C090E0892F089547
:1048E00091E0FCCFCF93DF93C82FD62F0E94941E68
:1048F000882321F0DF91CF910C9462248C2F0E94A9
:10490000461E811101C08D2FDF91CF9108950E9425
:104910002424CB010895CF93DF93EB010E94941ED2
:10492000882321F0DF91CF910C948724CE01DF9171
:10493000CF9108950F931F93CF9380910705909186
:1049400008050097E9F0FC018F01C1912C2F2F7D04
:1049500081F0C53411F0C536B9F7F801108270E066
:1049600060E00F94C420F801C083CF911F910F9194
:10497000089570E060E0CF911F910F910D94C420D5
:1049800060E070E0CB01F1CFCF92DF92EF92FF9227
:104990006A017B010E94941E882331F0FF90EF9002
:1049A000DF90CF900C949A24C701B601FF90EF904E
:1049B000DF90CF9008954F925F926F927F928F9287
:1049C0009F92AF92BF92CF92DF92EF92FF921F938E
:1049D000CF93DF9300D01F92CDB7DEB719821A8232
:1049E0001B821C82CE0101964C0184E7C82E87E011
:1049F000D82E98E2E92E9CE0F92E20EDA22E28E098
:104A0000B22E10E088E5810F0E94941EF40181937C
:104A10004F01882309F4E0C00E949A242B013C0135
:104A2000812F0E946B1D882309F4CCC0F7012081DF
:104A3000318142815381C301B2010F94052CF601EB
:104A400060837183828393831F5FF4E0CF0ED11C58
:104A500084E0E80EF11C94E0A90EB11C133091F62D
:104A600085E40E94941E8C83882309F4C0C00E94B0
:104A70009A246B017C0183E00E946B1D882371F0F6
:104A80002091340C3091350C4091360C5091370CFC
:104A9000C701B6010F94052C6B017C01C092800701
:104AA000D0928107E0928207F09283078091CD0532
:104AB000882359F18091311482FF27C08C8188238B
:104AC00021F18981811103C08A818823F1F02DECC5
:104AD0003CEC4CE45DE360911B0870911C088091F4
:104AE0001D0890911E080F94052C9B01AC0160914C
:104AF000300C7091310C8091320C9091330C0F94EA
:104B0000652E181614F40E9416F740E050E0BA0122
:104B100086E40E94C42420E030E0A9010F94652EB1
:104B2000181684F40E949A2420E030E040E752E412
:104B30000F94FF2C609341027093420280934302D2
:104B4000909344028091E60B83FD28C080919306E8
:104B5000882321F12091340C3091350C4091360C92
:104B60005091370C60918007709181078091820786
:104B7000909183070F94042C2091A0063091A106F8
:104B80004091A2065091A3060F94052C6093A006B5
:104B90007093A1068093A2069093A3060F900F90A6
:104BA0000F900F90DF91CF911F91FF90EF90DF90CA
:104BB000CF90BF90AF909F908F907F906F905F90BD
:104BC0004F900895F5012081318142815381C301C5
:104BD000B2010F94042C33CFF70180819181A2811F
:104BE000B381F60180839183A283B3832DCF80911B
:104BF000340C9091350CA091360CB091370C809309
:104C0000800790938107A0938207B09383074ECFCC
:104C1000CF92DF92EF92FF926B017C0183E3C81683
:104C2000D104E104F10470F082E3C81AD108E1086C
:104C3000F10862E370E080E090E00E94DBFC0E94FB
:104C40000EC2ECCFC701B6010E94DBFCFF90EF90D3
:104C5000DF90CF900C940EC2CF92DF92EF92FF9232
:104C60000F931F93CF93DF936B017A01EC01C4562E
:104C7000DB4F28813CE0389F8001399F100D1124C3
:104C800027FF24C0FB011182108288818F5F8883F7
:104C900088819801280F311D87FD3A95C90120911F
:104CA0007412F6012817190629F024F088818C3037
:104CB0000CF43CC080819181049680349C4908F4B6
:104CC00075C0F60180819181049672C08881980137
:104CD000280F311D87FD3A95C901209174122817BC
:104CE000190699F294F28881A801480F511D87FD99
:104CF0005A95FA01EE0FFF1FE40FF51FE45DFD4E1C
:104D0000808187FFC2CF8881F801E80FF11D87FD00
:104D1000FA95CF01EE0FFF1FE80FF91FE45DFD4E7E
:104D2000808160E08F770E9479FBAFCF8081918195
:104D30002881A801420F511D27FD5A959A01FA01B9
:104D4000EE0FFF1FE20FF31FE45DFD4E2181328164
:104D5000820F931FF7019183808388819801280F28
:104D6000311D87FD3A95F901EE0FFF1FE20FF31F8A
:104D7000E45DFD4E808187FF20C08881080F111DF2
:104D800087FD1A95F801EE0FFF1FE00FF11FE45D9C
:104D9000FD4E808161E08F77DF91CF911F910F9160
:104DA000FF90EF90DF90CF900C9479FB80E49CE92A
:104DB000F701918380838FEF8883DF91CF911F91DB
:104DC0000F91FF90EF90DF90CF9008950F931F9376
:104DD000CF93DF9302E51CE0C6E6D1E1F801219113
:104DE0003191419151918F0160E070E080E89FE343
:104DF0000F94FF2C6993799389939993F1E1C637C6
:104E0000DF0761F70E9455F5DF91CF911F910F9158
:104E10000C94B11BCF92DF92EF92FF92CF93DF936E
:104E20002091390C222329F1EC0108960E948B1D58
:104E30006B017C0120E030E0A9010F94352520E0D2
:104E400030E0A901882359F0CE010E94311F9B0157
:104E5000AC01C701B6010F949B259B01AC0168858D
:104E600079858A859B850F94052C688779878A8741
:104E70009B87DF91CF91FF90EF90DF90CF900895C7
:104E80002F923F924F925F926F927F928F929F925A
:104E9000AF92BF92CF92DF92EF92FF920F931F9348
:104EA000CF93DF93CDB7DEB76C970FB6F894DEBF24
:104EB0000FBECDBF8C015B015A834983FC01EA5BC5
:104EC000FF4F208131814281538129873A874B8767
:104ED0005C87CA01B9010F943A256B017C01D501A9
:104EE0002D913D914D915C910F949B250F94E32C56
:104EF0002B013C01E981FA8120813181428153817A
:104F0000C701B6010F949B250F94E32C4B015C0164
:104F1000C301B2010F94782D698B7A8B8B8B9C8B9C
:104F2000683771058105910540F428E730E040E0DD
:104F300050E0298B3A8B4B8B5C8BC501B4010F94ED
:104F4000782D6D877E878F87988B683771058105EF
:104F5000910540F448E750E060E070E04D875E87DF
:104F60006F87788BF801EE5AFF4F40805180628046
:104F70007380C301B2010F943C2569837A838B83CC
:104F80009C8369897A898B899C890F943A256D8BDA
:104F90007E8B8F8B988F20E030E0A90169817A8128
:104FA0008B819C810F943525882309F4E1C1A701E9
:104FB0009601C701B6010F949B254B015C012D8919
:104FC0003E894F89588DCA01B9010F949B259B01D9
:104FD000AC01C501B4010F94042C4B015C01298183
:104FE0003A814B815C81CA01B9010F94052C9B0168
:104FF000AC01C501B4010F94FF2C0F94E32C0F9466
:10500000782D6D837E838F83988766277727CB01E2
:1050100064197509860997090F943C254B015C01B9
:105020006D857E858F8598890F943A252B013C01EB
:1050300020E030E0A901C501B4010F943525882393
:1050400009F49AC1A3019201C301B2010F949B25F7
:10505000698F7A8F8B8F9C8FA7019601C701B6014C
:105060000F949B259B01AC01698D7A8D8B8D9C8D56
:105070000F94042C6B017C01A5019401C501B401BE
:105080000F94052C9B01AC01C701B6010F94FF2CB6
:105090000F94A72DD80195968D909D90AD90BC90C2
:1050A0009897750164012D813E814F815885C21A00
:1050B000D30AE40AF50A0F94782DC61AD70AE80A2B
:1050C000F90AF7FE8EC02D893E894F89588DCA0195
:1050D000B9010F949B256B017C0129813A814B8199
:1050E0005C81CA01B9010F94052C69877A878B8787
:1050F0009C8720E030E0A90169817A818B819C81C5
:105100000F943525882309F43BC1C501B4010F94E0
:105110003A2529853A854B855C850F949B25A70107
:1051200096010F94042C6D837E838F839887A3014F
:105130009201C301B2010F949B259B01AC016D81CB
:105140007E818F8198850F94052C2B013C0120E0F6
:1051500030E040E850E469817A818B819C810F9432
:105160009B259B01AC01C301B2010F94FF2C0F944E
:10517000E32C2B013C0120E030E0A9010F94652EC7
:1051800018161CF0412C512C3201C301B2010F94AE
:10519000782D6D837E838F83988786169706A80661
:1051A000B90620F48D829E82AF82B8866D817E81A1
:1051B0008F8198850F943A2529853A854B855C85A2
:1051C0000F949B25A70196010F94052C0F94B32EE5
:1051D0000F94782D69877A878B879C87C12CD12C77
:1051E000760169857A858B859C8529893A894B89E1
:1051F0005C89621B730B840B950B0F943A252981F4
:105200003A814B815C810F94FF2C20E034E244EF23
:1052100059E40F949B250F94782D4B015C0169850F
:105220007A858B859C852D853E854F855889621BA7
:10523000730B840B950B0F943A2529813A814B818E
:105240005C810F94FF2C20E034E244EF59E40F948A
:105250009B250F94782D2B013C013FE6831691048A
:10526000A104B10408F090C0F401EE0FFF1FEE0F8F
:10527000FF1FEF55F64E85919591A591B4918983C5
:10528000292E3A2EBD8B4FE6441651046104710459
:1052900008F083C0F201EE0FFF1FEE0FFF1FEF5566
:1052A000F64E45915591659174919A01CB014D81CE
:1052B0005E816F817885D80199964D935D936D934A
:1052C0007C939C974C0D5D1D6E1D7F1DF80145A7BD
:1052D00056A767A770ABE65BFF4F49895A896B8970
:1052E0007C894083518362837383D5968D929D928E
:1052F000AD92BC92D897F80141AE52AE63AE74AE97
:10530000FD9649814083218232825D8953833496A0
:10531000208331838283938369857A858B859C85FD
:10532000D1966D937D938D939C93D4973D962D85C7
:105330003E854F85588920833183428353836C9601
:105340000FB6F894DEBF0FBECDBFDF91CF911F9196
:105350000F91FF90EF90DF90CF90BF90AF909F9014
:105360008F907F906F905F904F903F902F90089517
:1053700060E070E0CB0141CE60E070E0CB0188CE10
:1053800060E070E0CB01F3CEC501B4010E94B31A16
:105390006983272E382E9D8B76CFC301B2010E94E0
:1053A000B31A9B0184CF8091891290918A12891B34
:1053B000877019F490E080E0089590918612992307
:1053C00051F0833030F48FEF890F19F080938612FB
:1053D000F1CF1092861280918A122CE5829FC00133
:1053E00011248A5F964FFC01208120FDE3CF20919C
:1053F0008A122F5F27702093871230918A12209192
:105400008812321304C020918712209388120895C5
:1054100090916F0081E091FD02C080E0089590912D
:105420006F009D7F90936F00089580FF04C090915E
:105430009E0590FD8E7F81FF05C090919E059695FB
:1054400090FD8D7F82FF06C090919E059695969562
:1054500090FD8B7F08958F929F92AF92BF92CF92D3
:10546000DF92EF92FF92CF93DF93209145022223A8
:1054700009F49EC0EC0180919E05C82ED12CF12C20
:10548000E12C80FF2CC08090470290904802A090B1
:105490004902B0904A02288139814A815B81C50165
:1054A000B4010F94652E181624F488829982AA827A
:1054B000BB828090530290905402A0905502B0900D
:1054C0005602288139814A815B81C501B4010F945C
:1054D000352587FF04C088829982AA82BB82D701C2
:1054E000C601B695A7959795879580FF2CC08090AB
:1054F0004B0290904C02A0904D02B0904E022C8135
:105500003D814E815F81C501B4010F94652E18164F
:1055100024F48C829D82AE82BF828090570290904C
:105520005802A0905902B0905A022C813D814E81C0
:105530005F81C501B4010F94352587FF04C08C82BB
:105540009D82AE82BF8282E0F694E794D794C7949E
:105550008A95D1F7C0FE2CC0C0904F02D090500267
:10556000E0905102F0905202288539854A855B858A
:10557000C701B6010F94652E181624F4C886D98683
:10558000EA86FB86C0905B02D0905C02E0905D02F0
:10559000F0905E02288539854A855B85C701B60192
:1055A0000F94352587FF04C0C886D986EA86FB8616
:1055B000DF91CF91FF90EF90DF90CF90BF90AF90B1
:1055C0009F908F900895CF92DF92EF92FF920F936A
:1055D0001F93C12CD12C76018C0124E33CE040E3E5
:1055E0005CE06CE27CE088E29CE00E9451F41F9158
:1055F0000F91FF90EF90DF90CF9008950C9455F5A8
:105600008091A506811105C080918407882309F443
:1056100063C080918B05659B59C0816080938B0529
:105620009091030180918B0591FF52C0826080931D
:105630008B0580918B054B9B4DC0846080938B05BF
:105640008091F20580FF10C08091A60680FF0CC0FB
:1056500080918B0580FF08C08091E806816080936F
:10566000E80680E00E946EC68091F205869580FF74
:1056700011C08091A606869580FF0CC080918B0595
:1056800081FF08C08091E80682608093E80681E08F
:105690000E946EC68091F2058695869580FF1CC09B
:1056A0008091A6068695869580FF16C08091840716
:1056B000882391F080918B0582FF0EC08091E806CF
:1056C00084608093E80682E00C946EC68E7FA6CF3D
:1056D0008D7FADCF8B7FB2CF08958091A5068111CC
:1056E00004C080918407882331F062E070E080E09C
:1056F00090E00C94082608950F931F938091241135
:10570000813019F50E940EFD0091A7051091A805A2
:105710002091A9053091AA05601B710B820B930B98
:1057200028EE33E040E050E00F94792B6091AB0518
:105730007091AC058091AD059091AE05620F731F1D
:10574000841F951F1F910F9108956091AF0570916F
:10575000B0058091B1059091B205D6CF1092241179
:105760001092A7051092A8051092A9051092AA05FB
:105770001092AF051092B0051092B1051092B205CB
:105780001092AB051092AC051092AD051092AE05CB
:105790000895CF92DF92EF92FF92CF93DF93C62FBF
:1057A000FC01C080D180E280F38020E030E0A901DC
:1057B000C701B6010F94352520E030E0A90187FD2F
:1057C00014C020E030E048EC52E4C701B6010F9469
:1057D000652E24E630E040E050E0181634F0C701B2
:1057E000B6010F94712D9B01AC01C230A0F4D0E042
:1057F000CF5FD64FAFEFB0E00F94BA2B24E630E086
:1058000040E050E00F949B2B2F3F310519F010F032
:105810002FEF30E02883DF91CF91FF90EF90DF9062
:10582000CF9008958091090180FD06C080913114C8
:1058300083FB882780F9089580E00895CF92DF9256
:10584000EF92FF92FC01C080D180E280F38066304D
:1058500019F5109217061092180610921906109258
:105860001A0610921B060E9494BE20E030E0A901A7
:10587000C701B6010F94352587FF1DC0C12CD12C5F
:105880007601C701B6010F94722ECB01FF90EF9005
:10589000DF90CF900C945A220E94281F20E030E025
:1058A000A901C701B6010F94352587FF15C0C12C8A
:1058B000D12C760121C020E030E04CE053E4C70158
:1058C000B6010F94652E1816E4F6C12CD12C9CE07D
:1058D000E92E93E4F92ED5CF20E030E046E953E4F9
:1058E000C701B6010F94652E181634F4C12CD12CC3
:1058F00086E9E82E83E4F82EC701B6010F94722ED4
:10590000CB01FF90EF90DF90CF900C941C1F9091F3
:10591000380C977081E0973009F080E0089520916D
:10592000890520FF14C020E83EE3629FA001639F29
:10593000500D729F500D1124CA019695879596952A
:105940008795009731F08A950000E9F708950C9447
:1059500008260895CF93DF931092E70B10928A0CDC
:1059600010928C0C10928B0C109288051092870567
:10597000CFEFDFEF8091311485FD07C00E94ADAA03
:10598000D093B012C093AF12F5CF8FEF9FEF9093EB
:10599000B0128093AF12DF91CF9108958F929F92B2
:1059A000AF92BF92CF92DF92EF92FF920F931F932D
:1059B000CF93DF9310923C0510923B052FE3209389
:1059C0003605109235051092340510923305109269
:1059D0003705109238051092390510923A059C014E
:1059E000F90190812F5F3F4F9032D1F39E34C9F47B
:1059F000818190ED980F9A3020F08D3211F08B322A
:105A000081F432969F012F5F3F4F808180538A300F
:105A100008F47BC09F012F5F3F4F8081803209F4E3
:105A200076C0F0938707E09386078F010F5F1F4FC3
:105A3000C0816AE270E0C8010F94532F009731F0E3
:105A4000FC01319780818032E1F31182CD3429F05D
:105A5000C43519F0C73409F04BC0F80180810F5FDD
:105A60001F4F8032D1F380538A3008F041C0C09379
:105A7000360530E020E04AE0DF011196429FC00188
:105A8000439F900D11249C01205331098081280FE0
:105A9000311D87FD3A95818190ED980F9A30C8F1BC
:105AA00030933505209334058E3261F4329690E0C0
:105AB0004AE0DF0131968C9150ED580F5A3058F181
:105AC00090933305CD01DC0101964C914032D9F31E
:105AD000CD3489F52E31310539F018F527313105EE
:105AE00019F02C31310539F5B0933C05A0933B05F5
:105AF000DF91CF911F910F91FF90EF90DF90CF90AA
:105B0000BF90AF909F908F900895F9017BCFF901DE
:105B100081CFFD01B1CF949F800D112490ED980F9E
:105B2000C8CF2537310538F027373105E8F2203A5C
:105B300083E03807C9F2D091860740E050E0BA010F
:105B400010E000E0C12CD12C7601C394FD01319608
:105B50008C91882309F47FC08132E1F4CD34D1F4F3
:105B600020323105B9F440933705509338056093DE
:105B7000390570933A05F0933C05E0933B0563E2E9
:105B800070E0CF010F94532F009709F4B1CFFC01BF
:105B90001082AECF81548A3108F058C0DF019D9148
:105BA000903291F0A0EDA90FAA30E8F09E3271F486
:105BB000918190539A30B8F00115110519F48F01B5
:105BC0000150110990E013C0FD01E8CF9D3211F0A2
:105BD0009B3291F79181A0EDA90FAA3020F09E325F
:105BE00059F79281E6CF9E2F9D1B309759F3A82F2E
:105BF000B0E04601570104C0880C991CAA1CBB1CCC
:105C00008A95D2F7482959296A297B29A75EBA4F74
:105C10009C9380818154DF018A3108F497CFDF01A2
:105C20008191882309F492CF90ED980F9A30B8F3C0
:105C300093ED980F923098F38B3289F3CD01019652
:105C4000EC91E03209F082CFDC01F8CF01151105AB
:105C500001F78D01DECF10933C0500933B05409387
:105C60003705509338056093390570933A0540CF56
:105C70004F925F926F927F928F929F92AF92BF925C
:105C8000CF92DF92EF92FF92CF93DF9300D000D0BC
:105C90001F921F92CDB7DEB75C01DB01CD90DD9086
:105CA000ED90FC90E0918412F0918512FE83ED83DB
:105CB00084819581A681B78189839A83AB83BC83D4
:105CC0009C01AD01C701B6010F94042C2B013C01CE
:105CD000F50180809180A280B380AD81BE818D91DD
:105CE0009D910D90BC91A02D8D839E83AF83B8872D
:105CF00027E137EB41ED58EBC301B2010F94652E5C
:105D000087FDD2C023E030E04BE953E4C301B20188
:105D10000F94352518160CF4C7C02D813E814F8194
:105D20005885C501B4010F94042C2B013C0127E1D7
:105D300037EB41ED58EB0F94652E87FDB5C023E09E
:105D400030E84DE953E4C301B2010F94352518162C
:105D50000CF4AAC020E030E0A9016D817E818F8122
:105D600098850F94052C2B013C0120E030E040E4A5
:105D700050E40F94352587FF05C0412C512C30E4A9
:105D8000632E762C27E137EB41ED58E3C301B201D6
:105D90000F94042C9B01AC01C501B4010F94652E36
:105DA00087FD82C020E030E84DE953E46D817E81BB
:105DB0008F8198850F94052C2B013C0120E030E861
:105DC00044E953E40F94652E18163CF4412C20E866
:105DD000522E24E9622E23E4722E27E137EB41EDA7
:105DE00058E3C301B2010F94052C9B01AC01C5011E
:105DF000B4010F94352518160CF456C020E030E09D
:105E0000A90169817A818B819C810F94052C4B01BA
:105E10005C0120E030E040E551E40F94352587FF38
:105E200006C0812C912C90E5A92E91E4B92E27E192
:105E300037EB41ED58E3C501B4010F94042C9B01ED
:105E4000AC01C701B6010F94652E87FD2DC020E07F
:105E500030E04BE953E469817A818B819C810F9416
:105E6000052C4B015C0120E030E84FE853E40F942F
:105E7000652E18163CF4812C80E8982E8FE8A82E09
:105E800083E4B82E27E137EB41ED58E3C501B401B7
:105E90000F94052C9B01AC01B1E0B983C701B60199
:105EA0000F94352518160CF41982898128960FB69F
:105EB000F894DEBF0FBECDBFDF91CF91FF90EF9082
:105EC000DF90CF90BF90AF909F908F907F906F901A
:105ED0005F904F900895E2E1F8E082EBDF011D92C0
:105EE0008A95E9F708958091CD05811104C00E943B
:105EF0006B2F0C940EB88091311482FD0C9416F720
:105F0000089580911208882361F09091C308891345
:105F100008C08091311483FF04C080E598E00C94A0
:105F2000D8B680E00895FC01238121110C940DB3B3
:105F30000895EFE6F0E08081826080830895CF923B
:105F4000DF92EF92FF92CF93DF93C82F0E94082A2F
:105F500094E0C99FE0011124FE01E050FA4FC08097
:105F6000D180E280F38081110E94992FCA59DE4EC0
:105F7000C701B6010F943C25288139814A815B8194
:105F80000F949B25DF91CF91FF90EF90DF90CF9002
:105F900008958F929F92AF92BF92CF92DF92EF922D
:105FA000FF921F93CF93DF93CDB7DEB760970FB605
:105FB000F894DEBF0FBECDBF182F80E00E949F2F48
:105FC0004B015C0180928C0590928D05A0928E050C
:105FD000B0928F0581E00E949F2F6B017C01C092DF
:105FE0009005D0929105E0929205F092930582E09F
:105FF0000E949F2F6093940570939505809396055A
:10600000909397051D861E861F86188A89829A821C
:10601000AB82BC82CD82DE82EF82F88669877A8786
:106020008B879C8783E00E949F2F6D877E878F8759
:10603000988B8091390C882321F0CE0101960E9423
:106040001E211E3FD9F480E1FE013196A8E2BCE09A
:1060500001900D928A95E1F760960FB6F894DEBF35
:106060000FBECDBFDF91CF911F91FF90EF90DF90DA
:10607000CF90BF90AF909F908F90089584E0189F2D
:10608000F0011124DF01A85DB34F81E090E08C0F97
:106090009D1FE80FF91F40815181628173814D93EB
:1060A0005D936D937C931397D7CFCF92DF92EF924E
:1060B000FF92CF93DF93C82F0E94082A94E0C99FD4
:1060C000E0011124FE01EC50FA4FC080D180E28043
:1060D000F38081110E94992FCA59DE4EC701B60183
:1060E0000F943C25288139814A815B810F949B253F
:1060F000DF91CF91FF90EF90DF90CF9008950E94B5
:10610000082A90918A129093891290938812909302
:10611000871294E69093861220ED33E030930509C0
:106120002093040981110E94992F81E08093F30547
:106130000895CF93DF93CDB7DEB72C970FB6F894C1
:10614000DEBF0FBECDBF0E9433F60E94082A9CE03E
:10615000E0E0F6E0DE01119601900D929A95E1F7EC
:1061600081110E94992FCE0101960E944EC62C9655
:106170000FB6F894DEBF0FBECDBFDF91CF9108956B
:106180002F923F924F925F926F927F928F929F9247
:10619000AF92BF92CF92DF92EF92FF920F931F9335
:1061A000CF93DF9300D0CDB7DEB78090280C9090CE
:1061B000290CA0902A0CB0902B0C40902C0C5090E5
:1061C0002D0C60902E0C70902F0CC090300CD09045
:1061D000310CE090320CF090330C0E94B11B0E9405
:1061E000FF1B01E81CE187E492E09B838A8385E73B
:1061F000282E8CE1382E198289810E94A21CC801A8
:106200000E94851DEA81FB81619371938193919333
:10621000FB83EA83C1010E94851DEA81FB816087BF
:10622000718782879387F981FF5FF9830C5F1F4F26
:1062300084E0280E311CF330F9F68EED95E00E94D3
:1062400098F60E94A11E0E94E626A5019401609185
:10625000280C7091290C80912A0C90912B0C0F9492
:10626000352581111CC0A301920160912C0C709105
:106270002D0C80912E0C90912F0C0F9435258111AF
:106280000EC02091300C3091310C4091320C509165
:10629000330CC701B6010F9435258823B9F00F9050
:1062A0000F900F90DF91CF911F910F91FF90EF9082
:1062B000DF90CF90BF90AF909F908F907F906F9026
:1062C0005F904F903F902F900C9499300F900F90CB
:1062D0000F90DF91CF911F910F91FF90EF90DF9082
:1062E000CF90BF90AF909F908F907F906F905F9076
:1062F0004F903F902F90089580917A1190917B114B
:10630000892B79F480917A1190917B11892B49F432
:1063100020917A1130917B1181E0232B19F480E0D8
:10632000089581E008951092ED04809122029091E9
:106330002302A0912402B09125028093EA05909354
:10634000EB05A093EC05B093ED05089590919111A4
:1063500010929111923071F0943079F0913099F45B
:10636000813089F48091ED04882369F0109226022F
:106370000C9493311092270C089588E898E190933B
:10638000870C8093860C08959091311493FB882795
:1063900080F993FF06C081E090919815911101C09A
:1063A00080E00895CF93C0918A05CF7739F50E9498
:1063B000C431882319F18091291490912A14A09155
:1063C0002B14B0912C140097A105B105B9F0BC01B4
:1063D000CD016D597F4F8F4F9F4F24E630E040E055
:1063E00050E00F94792B60912D1470912E148091B0
:1063F0002F14909130140F94792BC22F8C2FCF91A2
:106400000895E1E0F9E010821182089581E0089595
:10641000DC01EC918E2F90E0FC01EE0FFF1FE80FE6
:10642000F91FE45DFD4E80818F77808308958F9200
:106430009F92AF92BF92CF92DF92EF92FF920F9313
:10644000CF93DF931F92CDB7DEB75C017B0149018B
:106450006B01C40ED51EF501808191810F94532BE1
:106460008983002311F0F7018083BE016F5F7F4FA6
:10647000C4010E94B6E0F50180819181019691836B
:106480008083FFEFEF1AFF0AEC14FD0421F780E090
:106490000F90DF91CF910F91FF90EF90DF90CF9011
:1064A000BF90AF909F908F9008950F93AB01009194
:1064B000E20521E0022723EE35E0BC0183EC95E004
:1064C0000E9417320F910895009781F41092900066
:1064D00082E0809391001092950010929400C19AEE
:1064E000809171008260809371000895019761F43A
:1064F0001092A00082E08093A1001092A50010925B
:10650000A40089BB8093720008957F928F929F921E
:10651000AF92BF92CF92DF92EF92FF920F931F93B1
:10652000CF93DF93EC017B018881883108F0C3C0F1
:1065300090E0FC01EE0FFF1FE80FF91FE45DFD4E38
:1065400080818F770E94FEE619821A8288812CE072
:10655000622F0F94DC2B829FB001112430E020E0E9
:10656000AB01420F531FFA01EE0FFF1FE40FF51F9F
:10657000E45DFD4E908197FD08C02F5F3F4F2C30AA
:10658000310571F790E00E9464327880072D10E0A9
:106590006801CC0CDD1CF601E00FF11FE45DFD4E3F
:1065A00080818068808377FC86C080E2E81682E084
:1065B000F8060CF03FC08A8128E532E0281B31093B
:1065C00087FD3395220F331F220F331F032E000C3C
:1065D000440B550B898178E8872E912C881A9108F5
:1065E00087FD9394880C991C880C991C092C000C2D
:1065F000AA08BB0860E070E0CB01F7FC0AC0B70155
:10660000653B710514F064EB70E0072E000C880BFD
:10661000990B281939094A095B090F94692B24EB56
:1066200030E040E050E00F949B2B820E931EA41E9E
:10663000B51E740187E18715D8F0298188E890E0BC
:10664000821B910927FD9395880F991F880F991F29
:10665000E816F90604F502972FB7F894E601C00F83
:10666000D11FC45DDD4E880F991F9A8389832FBF88
:1066700062E370E080E090E0DF91CF911F910F9195
:10668000FF90EF90DF90CF90BF90AF909F908F9052
:106690007F900C9408262A8188E592E0821B91095C
:1066A00027FD9395880F991F880F991FE816F90603
:1066B00094F6C701D0CFDF91CF911F910F91FF903A
:1066C000EF90DF90CF90BF90AF909F908F907F9092
:1066D0000895CF93DF93EB01682F70E085E792E197
:1066E0000E948532688179818A819B81643F21E0A3
:1066F00072078105910520F464EF71E080E090E07D
:106700000E94082689B183FB882780F9DF91CF9109
:106710000895CF93DF9300D01F92CDB7DEB78EEEF2
:1067200092E0A0E0B0E089839A83AB83BC83BE0192
:106730006F5F7F4F8AE50E9469330F900F900F9033
:106740000F90DF91CF910895CF93DF9300D01F92E8
:10675000CDB7DEB78EEE92E0A0E0B0E089839A83F9
:10676000AB83BC83BE016F5F7F4F8AE00E946933B9
:106770000F900F900F900F90DF91CF910895CF93CE
:10678000DF9300D01F92CDB7DEB784EF91E0A0E099
:10679000B0E089839A83AB83BC83BE016F5F7F4F78
:1067A00080EA0E9469330F900F900F900F90DF9155
:1067B000CF9108951F920F920FB60F9211240BB62E
:1067C0000F922F933F934F935F936F937F938F938A
:1067D0009F93AF93BF93EF93FF9348EA50E064EA2F
:1067E00070E081E090E00E942C26FF91EF91BF9134
:1067F000AF919F918F917F916F915F914F913F9159
:106800002F910F900BBE0F900FBE0F901F901895F9
:106810001F920F920FB60F9211240BB60F922F9367
:106820003F934F935F936F937F938F939F93AF9318
:10683000BF93EF93FF9348E950E064E970E090E084
:1068400080E00E942C26FF91EF91BF91AF919F9124
:106850008F917F916F915F914F913F912F910F9009
:106860000BBE0F900FBE0F901F9018959091D10006
:1068700095FD0CC09091D00095FF08C08093D60084
:106880008091D00080648093D000089520911A04F4
:106890002F5F2F770FB607FC27C090911B04921330
:1068A00028C09091D00095FF1EC090911B0440918C
:1068B0001A04941306C09091D1009F7D9093D1004B
:1068C00012C0E92FF0E0E65EFB4F32819F5F9F77B9
:1068D0003093D60090931B043091D00030643093F5
:1068E000D000491741F3D9CF90911B04921301C0F6
:1068F000FBCFE0911A04F0E0E65EFB4F8283209329
:106900001A048091D10080628093D10008958F9203
:106910009F92AF92BF92CF92DF92EF92FF920F932E
:106920001F93CF93DF937C0121E5E20EF11CD70189
:106930004C914A3509F0A4C06C01B2E5CB0ED11CD4
:10694000F6013081353A09F09BC0EC01C05BDF4FA6
:106950002881233008F494C08C0100561F4FD801C1
:106960004C93E15BFF4F308331962083EF54F10964
:106970003081E05BFF4F30833038B1F43196AC5456
:10698000B1093C913083E854F109AF5ABF4F50E050
:1069900040E02250330B42175307CCF480813296EB
:1069A0008D934F5F5F4FF7CF233031F5313809F0CA
:1069B00074C0FC01EC55FF4FDC01AC5ABF4F2C9169
:1069C00020833196885A9F4FDC018C918083480147
:1069D000B12CA12C888190E002968A159B050CF4BD
:1069E0003FC0F40181914F010E9436340E94CCE0F7
:1069F000FFEFAF1ABF0AEECF323821F5FC01EC5A97
:106A0000FF4F30814181E05BFF4F408331963083FF
:106A1000DC01AA55BF4F50E040E02350330B421732
:106A20005307ACF6FA01EE7FE45AFF4FE80FF91F67
:106A3000608171817C9311966C9311974E5F5F4FCB
:106A40001296EDCF243019F6333809F6FC01EC5AD2
:106A5000FF4F20813181E05BFF4F30833196B0CF13
:106A600080E5DE011D928A95E9F78AE1F80111922D
:106A70008A95E9F78AE5D7018C9385EAF601808348
:106A8000DF91CF911F910F91FF90EF90DF90CF900A
:106A9000BF90AF909F908F900895323809F097CFB4
:106AA000ADCFAF92BF92CF92DF92EF92FF920F9352
:106AB0001F93CF93DF93EC0184E6C82E80E2D82E9B
:106AC000E12CF12C02E8A12C90E2B92E15E0009304
:106AD000BE13C092BF13D092C013E092C113F092C4
:106AE000C213B092C813A092C7131093BB138BE6C6
:106AF00093E10E9487348FEFC81AD80AE80AF80A8F
:106B000088E7C81680E2D806E104F10401F724E61C
:106B100030E240E050E0BE018BE693E1DF91CF919F
:106B20001F910F91FF90EF90DF90CF90BF90AF90AB
:106B30000C94D1E0CF92DF92EF92FF920F931F93CC
:106B4000CF93DF93CDB7DEB77C01CDB6DEB60F9421
:106B5000822401962DB73EB7281B390B0FB6F89447
:106B60003EBF0FBE2DBF0DB71EB70F5F1F4FB70142
:106B7000C8010F947B24F80101900020E9F73197B8
:106B8000E01BF10B759720F08BE792E0F801848B06
:106B9000C8010E9451350FB6F894DEBE0FBECDBEBF
:106BA000DF91CF911F910F91FF90EF90DF90CF90E9
:106BB00008958F929F92AF92BF92CF92DF92EF9201
:106BC000FF920F931F93CF93DF930E94AA2C3AE07A
:106BD000C32E30E2D32EE12CF12C15E002E8460161
:106BE0005701CAE0D0E01092C8131092C713109357
:106BF000BB130093BE138092BF139092C013A09258
:106C0000C113B092C2138BE693E10E94873421979F
:106C10008FEF881A980AA80AB80A209721F78AE005
:106C2000C80ED11CE11CF11C82EDC81680E2D8060A
:106C3000E104F104A1F6C12C20E2D22EE12CF12CCA
:106C4000D5E0C2E81092C8131092C713D093BB13BB
:106C5000C093BE13C092BF13D092C013E092C11371
:106C6000F092C2138BE693E10E9487341092C8130E
:106C70001092C713D093BB13C093BE13D701C601A4
:106C80008C529F4FAF4FBF4F8093BF139093C01351
:106C9000A093C113B093C2138BE693E10E94873493
:106CA0008FEFC81AD80AE80AF80A8AE0C81680E204
:106CB000D806E104F10431F69EEDC92E90E2D92EFA
:106CC000E12CF12CD5E0C2E81092C8131092C71342
:106CD000D093BB13C093BE13C092BF13D092C01306
:106CE000E092C113F092C2138BE693E10E948734C5
:106CF0008FEFC81AD80AE80AF80A86EEC81680E2AA
:106D0000D806E104F10401F7CC24C39482E1D82E23
:106D1000E12CF12C0AE010E0D5E0C2E81093C81392
:106D20000093C713D093BB13C093BE13C092BF137D
:106D3000D092C013E092C113F092C2138BE693E19C
:106D40000E9487341093C8130093C713D093BB13CA
:106D5000C093BE13D701C6018096A11DB11D8093BB
:106D6000BF139093C013A093C113B093C2138BE6CB
:106D700093E10E9487348FEFC81AD80AE80AF80A0C
:106D800085E1C81682E1D806E104F10439F682E112
:106D900090E09093C8138093C713D093BB13C09314
:106DA000BE1384E190E1A0E0B0E08093BF13909324
:106DB000C013A093C113B093C2138BE693E1DF918C
:106DC000CF911F910F91FF90EF90DF90CF90BF90E8
:106DD000AF909F908F900C9487341F920F920FB6B4
:106DE0000F9211240BB60F922F938F939F93EF93D3
:106DF000FF9380911B0420911A04821306C0809196
:106E0000D1008F7D8093D10012C0E82FF0E0E65EC4
:106E1000FB4F92818F5F8F779093D60080931B04F6
:106E20009091D00090649093D000281741F3FF9187
:106E3000EF919F918F912F910F900BBE0F900FBEEE
:106E40000F901F9018951F920F920FB60F9211245A
:106E50000BB60F920F931F932F933F934F935F9314
:106E60006F937F938F939F93AF93BF93CF93DF9352
:106E7000EF93FF93C091D60000913E05D0913D0560
:106E800011E01D0F1F7390911904913108F09FC0FC
:106E9000E92FF0E08827E05BF84C8F4F0D94FC2B36
:106EA000613790379F37AE37B537E737B937E737B0
:106EB000BD37C137E737C537C937CD37D437E7379F
:106EC000DF37C03229F028F5CA3011F0CD3031F566
:106ED000011731F0ED2FF0E0E35CFA4FC283D12FC0
:106EE000D0933D05FF91EF91DF91CF91BF91AF918D
:106EF0009F918F917F916F915F914F913F912F91D2
:106F00001F910F910F900BBE0F900FBE0F901F900F
:106F10001895CD3481F081E0CE3471F080E10CC061
:106F2000CA3338F4C033A0F6C03291F2CD32B1F793
:106F3000CFCFCD3499F782E080931904C9CFC13304
:106F400059F018F4C03221F2E9CF88E0C433A1F33C
:106F50008BE0C83389F3E2CF83E0EECF84E0C03327
:106F600059F386E0C13341F3D9CF85E0C833B1F698
:106F7000E3CF87E0C23391F6DFCF89E0C13371F60A
:106F8000DBCF8AE0C03351F6D7CF8CE0C73331F680
:106F9000D3CF8DE0C63311F6CFCFC03209F498CFEE
:106FA0008EE0C33549F2BACF80ED8C0F8A3008F0FD
:106FB0008FCF9FE0909319048093180489CFCA3033
:106FC00019F0CD3009F084CF1092190481CFCA3066
:106FD00019F0CD3009F07CCF809125148823A1F3DE
:106FE000973089F038F4953079F710923C0210927E
:106FF000270CEACF9A3059F09F3031F7809118046E
:107000000E94A631E1CF81E080931106DDCF81E0BF
:1070100080931006D9CF9091C00095FFFCCF80934C
:10702000C6000895CF93DF93EC018991882319F06E
:107030000E940B38FACF8DE00E940B388AE0DF9176
:10704000CF910C940B38CF92DF92EF92FF92CF93B7
:107050006B017C01C42F4A3069F4F7FE0BC0F09439
:10706000E094D094C094C11CD11CE11CF11C8DE2B1
:107070000E940B384C2FC701B601CF91FF90EF90C3
:10708000DF90CF900C9446AACF93DF93EC01FE01E2
:1070900084912196882319F00E940B38F8CFDF9154
:1070A000CF910895CF93DF93D09124118DE59CE18A
:1070B0000E9444388AE00E940B388091A30C8730EC
:1070C00009F449C083E08093A10C81E080936E02B3
:1070D00080E190E09093C8138093C71385E080937C
:1070E000BB13C2E8C093BE1384E190E1A0E0B0E01E
:1070F0008093BF139093C013A093C113B093C21396
:107100008BE693E10E94873461E070E080E090E0DC
:107110000E948F2C81E09AE59093C8138093C71347
:1071200085E390E09093CA138093C91387E080931E
:10713000BB13C093BE1384E890E0A0E0B0E080935E
:10714000BF139093C013A093C113B093C2138BE6E7
:1071500093E10E94873480912411813089F182303B
:1071600061F50E947C2B6093AB057093AC05809316
:10717000AD059093AE0581E0809324110E940EFD31
:107180006093A7057093A8058093A9059093AA051D
:10719000D23089F080919406909195060196909353
:1071A0009506809394061092B3051092B405109240
:1071B000B5051092B60581E004C00E94AE2BDBCF6E
:1071C00080E0DF91CF910895CF93C82FCB010E942B
:1071D000443881ED98E10E94443882EC98E1CC2358
:1071E00011F087EC98E10E9444388AE0CF910C942A
:1071F0000B38CF93DF9300D01F92CDB7DEB784EF6B
:1072000091E0A0E0B0E089839A83AB83BC83BE01A8
:107210006F5F7F4F8CE30E9469338FEE98E10E948D
:1072200044388CB169EE78E185FB882780F90E94AB
:10723000E4388091030163EE78E1869581700E94C5
:10724000E43889B16DED78E183FB882780F90E94ED
:10725000E4388CB164ED78E1829581700E94E43865
:107260004B9909C00E94A4330F900F900F900F907C
:10727000DF91CF9108950E9489330F900F900F9066
:107280000F90DF91CF910895809124118130C1F545
:107290008DE998E10E9444388AE00E940B3881E031
:1072A0009AE59093C8138093C71387E590E0909375
:1072B000CA138093C91387E08093BB1382E880933D
:1072C000BE1384E890E0A0E0B0E08093BF139093F9
:1072D000C013A093C113B093C2138BE693E10E9435
:1072E000873482E0809324110E940EFD6093AF05E5
:1072F0007093B0058093B1059093B20581E0089535
:1073000080E008950F931F930E940EFD00918F0659
:107310001091900620919106309192060115110569
:107320002105310509F067C020919D12222309F43F
:107330005FC0E0919B12215020939D1221E02E0FFF
:1073400020939B1230919E12231302C010929B1225
:1073500024E0E29FF0011124E156FD4E00811181ED
:107360002281338100938B0610938C0620938D0627
:1073700030938E06600F711F811D911D60938F06E3
:1073800070939006809391069093920680918D065B
:1073900090918E06892B61F11FB7F8948CE898E1E3
:1073A0000E9444388AE00E940B3884E096E0909373
:1073B000C8138093C71380EA90E89093CA13809310
:1073C000C91387E08093BB1382E88093BE1380EAE1
:1073D00090E0A0E0B0E08093BF139093C013A0931F
:1073E000C113B093C2138BE693E10E9487341FBF91
:1073F0001F910F910895601B710B820B930B97FDEA
:10740000F7CF409810928F06109290061092910636
:1074100010929206EDCF0F931F93CF93DF938C01C1
:10742000EB0190919D1220919E12921305C00E9433
:1074300082390E940EC2F5CF80919C1234E0839F66
:10744000F0011124E156FD4E11830083D383C283E2
:107450009F5F90939D128F5F281739F080939C1245
:10746000DF91CF911F910F91089510929C12F8CF48
:10747000CF92DF92EF92FF921F93CF93DF93182F5B
:10748000662351F01092EC041092E8041092E90483
:107490001092EA041092EB040E940EFD6B017C0135
:1074A0008091E8049091E904A091EA04B091EB0482
:1074B000A7019601281B390B4A0B5B0BDA01C901A6
:1074C000B7FD3DC02091EC0417FD13C0412F012EE4
:1074D000000C550B4C5F5F4F822F022E000C990B56
:1074E0004817590764F184EF91E0A0E0B0E021175C
:1074F00024F488EE93E0A0E0B0E08C0D9D1DAE1D5D
:10750000BF1D8093E8049093E904A093EA04B0932C
:10751000EB042170C22F30E0D32F84E28C9FB001A6
:107520008D9F700D7C1B112460597C4F82E390E08D
:107530000E940B3A8091EC048F5F8093EC04DF9102
:10754000CF911F91FF90EF90DF90CF900895CF9350
:10755000DF9300D01F92CDB7DEB782E198E10E94A1
:1075600044388AE00E940B388091A30C8330D9F113
:1075700019821A821B821C8260E0CE0101960E9451
:10758000C92B19821A821B821C8261E0CE010196EE
:107590000E94C92B81E080936D021092A00C809311
:1075A0006E0281E09AE59093C8138093C71383E33A
:1075B00090E09093CA138093C91387E08093BB1324
:1075C00082E88093BE1384E890E0A0E0B0E080936E
:1075D000BF139093C013A093C113B093C2138BE653
:1075E00093E10E9487340F900F900F900F90DF91DE
:1075F000CF9108956F927F928F929F92AF92BF9298
:10760000CF92DF92EF92FF920F931F93CF93DF936E
:10761000CDB7DEB764970FB6F894DEBF0FBECDBF0F
:107620001092D0008091D00082608093D0001092A0
:10763000D50080E18093D4008091D1008061809357
:10764000D1008091D10088608093D1008091D100D9
:1076500080688093D1008091D1008F7D8093D1008C
:107660008AE58093BC1380936C1385EA8093BD13E5
:1076700080936D13EBE0F4E18AE1DF011D928A95BE
:10768000E9F780919F0C882309F473C283E090E0AE
:107690009093C8138093C71385E08093BB1382E84F
:1076A0008093BE138FE190E1A0E0B0E08093BF1320
:1076B0009093C013A093C113B093C2138BE693E1D0
:1076C0000E94873484E690E09093C8138093C71398
:1076D00005E00093BB1312E81093BE1386E090E11F
:1076E000A0E0B0E08093BF139093C013A093C113A8
:1076F000B093C2138BE693E10E9487348BE090E055
:107700009093C8138093C7130093BB131093BE13B9
:1077100080E092E1A0E0B0E08093BF139093C013AB
:10772000A093C113B093C2138BE693E10E948734F8
:107730001092C8131092C7130093BB131093BE137B
:1077400084E390E1A0E0B0E08093BF139093C01376
:10775000A093C113B093C2138BE693E10E948734C8
:107760001092C8131092C7130093BB131093BE134B
:107770008AE390E1A0E0B0E08093BF139093C01340
:10778000A093C113B093C2138BE693E10E94873498
:107790008091EB119091EC119093C8138093C713D3
:1077A0000093BB131093BE1386E390E1A0E0B0E01A
:1077B0008093BF139093C013A093C113B093C213CF
:1077C0008BE693E10E948734809180119091811122
:1077D0009093C8138093C7130093BB131093BE13E9
:1077E0008CE390E1A0E0B0E08093BF139093C013CE
:1077F000A093C113B093C2138BE693E10E94873428
:1078000082E090E09093C8138093C7130093BB135A
:107810001093BE138EE190E1A0E0B0E08093BF131F
:107820009093C013A093C113B093C2138BE693E15E
:107830000E94873481E080936D0270E6C72E70E16C
:10784000D72EE12CF12C1092C8131092C71300937D
:10785000BB131093BE13C092BF13D092C013E0921B
:10786000C113F092C2138BE693E10E948734BFEFFD
:10787000CB1ADB0AEB0AFB0AE4E7CE16E0E1DE06F0
:10788000E104F10401F7CE0101967C0184E1D70106
:107890001D928A95E9F781E08F9390E99F938F93EA
:1078A0009CE29F938F939F9389E993E09F938F939B
:1078B000FF92EF920F948D2F20E630E140E050E0F0
:1078C00066EA73E08BE693E10E94D1E02AE630E1BC
:1078D00040E050E062EB73E08BE693E10E94D1E080
:1078E00024E730E140E050E0B7018BE693E10E94ED
:1078F000D1E02EE730E140E050E06EEB73E08BE644
:1079000093E10E94D1E01092C8131092C713009324
:10791000BB131093BE138EE090E1A0E0B0E0809323
:10792000BF139093C013A093C113B093C2138BE6FF
:1079300093E10E9487341092C8131092C7130093EA
:10794000BB131093BE138FE090E1A0E0B0E08093F2
:10795000BF139093C013A093C113B093C2138BE6CF
:1079600093E10E9487340FB6F894DEBF0FBECDBFFF
:107970004AE0C42E40E2D42EE12CF12C55E0752EC5
:1079800062E8662E460157010AE010E01092C81323
:107990001092C7137092BB136092BE138092BF13F4
:1079A0009092C013A092C113B092C2138BE693E1E0
:1079B0000E94873401501109FFEF8F1A9F0AAF0A06
:1079C000BF0A0115110511F78AE0C80ED11CE11C90
:1079D000F11C92EDC91690E2D906E104F10491F68A
:1079E000C12C30E2D32EE12CF12C05E012E81092EC
:1079F000C8131092C7130093BB131093BE13C09209
:107A0000BF13D092C013E092C113F092C2138BE661
:107A100093E10E9487341092C8131092C713009309
:107A2000BB131093BE13D701C6018C529F4FAF4FAB
:107A3000BF4F8093BF139093C013A093C113B09313
:107A4000C2138BE693E10E948734AFEFCA1ADA0AB9
:107A5000EA0AFA0ABAE0CB16B0E2DB06E104F10466
:107A600031F62EEDC22E20E2D22EE12CF12C05E0D3
:107A700012E81092C8131092C7130093BB1310930F
:107A8000BE13C092BF13D092C013E092C113F09204
:107A9000C2138BE693E10E948734EFEFCE1ADE0A21
:107AA000EE0AFE0AF6EECF16F0E2DF06E104F1047C
:107AB00001F7CC24C39482E1D82EE12CF12C9AE07A
:107AC000A92EB12C05E012E8B092C813A092C713FA
:107AD0000093BB131093BE13C092BF13D092C01378
:107AE000E092C113F092C2138BE693E10E948734B7
:107AF000B092C813A092C7130093BB131093BE1388
:107B0000D701C6018096A11DB11D8093BF1390932C
:107B1000C013A093C113B093C2138BE693E10E94EC
:107B200087348FEFC81AD80AE80AF80A95E1C9160F
:107B300092E1D906E104F10439F688E797E10E9461
:107B400044388AE00E940B3864960FB6F894DEBF82
:107B50000FBECDBFDF91CF911F910F91FF90EF909E
:107B6000DF90CF90BF90AF909F908F907F906F905D
:107B7000089582E090E08CCD0E94FA3A109286053A
:107B800081E080936E028AE298E10E9444388AE0A4
:107B90000C940B380F931F93CF938C01C62F83E265
:107BA00094E10E944438C8010E9444388AE30E944C
:107BB0000B3880E38C0F0E940B388AE0CF911F9125
:107BC0000F910C940B3886EA95E10E94443860E0EE
:107BD00086E995E10E94CA3D60E081E895E10E9456
:107BE000CA3D61E08AE795E10E94CA3D61E08FE607
:107BF00095E10E94CA3D61E08FE595E10E94CA3D92
:107C000060E086E595E10E94CA3D61E08CE495E183
:107C10000E94CA3D61E082E495E10E94CA3D61E0B4
:107C20008BE395E10E94CA3D61E083E395E10E9408
:107C3000CA3D61E085E295E10E94CA3D61E087E1CD
:107C400095E10E94CA3D60E088E095E10E94CA3D4E
:107C500060E08AEF94E10E94CA3D60E084EE94E126
:107C60000E94CA3D61E083ED94E10E94CA3D61E05B
:107C700084EC94E10E94CA3D61E08DEB94E10E94A6
:107C8000CA3D60E086EB94E10E94CA3D61E08DEA66
:107C900094E10E94CA3D61E088E994E10E94CA3DF6
:107CA00061E08AE894E10E94CA3D61E087E794E1DF
:107CB0000E94CA3D60E08AE694E10E94CA3D61E00C
:107CC00085E694E10E94CA3D61E088E594E10E9466
:107CD000CA3D60E084E494E10E94CA3D60E081E333
:107CE00094E10E94CA3D60E084E394E10E94681D33
:107CF000682F617088E294E10C94CA3D8091370549
:107D0000827149F4809139058C7829F480913A0583
:107D1000837009F475C082E40E94461E882351F0E6
:107D20000E94142460934E0C70934F0C8093500C5F
:107D30009093510C83E50E94461E882351F00E94C7
:107D40009A2460937E0C70937F0C8093800C9093A8
:107D5000810C84E50E94461E882351F00E949A24DB
:107D60006093820C7093830C8093840C9093850CA9
:107D700088E50E94461E882351F00E949A24609351
:107D8000DD087093DE088093DF089093E00889E5B2
:107D90000E94461E882351F00E949A246093E108B5
:107DA0007093E2088093E3089093E4088AE50E94C8
:107DB000461E8823B1F00E949A246093E5087093D0
:107DC000E6088093E7089093E8082DEC3CEC4CEC37
:107DD0005DE30F943525181624F088E99EE00E9493
:107DE000443885E40E94461E882351F00E949A245C
:107DF0006093E9087093EA088093EB089093EC088D
:107E00000895AF92BF92CF92DF92EF920F931F939C
:107E1000CF93DF935B01EA016901882309F463C012
:107E200081E99EE00E944438F50160817181828180
:107E3000938146E00E944EBAE1100BC088E89EE0B4
:107E40000E944438688179818A819B8146E00E9442
:107E50004EBA81E89EE00E944438F601608171814B
:107E60008281938143E00E944EBA8AE79EE00E949D
:107E70004438F801608171818281938143E00E94DE
:107E80004EBA81E79EE00E944438F601208131819C
:107E900042815381F80160817181828193810F94C5
:107EA000042C43E00E944EBAEE20F9F08AE00E94D2
:107EB0000B388CE59EE00E944438688179818A8184
:107EC0009B8146E00E944EBA8AE00E940B388AE00D
:107ED000DF91CF911F910F91EF90DF90CF90BF90E6
:107EE000AF900C940B38E110E4CFDF91CF911F914C
:107EF0000F91EF90DF90CF90BF90AF9008950F93C8
:107F00001F93CF938C01C62F89E798E00E944438D5
:107F1000C8010E944438CC2331F08AE0CF911F91F0
:107F20000F910C940B38CF911F910F9108950E94DF
:107F300066E41092270C10923C020E94C431882300
:107F400051F08091311482FD06C088E898E1909349
:107F5000870C8093860C61E081E898E10E947F3F66
:107F60000C9452380F931F93CF93DF938C016F3F84
:107F700019F41092651160E020916511862F062E8C
:107F8000000C990B2817190609F08CF56093651100
:107F900060E08BE498E10E947F3FC8010E94443872
:107FA0008AE00E940B38C8010F948224800F911F31
:107FB000EC01C01BD10BC034D1053CF00197FC0192
:107FC0002491207C2038D1F3F3CFDD27AE01B80116
:107FD00085E291E10F94A324CB5DDE4E188285E209
:107FE00091E1DF91CF911F910F910C945135DF9169
:107FF000CF911F910F9108951092270C10923C027F
:108000008091311480648093311461E089E598E1B6
:108010000E947F3F4EE658E166E778E185E00E94E6
:10802000EBE260E080E698E10C94B23F0F931F937F
:10803000CF938C01C62F60E083E898E00E947F3FD9
:10804000C8010E944438CC2331F08AE0CF911F91BF
:108050000F910C940B38CF911F910F91089561E00F
:108060008BE898E00C941640EF92FF920F931F93C9
:10807000CF937C018B01C42F60E083E898E00E94DD
:108080007F3FC7010E94443880E20E940B38C8013C
:108090000E944438CC2319F08C2F0E940B388AE0C0
:1080A000CF911F910F91FF90EF900C940B38DF92BE
:1080B000EF92FF920F931F93CF93DF93D82E7B0104
:1080C0008A01E9010E942F40D092911140E0B7014E
:1080D00084E799E00E9434400115110531F040E039
:1080E000B8018DE699E00E943440209731F040E0DD
:1080F000BE018DE699E00E94344061E088E699E097
:10810000DF91CF911F910F91FF90EF90DF900C9432
:108110001640AF92BF92CF92DF92EF92FF920F93F1
:108120001F93CF93DF9386EE97E00E944438C0E020
:10813000D7E0D15021F080E20E940B38FACF8C2F8B
:108140000E9424E1CF5FC53099F78AE00E940B3886
:1081500000E917E0C0E080E20E940B388C2F0E94FB
:1081600024E15801D5E080E20E940B38F501C0807F
:10817000D180E280F380A7019601C701B6010F9478
:10818000F72E882369F180E20E940B388DE30E946C
:108190000B388DE30E940B388DE30E940B388DE382
:1081A0000E940B388DE30E940B38D150F4E1AF0EE2
:1081B000B11CD111D8CF8AE00E940B38CF5F0C5F81
:1081C0001F4FC53041F68AE0DF91CF911F910F918B
:1081D000FF90EF90DF90CF90BF90AF900C940B3852
:1081E00020E030E0A901C701B6010F94652E87FD9C
:1081F00003C08BE20E940B3843E0C701B6010E9426
:108200004EBAD3CF811107C08AEC9EE00E94443859
:108210008AE00C940B388EEC9EE0F8CFCF93DF937E
:10822000EB010E944438CE01DF91CF910C94E2E142
:10823000CF93C62F0E9444388C2FCF910C9424E109
:10824000CF92DF92EF92FF926A017B010E94443845
:1082500042E0C701B601FF90EF90DF90CF900C9401
:108260004EBACF92DF92EF92FF926A017B010E9499
:1082700044384AE0C701B601FF90EF90DF90CF90FD
:108280000C942338CF93DF93EB010E944438CE0146
:10829000DF91CF910C942BE14F925F926F927F927E
:1082A0008F929F92AF92BF92CF92DF92EF92FF9206
:1082B0000F931F93CF93DF9300D000D01F921F9294
:1082C000CDB7DEB78091850581110AC48091830501
:1082D000909184059C012F5F3F4F3093840520933C
:1082E00083058E3E924008F4FBC38091EB11909180
:1082F000EC119093C8138093C71305E00093BB1350
:1083000012E81093BE1386E390E1A0E0B0E0809302
:10831000BF139093C013A093C113B093C2138BE605
:1083200093E10E9487348091801190918111909304
:10833000C8138093C7130093BB131093BE138CE331
:1083400090E1A0E0B0E08093BF139093C013A0939E
:10835000C113B093C2138BE693E10E9487348091DE
:10836000ED119091EE119093C8138093C713009371
:10837000BB131093BE1384E390E1A0E0B0E08093C0
:10838000BF139093C013A093C113B093C2138BE695
:1083900093E10E9487348091821190918311909390
:1083A000C8138093C7130093BB131093BE138AE3C3
:1083B00090E1A0E0B0E08093BF139093C013A0932E
:1083C000C113B093C2138BE693E10E94873481E01E
:1083D0008093850510928405109283058091A30CEB
:1083E000882339F10E94FA1C811123C080918205F3
:1083F0008F5F8093820580918205853620F01092F0
:1084000082051092A30CE091A30CE150E73008F034
:108410006AC00E2E000CFF0B8827EE5EFD4B8F4FBF
:108420000D94FC2B1C426B4237446344A444DC444F
:108430006F4210928205DFCF0E94872C882309F4B7
:1084400052C081E080936E0284E098E10E9444383B
:108450008AE00E940B3880E190E09093C8138093EB
:10846000C71385E08093BB1312E81093BE1384E119
:1084700090E1A0E0B0E08093BF139093C013A0936D
:10848000C113B093C2138BE693E10E94873481E05D
:108490009AE59093C8138093C71386E390E0909376
:1084A000CA138093C91387E08093BB131093BE1344
:1084B00084E890E0A0E0B0E08093BF139093C013F5
:1084C000A093C113B093C2138BE693E10E9487344B
:1084D0001092A30C08C00E94872C882321F00E94D0
:1084E000FA1C8823A9F380916E02882309F433C70C
:1084F000809186058111C0C284E096E09093C813F4
:108500008093C71380EA90E89093CA138093C913AD
:1085100017E01093BB1302E80093BE1380EA90E0CB
:10852000A0E0B0E08093BF139093C013A093C11359
:10853000B093C2138BE693E10E9487348091690265
:1085400090916A02A0916B02B0916C020097A10514
:10855000B10509F03FC21092C8131092C71315E07D
:108560001093BB130093BE138AE890E1A0E0B0E043
:108570008093BF139093C013A093C113B093C21301
:108580008BE693E10E94873489E090E09093C813D2
:108590008093C7131093BB130093BE138CE890E134
:1085A000A0E0B0E08093BF139093C013A093C113D9
:1085B000B093C2138BE693E10E94873480916902E5
:1085C00090916A02A0916B02B0916C020097F1E069
:1085D000AF07B10508F441C2B093C813A093C71305
:1085E0009093CA138093C91387E08093BB1382E8EA
:1085F0008093BE1388E890E1A0E0B0E08093BF13C1
:108600009093C013A093C113B093C2138BE693E170
:108610000E9487348091690290916A02A0916B0256
:10862000B0916C02BA2FA92F982F8827009721E0CC
:10863000A207B10508F417C2B093C813A093C713DB
:108640009093CA138093C91387E08093BB1312E8F9
:108650001093BE1381EA90E0A0E0B0E08093BF13D6
:108660009093C013A093C113B093C2138BE693E110
:108670000E9487348091390C882309F4FAC183E081
:1086800090E09093C8138093C71385E08093BB1349
:108690001093BE1385E490E1A0E0B0E08093BF1397
:1086A0009093C013A093C113B093C2138BE693E1D0
:1086B0000E94873480918605875E8093860520918D
:1086C0008605822F90E0253608F021C29093C813CA
:1086D0008093C71385E08093BB1382E88093BE1319
:1086E00080E090E1A0E0B0E08093BF139093C013CE
:1086F000A093C113B093C2138BE693E10E94873419
:108700000E94FA1C811114C20E94C431811105C05B
:108710009091890591FD0E94FA1C9091890580FB3A
:1087200091F99093890591FD03C28091311482FDE6
:10873000FFC1809124118150823008F4F9C1609109
:10874000821170918311072E000C880B990B0F94E6
:108750003C256B017C0120E030E0A9010F94352518
:10876000882309F4BBC66091801170918111072E96
:10877000000C880B990B0F943C252B013C0120E049
:1087800030E040E050E4C701B6010F94042CA3018F
:1087900092010F94652E18160CF4C2C66091EB116D
:1087A0007091EC11072E000C880B990B0F943C254F
:1087B0006D837E838F8398876091ED117091EE11A8
:1087C000072E000C880B990B0F943C254B015C0184
:1087D00020E030E040E251E40F94042C2D813E81F2
:1087E0004F8158850F94652E18160CF499C620E019
:1087F00030E040E050E4C701B6010F94052CA3011E
:1088000092010F94352587FD10C020E030E040E252
:1088100051E4C501B4010F94052C2D813E814F8197
:1088200058850F94352587FF6AC684E190E09093C0
:10883000C8138093C71385E08093BB1382E88093AD
:10884000BE1384E190E1A0E0B0E08093BF13909369
:10885000C013A093C113B093C2138BE693E10E949F
:1088600087348091A10C81117CC682E07AC686EFA4
:1088700097E10E9444388AE00E940B3881E09AE533
:108880009093C8138093C71380E490E09093CA1329
:108890008093C91317E01093BB1382E88093BE1333
:1088A00084E890E0A0E0B0E08093BF139093C01301
:1088B000A093C113B093C2138BE693E10E94873457
:1088C0001093A30C10CE8091900C882309F40BCE4A
:1088D0000E94872C882309F406CE0E94FA1C81117D
:1088E00002CE88EE97E10E9444388AE00E940B385D
:1088F0008091910C90E0B0E0A0E0895B9F4FAE4F7B
:10890000B54A21E03AE53093C8132093C7139093FA
:10891000CA138093C91387E08093BB1382E88093C6
:10892000BE1384E890E0A0E0B0E08093BF13909382
:10893000C013A093C113B093C2138BE693E10E94BE
:1089400087341092900CC4CD0E94872C882309F4A0
:10895000CACD0E94FA1C8111C6CD81E080936E02BF
:108960001092A30C8AED97E10E9444388AE00E949D
:108970000B3881E09AE59093C8138093C7138EE477
:1089800090E09093CA138093C91387E08093BB1340
:1089900082E88093BE1384E890E0A0E0B0E080938A
:1089A000BF139093C013A093C113B093C2138BE66F
:1089B00093E10E94873497CD0E94FA1C811193CDD8
:1089C00019821A821B821C8262E0CE0101960E94EB
:1089D000B3F47ECD0196A11DB11D35E0B695A795E6
:1089E000979587953A95D1F70197A109B109009715
:1089F000E1E0AE07B10548F1B093C813A093C713E7
:108A00009093CA138093C9131093BB1312E8109369
:108A1000BE138AE890E1A0E0B0E08093BF1390938A
:108A2000C013A093C113B093C2138BE693E10E94CD
:108A3000873488E090E09093C8138093C71385E053
:108A40008093BB131093BE13A9CD9093C81380934A
:108A5000C71385E08093BB13D9CF9093C81380933D
:108A6000C71385E0C2CD9093C8138093C71385E0E8
:108A7000ECCD82E090E005CE8A3F08F020CE8EEF6C
:108A80008093860589EC97E10E9444388AE00E9431
:108A90000B3881E080936E0281E09AE59093C813D1
:108AA0008093C7138DE290E09093CA138093C9130B
:108AB00087E08093BB1382E88093BE1384E890E044
:108AC000A0E0B0E08093BF139093C013A093C113B4
:108AD000B093C2138BE693E10E9487341092850510
:108AE00028960FB6F894DEBF0FBECDBFDF91CF91B1
:108AF0001F910F91FF90EF90DF90CF90BF90AF90BC
:108B00009F908F907F906F905F904F9008958456C4
:108B100091099093C8138093C71385E08093BB138A
:108B200082E88093BE1381E090E1A0E0B0E0DCCD6C
:108B30008CE090E09093C8138093C71315E01093D6
:108B4000BB1382E88093BE1384E190E1A0E0B0E023
:108B50008093BF139093C013A093C113B093C2131B
:108B60008BE693E10E9487340E947C2B20E13EE05B
:108B700040E050E00F94792B2115310581E0480742
:108B8000510508F470C05093C8134093C713309335
:108B9000CA132093C91387E08093BB1312E8109384
:108BA000BE1380E190E1A0E0B0E08093BF1390930A
:108BB000C013A093C113B093C2138BE693E10E943C
:108BC00087340E947C2B20E13EE040E050E00F948F
:108BD000792B2CE330E040E050E00F94792B309378
:108BE000C8132093C71305E00093BB131093BE1363
:108BF00082E190E1A0E0B0E08093BF139093C013B6
:108C0000A093C113B093C2138BE693E10E94873403
:108C10000E94D231882309F45CC48F5F8093810560
:108C2000E82EF12C833330F5EE0CFF1CF092C813C4
:108C3000E092C7130093BB131093BE138EE090E134
:108C4000A0E0B0E08093BF139093C013A093C11332
:108C5000B093C2138BE693E10E9487341092C8133D
:108C60001092C7132BC03093C8132093C7131093CF
:108C7000BB1394CF84E690E09093C8138093C713FE
:108C80000093BB131093BE138EE090E1A0E0B0E020
:108C90008093BF139093C013A093C113B093C213DA
:108CA0008BE693E10E948734A2E3EA1AA0E8FA0A6D
:108CB000EE0CFF1CF092C813E092C7130093BB1395
:108CC0001093BE138FE090E1A0E0B0E08093BF135B
:108CD0009093C013A093C113B093C2138BE693E19A
:108CE0000E9487340E94D23190E09093C813809301
:108CF000C71385E08093BB1382E88093BE1386E19F
:108D000090E1A0E0B0E08093BF139093C013A093D4
:108D1000C113B093C2138BE693E10E94873420E025
:108D200030E0A901609180127091811280918212CD
:108D3000909183120F94052C20E030E048EC52E42F
:108D40000F949B250F94712D7093C8136093C713D4
:108D500005E00093BB1312E81093BE1386E290E186
:108D6000A0E0B0E08093BF139093C013A093C11311
:108D7000B093C2138BE693E10E9487348091650221
:108D8000909166029093C8138093C7130093BB130E
:108D90001093BE1380E093E1A0E0B0E08093BF1396
:108DA0009093C013A093C113B093C2138BE693E1C9
:108DB0000E94873420E030E040E251E46091520CA0
:108DC0007091530C8091540C9091550C0F949B25ED
:108DD0000F94782D7093C8136093C7130093BB133F
:108DE0001093BE1382E492E1A0E0B0E08093BF1341
:108DF0009093C013A093C113B093C2138BE693E179
:108E00000E94873420E030E040E251E46091560C4B
:108E10007091570C8091580C9091590C0F949B2590
:108E20000F94782D7093C8136093C7130093BB13EE
:108E30001093BE1386E492E1A0E0B0E08093BF13EC
:108E40009093C013A093C113B093C2138BE693E128
:108E50000E94873420E030E040E251E460915A0CF7
:108E600070915B0C80915C0C90915D0C0F949B2534
:108E70000F94782D7093C8136093C7130093BB139E
:108E80001093BE138AE492E1A0E0B0E08093BF1398
:108E90009093C013A093C113B093C2138BE693E1D8
:108EA0000E94873420E030E040E251E460915E0CA3
:108EB00070915F0C8091600C9091610C0F949B25D8
:108EC0000F94782D7093C8136093C7130093BB134E
:108ED0001093BE138EE492E1A0E0B0E08093BF1344
:108EE0009093C013A093C113B093C2138BE693E188
:108EF0000E94873420E030E048EC52E46091781220
:108F00007091791280917A1290917B120F949B2527
:108F10000F94712D7093C8136093C7130093BB1304
:108F20001093BE1386E392E1A0E0B0E08093BF13FC
:108F30009093C013A093C113B093C2138BE693E137
:108F40000E94873420E030E048EC52E460917C12CB
:108F500070917D1280917E1290917F120F949B25CB
:108F60000F94712D7093C8136093C7130093BB13B4
:108F70001093BE138AE392E1A0E0B0E08093BF13A8
:108F80009093C013A093C113B093C2138BE693E1E7
:108F90000E94873480917502909176029093C81355
:108FA0008093C7130093BB131093BE1382E592E125
:108FB000A0E0B0E08093BF139093C013A093C113BF
:108FC000B093C2138BE693E10E94873480917302C1
:108FD000909174029093C8138093C7130093BB13AE
:108FE0001093BE1384E592E1A0E0B0E08093BF133C
:108FF0009093C013A093C113B093C2138BE693E177
:109000000E94873420E030E040E251E46091F011AA
:109010007091F1118091F2119091F3110F949B25B1
:109020000F94782D7093C8136093C7130093BB13EC
:109030001093BE1386E592E1A0E0B0E08093BF13E9
:109040009093C013A093C113B093C2138BE693E126
:109050000E9487342CEA35EC47E25EE36091F4111C
:109060007091F5118091F6119091F7110F94FF2CEA
:1090700020E030E040E251E40F949B250F94782DDE
:109080007093C8136093C7130093BB131093BE1360
:109090008AE592E1A0E0B0E08093BF139093C01303
:1090A000A093C113B093C2138BE693E10E9487345F
:1090B0002CEA35EC47E25EE36091F8117091F9110A
:1090C0008091FA119091FB110F949B2520E030E0E4
:1090D00040E251E40F949B250F94782D7093C813B0
:1090E0006093C7130093BB131093BE138EE592E1F8
:1090F000A0E0B0E08093BF139093C013A093C1137E
:10910000B093C2138BE693E10E94873420E030E0F5
:1091100040E251E460918511709186118091871130
:10912000909188110F949B250F94782D7093C813FC
:109130006093C7130093BB131093BE1382E692E1B2
:10914000A0E0B0E08093BF139093C013A093C1132D
:10915000B093C2138BE693E10E9487342CEA35EC7E
:1091600047E25EE36091891170918A1180918B11C1
:1091700090918C110F94FF2C20E030E040E251E4FC
:109180000F949B250F94782D7093C8136093C71389
:109190000093BB131093BE1386E692E1A0E0B0E00B
:1091A0008093BF139093C013A093C113B093C213C5
:1091B0008BE693E10E9487342CEA35EC47E25EE3CC
:1091C00060918D1170918E1180918F1190919011FD
:1091D0000F949B2520E030E040E251E40F949B2562
:1091E0000F94782D7093C8136093C7130093BB132B
:1091F0001093BE138AE692E1A0E0B0E08093BF1323
:109200009093C013A093C113B093C2138BE693E164
:109210000E94873480919A0C811105C080919C0C2A
:10922000882309F46DC06091EB117091EC11072E49
:10923000000C880B990B0F943C2520E030E048ECA3
:1092400052E40F949B256B017C016091ED117091AC
:10925000EE11072E000C880B990B0F943C259B01F7
:10926000AC01C701B6010F94FF2C0F94782D653621
:10927000710510F064E670E07093C8136093C71333
:1092800005E00093BB1312E81093BE1384E290E153
:10929000A0E0B0E08093BF139093C013A093C113DC
:1092A000B093C2138BE693E10E9487346091EB1177
:1092B0007091EC11072E000C880B990B0F943C2534
:1092C0006B017C0120E030E04AE253E40F94652E0C
:1092D000181624F480919A0C811146C16091ED1109
:1092E0007091EE11072E000C880B990B0F943C2502
:1092F0009B01AC01C701B6010F94652E87FFAFC17A
:109300008091900C882339F180918F0C91E0980F17
:1093100090938F0C90E09093C8138093C71385E0CF
:109320008093BB1382E88093BE1382E490E1A0E0B7
:10933000B0E08093BF139093C013A093C113B09378
:10934000C2138BE693E10E94873480918F0C8A30A0
:1093500010F010928F0C0E94122C882309F4B5C1D2
:109360006091880C7091890CEE24E394F12C6115C6
:109370007105A9F090E080E00F943A2520E030E0FC
:1093800040E85EE30F949B250F94E32C20E030E04F
:1093900040E85FE30F94052C0F94782D7B0101E0EA
:1093A00010E080918A0C811102C010E000E08091F1
:1093B000AF129091B0128F3F980711F40E94A3B39F
:1093C0009093B0128093AF12080F191FB80190E06C
:1093D00080E00F943A2520E030E040E85EE30F940F
:1093E0009B250F94E32C4B015C01F092C813E09293
:1093F000C71305E00093BB1312E81093BE1380E17E
:1094000093E1A0E0B0E08093BF139093C013A093CA
:10941000C113B093C2138BE693E10E948734C50158
:10942000B4010F94782D7093C8136093C713009301
:10943000BB131093BE1382E193E1A0E0B0E08093F0
:10944000BF139093C013A093C113B093C2138BE6C4
:1094500093E10E9487340BE014E1AAE1FA2E809197
:109460003D0590913E0520917F0530918005891B37
:109470008F7309F449C12A3131050CF0DBC1909199
:109480003D0580913E054FEF5FEF981749F0E82FBB
:10949000F0E0E35CFA4F42818F5F8F7380933E056B
:1094A000F901E55FFB4E408380910B148A3509F08A
:1094B000B3C162E070E080E090E00E948F2C809168
:1094C0007F059091800501969093800580937F059C
:1094D000C6CF1092C8131092C713ACCB6091ED1198
:1094E0007091EE11072E000C880B990B0F943C2500
:1094F00020E030E0A9010F943525811134C98CE0BA
:1095000090E09093C8138093C71385E08093BB13BA
:1095100082E88093BE1384E190E1A0E0B0E0F3CB59
:109520008DE090E09093C8138093C71385E08093FB
:10953000BB1382E88093BE1384E190E1A0E0B0E029
:109540008093BF139093C013A093C113B093C21321
:109550008BE693E10E9487348091A10C811101C0B8
:1095600081E08093A10CDBCB10929A0C20E030E0DC
:1095700040E251E46091920C7091930C8091940CB4
:109580009091950C0F949B250F94712D7093C81397
:109590006093C7130093BB131093BE1384E590E14F
:1095A000A0E0B0E08093BF139093C013A093C113C9
:1095B000B093C2138BE693E10E94873420E030E041
:1095C00040E251E46091960C7091970C8091980C58
:1095D0009091990C0F949B250F94712D7093C81343
:1095E0006093C7130093BB131093BE1388E590E1FB
:1095F000A0E0B0E08093BF139093C013A093C11379
:10960000B093C2138BE693E10E94873488EA97E116
:109610000E9444388AE00E940B3881E09AE59093DA
:10962000C8138093C71381E490E09093CA1380938A
:10963000C91387E08093BB131093BE1384E890E0B6
:10964000A0E0B0E08093BF139093C013A093C11328
:10965000B093C2138BE693E10E94873451CE6091A0
:109660009C0C662309F44CCE062E000C770B8FE879
:1096700097E10E9442418AE00E940B3810929C0CB4
:1096800084E090E09093C8138093C71385E08093A3
:10969000BB1312E81093BE138EE890E1A0E0B0E097
:1096A0008093BF139093C013A093C113B093C213C0
:1096B0008BE693E10E94873481E09AE59093C8138A
:1096C0008093C71383E590E0B0CF1092C813109237
:1096D000C71305E00093BB1312E81093BE1380E19B
:1096E00093E1A0E0B0E08093BF139093C013A093E8
:1096F000C113B093C2138BE693E10E94873410929A
:10970000C8131092C71393CE121613060CF492C00E
:1097100080916F1390917013A0917113B091721397
:109720008C34E0E19E07A105B10509F4D7C98A345C
:109730009041A105B10509F4D1C920E030E040E233
:1097400051E46091280C7091290C80912A0C909121
:109750002B0C0F949B250F94712D7093C81360935D
:10976000C71305E00093BB1312E81093BE1388E4FF
:1097700090E1A0E0B0E08093BF139093C013A0935A
:10978000C113B093C2138BE693E10E94873420E0AB
:1097900030E040E251E460912C0C70912D0C8091EE
:1097A0002E0C90912F0C0F949B250F94712D70937C
:1097B000C8136093C7130093BB131093BE138AE4BE
:1097C00090E1A0E0B0E08093BF139093C013A0930A
:1097D000C113B093C2138BE693E10E94873420E05B
:1097E00030E040E251E46091300C7091310C809196
:1097F000320C9091330C0F949B250F94712D709324
:10980000C8136093C7130093BB131093BE138CE46B
:1098100090E1A0E0B0E056C9121613060CF01FCE7E
:10982000F8012F2D11922A95E9F7109280051092D8
:109830007F0515CE90916C1380910B14981321C065
:1098400090916D1380910C1498131BC02330310537
:10985000C4F090910D1490936B1380910E1480932B
:109860006E139330D1F4982F9D7F9038B1F490917E
:109870000F149F3409F059C0909110149B3409F0D3
:1098800054C0EBE0F4E18AE1DF011D928A95E9F72B
:109890001092800510927F053BCF833809F045C0B8
:1098A00080910F1490911014982789279827B0E081
:1098B000A0E080936F1390937013A0937113B093F3
:1098C0007213C0901114D12CF12CE12CC09273139F
:1098D000D0927413E0927513F092761322E134E182
:1098E00040E050E0BA014C155D056E057F0508F0BB
:1098F0004AC0DB01CA01B695A7959795879506964C
:10990000880F991FFC01E559FC4ED9018C911196E5
:109910009C91892798278927918380834E5F5F4F89
:109920006F4F7F4F2E5F3F4FDECF813861F58091C3
:109930000F1490E0B0E0A0E080936F139093701349
:10994000A0937113B093721380911014482F50E0BC
:1099500070E060E040937313509374136093751339
:1099600070937613A1E1B4E1E7E7F3E190E030E032
:1099700020E08217930739F04D9150E041935193C5
:109980002F5F3F4FF6CFEBE0F4E18AE1DF011D925C
:109990008A95E9F71092800510927F050E94BEFD1E
:1099A000B7CE3F924F925F926F927F928F929F922B
:1099B000AF92BF92CF92DF92EF92FF920F931F93DD
:1099C000CF93DF938091390587FD38C080913A05A8
:1099D0008370A1F5C0918412D0918512488159817C
:1099E0006A817B8189E197E10E9420414C815D8100
:1099F0006E817F8180E69FE20E942041409180122B
:109A00005091811260918212709183128DE59FE2D4
:109A10000E9420418AE0DF91CF911F910F91FF902A
:109A2000EF90DF90CF90BF90AF909F908F907F90FE
:109A30006F905F904F903F900C940B38609078122D
:109A40007090791280907A1290907B12A0907C1284
:109A5000B0907D1200917E1210917F12C090801202
:109A6000D0908112E0908212F090831288E50E94DB
:109A7000941EC82F882309F49AC00E949A24362E77
:109A8000472E582ED92F20E030E046E953EC0F94B2
:109A9000652E87FD0DC020E030E046E953E4632DDC
:109AA000742D852D9D2F0F94352518160CF081C02F
:109AB0006CE271E086E097E10E9442416CE271E065
:109AC00081E097E10E9442418EEF96E10E94443886
:109AD000C0E089E50E94941E882361F10E949A24C7
:109AE000362E472E582ED92F20E030E046E953EC91
:109AF0000F94652E87FD0DC020E030E046E953E469
:109B0000632D742D852D9D2F0F94352518160CF07F
:109B100055C06CE271E08BEE96E10E9442416CE22E
:109B200071E086EE96E10E94424183EE96E10E944A
:109B30004438C0E08AE50E94941E882309F443C09B
:109B40000E949A246B017C0120E030E040E151EC5E
:109B50000F94652E87FD0AC020E030E040E151E41B
:109B6000C701B6010F94352518166CF567EF7FEF26
:109B700081ED96E10E94424169E070E08CEC96E153
:109B80000E94424189EC96E1DF91CF911F910F91A4
:109B9000FF90EF90DF90CF90BF90AF909F908F900D
:109BA0007F906F905F904F903F900C944438C1E04D
:109BB00090CF632C742C852C9D2E8BCFA32CB42C92
:109BC000052D1D2FB7CFCC23E1F0C301D401809325
:109BD000781290937912A0937A12B0937B12C501F8
:109BE000D80180937C1290937D12A0937E12B09343
:109BF0007F12C0928012D0928112E0928212F09273
:109C00008312DF91CF911F910F91FF90EF90DF9022
:109C1000CF90BF90AF909F908F907F906F905F900C
:109C20004F903F9008958FED97E00C94443889ED64
:109C300097E00C94443884E690E09093C4058093B8
:109C4000C3051092E4051092E3050C9495DBEF92A6
:109C5000FF920F931F93CF93DF93CDB7DEB7629739
:109C60000FB6F894DEBF0FBECDBF0E94152A882321
:109C700009F43FC04AEE53E082FF02C04EEC53E0CD
:109C80002AEE33E081FF02C020ED33E080FD2EC0DC
:109C90008AEE93E05F934F933F932F939F938F931D
:109CA00083E499E19F938F938E010F5F1F4F1F9362
:109CB0000F930F94CC240E94174EC8010E941238B3
:109CC000C8010E942EE40FB6F894DEBF0FBECDBFD0
:109CD00081E062960FB6F894DEBF0FBECDBFDF9174
:109CE000CF911F910F91FF90EF90089582ED93E037
:109CF000D1CF80E0EECFCF92DF92EF92FF928AE554
:109D00000E94941E882309F45AC00E949A2420E0DD
:109D100030E040E050EC0F943525C12CD12CE12CE3
:109D200090ECF92E87FD0FC00E949A2420E030E0CD
:109D300040E050E40F94652E18160CF462C00E94A7
:109D40009A246B017C0120915A0C30915B0C40915C
:109D50005C0C50915D0CC701B6010F949B250F94CC
:109D6000712DCB010E9447FD80E50E94461E8111A6
:109D70004EC0A7019601609180127091811280916E
:109D80008212909183120F94052C6093801270932D
:109D9000811280938212909383120E94174E4091F9
:109DA00080125091811260918212709183128AEB1D
:109DB00096E10E9420418AE00E940B3805C083E5AD
:109DC0000E94941E8111A1CF8091390587FD24C086
:109DD00080913A05837001F50E94174E40918012E0
:109DE0005091811260918212709183128BEA96E1F8
:109DF0000E9420418AE0FF90EF90DF90CF900C947A
:109E00000B38C12CD12CE12C80E4F82E9CCF0E9481
:109E100062248111AECFD8CF82E50E94461E811107
:109E2000DBCFFF90EF90DF90CF900895CF9384E544
:109E30000E94941EC0E08823D9F00E944224C82FBB
:109E40001816B4F40E94174E8DE40E940B388091CE
:109E50003405909135050E94E2E16C2FCC0F770B11
:109E600088EA9FE00E9442418AE00E940B38CFEFCF
:109E70008C2FCF9108954F925F926F927F928F9225
:109E80009F92AF92BF92CF92DF92EF92FF92CF93C9
:109E9000DF93CDB7DEB72C970FB6F894DEBF0FBEB9
:109EA000CDBF4090D0085090D1086090D2087090FB
:109EB000D3082091470230914802409149025091C5
:109EC0004A02C301B2010F94052C69837A838B8304
:109ED0009C838090D4089090D508A090D608B0902C
:109EE000D70820914B0230914C0240914D02509185
:109EF0004E02C501B4010F94052C6D837E838F83C0
:109F00009887C090D808D090D908E090DA08F090EF
:109F1000DB0820914F023091500240915102509144
:109F20005202C701B6010F94052C69877A878B8787
:109F30009C872091530230915402409155025091D8
:109F40005602C301B2010F94052C2B013C01209154
:109F50005702309158024091590250915A02C5015E
:109F6000B4010F94052C4B015C0120915B023091F0
:109F70005C0240915D0250915E02C701B6010F94F0
:109F8000052C6B017C010E94174E83EE9EE00E941F
:109F9000443883E50E94461E882321F00E946224F3
:109FA0008093450280914502811151C08AEC9EE068
:109FB0000E9444388BED9EE00E94443849815A81CA
:109FC0006B817C8181E19EE10E9420414D815E8117
:109FD0006F81788580E69FE20E94204149855A85FD
:109FE0006B857C858DE59FE20E94204189ED9EE096
:109FF0000E94443881ED9EE00E944438B301A201E2
:10A0000081E19EE10E942041B501A40180E69FE22A
:10A010000E942041B701A6018DE59FE20E942041E8
:10A020008AE02C960FB6F894DEBF0FBECDBFDF914D
:10A03000CF91FF90EF90DF90CF90BF90AF909F9027
:10A040008F907F906F905F904F900C940B388EECB8
:10A050009EE0AECF5F926F927F928F929F92AF926F
:10A06000BF92CF92DF92EF92FF920F931F93CF9305
:10A07000DF931F92CDB7DEB77C0139018B015B0105
:10A08000A40EB51ED12CC12CA016B10609F450C0E7
:10A09000F70180809180F80151908F015982C401AD
:10A0A0000F94532B5816B9F1652DC4010F945B2BF7
:10A0B000FFEFCF1ADF0AC6018F779927892B21F18D
:10A0C00062E070E080E090E00E94DBFCC4010F944D
:10A0D000532B99818917F9F00E94174E8FE694E06F
:10A0E0000E94443881E00F90DF91CF911F910F9132
:10A0F000FF90EF90DF90CF90BF90AF909F908F90A8
:10A100007F906F905F90089562E070E080E090E053
:10A110000E940826DBCFBE016F5F7F4FC3010E9404
:10A12000B6E0F70180819181019691838083ACCF65
:10A1300080E0D9CFDF92EF92FF920F931F93CF93DE
:10A14000DF93CDB7DEB7CA5AD1090FB6F894DEBF98
:10A150000FBECDBFCF55DF4F188219821A821B82E6
:10A16000C15AD0408091D4039091D503A091D603D9
:10A17000B091D703CB55DF4F88839983AA83BB83E4
:10A18000C55AD04084E690E09093C4058093C305FF
:10A190001092E4051092E3051092E50523EE35E0F8
:10A1A00044E050E0BE016B557F4F83EC95E00E9488
:10A1B0002A508091C3059091C40502969093C405DE
:10A1C0008093C3051092E4051092E30581E0C65523
:10A1D000DF4F8883CA5AD040CE0186559F4F0E94D8
:10A1E000BAD123EE35E048E450E06EE37CE083EC46
:10A1F00095E00E942A5023EE35E040E150E06DEDFD
:10A2000078E083EC95E00E942A508AE097EDA3EA7B
:10A21000BCE3CF55DF4F88839983AA83BB83C15AA0
:10A22000D040CE018F559F4F0E94B1D186E098E07B
:10A230000E94CCD186E292E00E94C3D182E292E0F9
:10A240000E94B1D18091CC089091CD08A091CE0808
:10A25000B091CF0889839A83AB83BC838E010F5F53
:10A260001F4FC8010E94B1D1CF55DF4F188219820C
:10A270001A821B82C15AD0407E018DE6E80EF11C85
:10A2800083E0D7018C938983CE018F559F4F0E9425
:10A29000B1D1C7010E94BAD1C8010E94BAD14AE027
:10A2A000D42EDA94DD2031F0CE018F559F4F0E94DD
:10A2B000B1D1F7CF88E792E10E94CCD1CF55DF4FE3
:10A2C000188219821A821B82C15AD0403AE0D32EDA
:10A2D000DA94DD2031F0CE018F559F4F0E94B1D12D
:10A2E000F7CF85E0D82ED982F701D082C8010E942D
:10A2F000BAD1C7010E94BAD123EE35E048E050E060
:10A3000066ED75E083EC95E00E942A5023EE35E07F
:10A3100048E050E06EEC75E083EC95E00E942A5036
:10A3200023EE35E044E650E060E977E083EC95E029
:10A330000E942A5019828FEFD7018C93C8010E9486
:10A34000C3D1C7010E94BAD123EE35E044E050E00A
:10A3500066EE72E083EC95E00E942A508091A70699
:10A360008983C8010E94C3D1198A1A8A1B8A1C8A50
:10A3700080E090E0A0E8BFE38D879E87AF87B88B31
:10A380008091F0119091F111A091F211B091F3111F
:10A3900089839A83AB83BC832CEA35EC47E25EE386
:10A3A0006091F4117091F5118091F6119091F7116F
:10A3B0000F94FF2C6D837E838F8398872CEA35EC76
:10A3C00047E25EE36091F8117091F9118091FA1102
:10A3D0009091FB110F949B2569877A878B879C87C7
:10A3E00023EE35E044E150E0B80183EC95E00E94B3
:10A3F0002A5084E190E09A838983C8010E949FD10A
:10A400008091851190918611A0918711B09188114A
:10A4100089839A83AB83BC832CEA35EC47E25EE305
:10A420006091891170918A1180918B1190918C119A
:10A430000F94FF2C6D837E838F8398872CEA35ECF5
:10A4400047E25EE360918D1170918E1180918F11C2
:10A45000909190110F949B2569877A878B879C87B1
:10A46000C8010E94A8D18CE0EDE7F2E0D80101908C
:10A470000D928A95E1F7C8010E94A8D11982C801FE
:10A480000E94BAD18FE790E09A838983C8010E9425
:10A490009FD1E9E8F2E0D80101900D92DA94E1F75A
:10A4A00023EE35E045E050E0B80183EC95E00E94F2
:10A4B0002A508091CD058983C8010E94C3D180E2D2
:10A4C000EEE8F2E0D80101900D928A95E1F723EED3
:10A4D00035E040E250E0B80183EC95E00E942A505C
:10A4E000F7011082C7010E94C3D189EF97E00E9453
:10A4F000C3D185EF97E00E94B1D1CF55DF4F1882CD
:10A5000019821A821B82C15AD040CE018F559F4FAB
:10A510000E94B1D180E2D8011D928A95E9F723EE1D
:10A5200035E040E250E0B80183EC95E00E942A500B
:10A53000FE01F99688E0DF011D928A95E9F744E66D
:10A5400050E060E070E049835A836B837C834D83E5
:10A550005E836F83788783E090E0A0E0B0E0898736
:10A560009A87AB87BC874D875E876F87788B498BCF
:10A570005A8B6B8B7C8B8D8B9E8BAF8BB88F898F1F
:10A580009A8FAB8FBC8F8D8F9E8FAF8FB8A38EE1CC
:10A5900090E0A0E0B0E089A39AA3ABA3BCA38DA3F5
:10A5A0009EA3AFA3B8A789A79AA7ABA7BCA78DA75F
:10A5B0009EA7AFA7B8AB89AB9AABABABBCAB8DAB2F
:10A5C0009EABAFABB8AF23EE35E040E450E0B8014E
:10A5D00083EC95E00E942A5090E1D92EF8018D2D50
:10A5E00011928A95E9F723EE35E040E150E0B80199
:10A5F00083EC95E00E942A50D8011D92DA94E9F785
:10A6000023EE35E040E150E0B80183EC95E00E9494
:10A610002A50CF55DF4F188219821A821B82C15AE5
:10A62000D040CE018F559F4F0E94B1D12CE0D22E49
:10A63000F8018D2D11928A95E9F723EE35E04CE073
:10A6400050E0B80183EC95E00E942A508CE6D801D6
:10A650001D928A95E9F723EE35E04CE650E0B8010B
:10A6600083EC95E00E942A5087EB95E00E94A8D1E8
:10A6700023EE35E048E050E065EC75E083EC95E0D2
:10A680000E942A50F7011192DA94E9F7C755DF4F7B
:10A690001882C95AD04080E090E0A0E4B0E4C356EC
:10A6A000DF4F88839983AA83BB83CD59D040C701EC
:10A6B0000E94CCD1CE0187559F4F0E94BAD1CE01C6
:10A6C00083569F4F0E94B1D180E3D7011D928A9596
:10A6D000E9F78DE89CE10E9444388AE00E940B383B
:10A6E00023EE35E040E350E0B70183EC95E00E94B3
:10A6F0002A508091E505811128C00091C305109171
:10A70000C4058091E3059091E405F701918380836E
:10A7100084E690E09093C4058093C30523EE35E072
:10A7200044E050E066EF72E083EC95E00E942A502E
:10A73000C7010E949FD191E00536134009F490E0D3
:10A740008091E505892B8093E5058091E5058111D0
:10A7500005C060E081EC9CE10E94B23F81EA9CE18F
:10A760000E9444388AE00E940B389091E50581E010
:10A770008927C655DF4F0FB6F894DEBF0FBECDBF99
:10A78000DF91CF911F910F91FF90EF90DF9008958F
:10A79000CF93DF9300D01F92CDB7DEB780919306A1
:10A7A0008823C1F083E390E09C838B831A82198213
:10A7B0009E012F5F3F4F40E150E064E976E0CE011B
:10A7C00003960E942A5081EA9CE10E9444388AE064
:10A7D0000E940B380F900F900F900F90DF91CF9148
:10A7E0000895CF92DF92EF92FF92CF93C82F80917E
:10A7F00024118150823008F069C00E94A73A10925B
:10A8000024110E940EFD6093AF057093B0058093F4
:10A81000B1059093B205C090B305D090B405E09017
:10A82000B505F090B6050E947C2BAB01BC014093AE
:10A83000B3055093B4056093B5057093B605809148
:10A84000980690919906A0919A06B0919B068C1952
:10A850009D09AE09BF09840F951FA61FB71F8093DE
:10A86000980690939906A0939A06B0939B06C111FF
:10A870000AC0C1E00E94C8538C2FCF91FF90EF9087
:10A88000DF90CF900895809196069091970601965B
:10A8900090939706809396060E947C2BC0909C060E
:10A8A000D0909D06E0909E06F0909F06C616D706B3
:10A8B000E806F906F0F60E947C2B60939C067093E4
:10A8C0009D0680939E0690939F06D3CFC0E0D2CF83
:10A8D00081E00C94F1530E94C1BE0E94685480E054
:10A8E0000E94DDF88091E9068130A1F40E94134EA8
:10A8F00082E697E00E94443860E088E597E00E9495
:10A90000B23F6EE571E080E090E00E94082688E0AA
:10A910008093E9060895CF92DF92EF92FF921F9302
:10A92000CF93DF9300D01F92CDB7DEB78EEEC82E47
:10A9300082E0D82EE12CF12CC982DA82EB82FC82F3
:10A94000BE016F5F7F4F8AE50E94693381110EC09F
:10A9500010E0812F0F900F900F900F90DF91CF910B
:10A960001F91FF90EF90DF90CF9008950E94BF332A
:10A97000C982DA82EB82FC82BE016F5F7F4F8AE57B
:10A980000E946933182F882319F30E94134E8CE319
:10A9900098E00E9444380E946B54DBCFCF92DF9244
:10A9A000EF92FF921F93CF93DF9300D01F92CDB70A
:10A9B000DEB78EEEC82E82E0D82EE12CF12CC982B3
:10A9C000DA82EB82FC82BE016F5F7F4F8AE00E94D9
:10A9D000693381110EC010E0812F0F900F900F90FE
:10A9E0000F90DF91CF911F91FF90EF90DF90CF906C
:10A9F00008950E94BF330E9489330E94A4330E94AD
:10AA00008933C982DA82EB82FC82BE016F5F7F4F9D
:10AA10008AE00E946933182F8823E9F20E94134EBE
:10AA20008FEF97E00E9444380E946B54D5CFCF93AC
:10AA3000DF9300D01F921F92CDB7DEB781E08093E5
:10AA4000930680E1E4E9F6E0DF011D928A95E9F7DB
:10AA50000E94C85386E18D8382E390E09C838B83C0
:10AA60001A8219829E012F5F3F4F41E050E0BE01E4
:10AA70006B5F7F4FCE0103960E942A500F900F907C
:10AA80000F900F900F90DF91CF910895CF93DF93A8
:10AA9000CDB7DEB7A8970FB6F894DEBF0FBECDBF17
:10AAA0008C01F42E0E94C1BE0E94134E88E397E0F1
:10AAB0000E9444380115110511F40FE217E080914E
:10AAC000890580FD79C08160809389058BE197E0DD
:10AAD0000E9444388AE00E940B38CC24C3948AE553
:10AAE000D82ED092C813C092C7138FE090E09093F5
:10AAF000CA138093C91397E0792E7092BB1322E892
:10AB0000E22EE092BE1334E8832E912CA12CB12CBE
:10AB10008092BF139092C013A092C113B092C2133F
:10AB20008BE693E10E948734D092C813C092C7137A
:10AB300088E590E09093CA138093C9137092BB1379
:10AB4000E092BE138092BF139092C013A092C113E3
:10AB5000B092C2138BE693E10E9487348AE2898324
:10AB60008A838B838C83F801DE011596BE016F5FAB
:10AB70007F4FCD01861B970B2491319621110CC07C
:10AB8000FB01E80FF91F8AE29F01261B370B2832D1
:10AB9000310524F48193F8CF2D93EBCF20E630E1FB
:10ABA00040E050E08BE693E10E94D1E06AE070E083
:10ABB00080E090E00E948F2C61E086E297E00E94A6
:10ABC0007F3F89EE93E030E6019729F0232F2A9505
:10ABD0000000E9F7F9CFF89489EE93E038EE019799
:10ABE00029F0232F2A950000E9F7F9CF0E94C1BE72
:10ABF000FF2031F00E94001F0E94191FA895FECF70
:10AC00000E94FE1EF9CF8091E806882319F0109269
:10AC1000E806089540E070E060E084EB98E10E946F
:10AC200046558091A40C9091A50C2FEF3FEF9817FB
:10AC300051F0E92FF0E0EC55F34F228130E09F5FB7
:10AC40009F779093A50CC90108951F920F920FB69C
:10AC50000F9211240F900FBE0F901F9018951F9206
:10AC60000F920FB60F9211240BB60F920F931F93F2
:10AC70002F933F934F935F936F937F938F939F9304
:10AC8000AF93BF93CF93DF93EF93FF93C091C60031
:10AC90000091A50CD091A40C11E01D0F1F7790918D
:10ACA0001704913108F09FC0E92FF0E08827E45A9B
:10ACB000F94A8F4F0D94FC2B6D569C56AB56BA56E5
:10ACC000C156F356C556F356C956CD56F356D1560E
:10ACD000D556D956E056F356EB56C03229F028F532
:10ACE000CA3011F0CD3031F5011731F0ED2FF0E021
:10ACF000EC55F34FC283D12FD093A40CFF91EF9169
:10AD0000DF91CF91BF91AF919F918F917F916F9183
:10AD10005F914F913F912F911F910F910F900BBE1B
:10AD20000F900FBE0F901F901895CD3481F081E0E9
:10AD3000CE3471F080E10CC0CA3338F4C033A0F6D1
:10AD4000C03291F2CD32B1F7CFCFCD3499F782E056
:10AD500080931704C9CFC13359F018F4C03221F2DF
:10AD6000E9CF88E0C433A1F38BE0C83389F3E2CFA5
:10AD700083E0EECF84E0C03359F386E0C13341F382
:10AD8000D9CF85E0C833B1F6E3CF87E0C23391F67F
:10AD9000DFCF89E0C13371F6DBCF8AE0C03351F6F3
:10ADA000D7CF8CE0C73331F6D3CF8DE0C63311F661
:10ADB000CFCFC03209F498CF8EE0C33549F2BACF75
:10ADC00080ED8C0F8A3008F08FCF9FE090931704AE
:10ADD0008093180489CFCA3019F0CD3009F084CFA0
:10ADE0001092170481CFCA3019F0CD3009F07CCF12
:10ADF000809125148823A1F3973089F038F4953099
:10AE000079F710923C021092270CEACF9A3059F051
:10AE10009F3031F7809118040E94A631E1CF81E084
:10AE200080931106DDCF81E080931006D9CF8EBDCF
:10AE30000DB407FEFDCF08958FEF8EBD0DB407FE54
:10AE4000FDCF8EB50895909164009B7F9093640030
:10AE5000982F906A96959CBD80FD03C091E0863046
:10AE600009F490E09DBD0895CF93DF93EB010E941C
:10AE70004438CE01DF91CF910C940BAF2F923F92CB
:10AE80004F925F926F927F928F929F92AF92BF92FA
:10AE9000CF92DF92EF92FF920F931F93CF93DF93A6
:10AEA000009709F0AAC110928C0C10928B0C909311
:10AEB000880580938705BAE0CB2EB0E2DB2EE12C2B
:10AEC000F12C15E002E846015701C4E1D0E01092F0
:10AED0000E1310920D13109301130093041380921C
:10AEE000051390920613A0920713B092081381EBFA
:10AEF00092E10E94873421972FEF821A920AA20AC8
:10AF0000B20A209721F744E1C40ED11CE11CF11CC8
:10AF10008AE5C81680E2D806E104F104A1F6C12C46
:10AF2000A0E2DA2EE12CF12CD5E0C2E810920E134B
:10AF300010920D13D0930113C0930413C092051304
:10AF4000D0920613E0920713F092081381EB92E17E
:10AF50000E94873410920E1310920D13D093011398
:10AF6000C0930413D701C6018C529F4FAF4FBF4F00
:10AF70008093051390930613A0930713B0930813BF
:10AF800081EB92E10E948734EFEFCE1ADE0AEE0ADF
:10AF9000FE0AFAE0CF16F0E2DF06E104F10431F632
:10AFA000FEEDCF2EF0E2DF2EE12CF12CD5E0C2E851
:10AFB00010920E1310920D13D0930113C09304132B
:10AFC000C0920513D0920613E0920713F092081373
:10AFD00081EB92E10E9487342FEFC21AD20AE20A73
:10AFE000F20A46EEC41640E2D406E104F10401F789
:10AFF000CC24C394E2E1DE2EE12CF12C0AE010E037
:10B00000D5E0C2E810930E1300930D13D0930113F3
:10B01000C0930413C0920513D0920613E092071355
:10B02000F092081381EB92E10E94873410930E1383
:10B0300000930D13D0930113C0930413D701C601DD
:10B040008096A11DB11D8093051390930613A093C4
:10B050000713B093081381EB92E10E9487348FEFBE
:10B06000C81AD80AE80AF80AE5E0CE16E2E1DE06D8
:10B07000E104F10439F600918B0C10918C0C011550
:10B08000110509F0D6C080918A0C882309F4E1C02B
:10B090002AE030E240E050E068ED73E081EB92E1BD
:10B0A0000E94D1E0C1E0D0E003E010E0E0908B0C22
:10B0B000F0908C0C35E0332E42E8242E44244A9440
:10B0C000542C64E0662E712C7FE1C72E74E0D72EDD
:10B0D00080918B0C90918C0C800F911FE816F906D3
:10B0E00008F0D5C0C7010E94E8E1882309F481C0B7
:10B0F00080919F1162E971E1882311F06FE971E19C
:10B10000FB0101900020E9F7CF010197861B970B07
:10B11000F4E1FC9F9001FD9F300D1124265F3F4D0F
:10B1200050E040E0459710F0FB01128A81EB92E17C
:10B130000E94D1E0CE018F5F9D4EB0E0A0E021964D
:10B140004E0124E0880C991C2A95E1F7FDEF8F1A37
:10B15000FFE99F0AB12CA12C2091311424FF7EC05D
:10B1600070920E1360920D1330920113209204130B
:10B170008093051390930613A0930713B0930813BD
:10B1800081EB92E10E948734D0920E13C0920D138E
:10B1900030920113209204138092051390920613AB
:10B1A000A0920713B092081381EB92E10E948734BA
:10B1B000B70189E498E10E940E4180919F116FE9E7
:10B1C00071E1811102C062E971E186E498E10E94B7
:10B1D000345767EE7BE082E498E10E94345762E9DD
:10B1E00071E181E498E10E9434578DE398E10E9477
:10B1F00044382FEFE21AF20A6BCF20918B0C30917A
:10B200008C0CA90141505109609187057091880506
:10B210006817790738F42C5F3F4F30938C0C2093DC
:10B220008B0C45CE4430510508F43DCE24503109F5
:10B23000F4CF0430110569F480918A0C882331F031
:10B2400083E090E090938C0C80938B0CD0E0C0E076
:10B250002DCFD0E0C0E004E010E028CF10920E1314
:10B2600010920D1330920113209204138093051352
:10B2700090930613A0930713B093081381EB92E108
:10B280000E94873450920E1340920D1381CFDF91AC
:10B29000CF911F910F91FF90EF90DF90CF90BF90D3
:10B2A000AF909F908F907F906F905F904F903F9066
:10B2B0002F900895AF92BF92CF92DF92EF92FF92BC
:10B2C0000F931F93CF93DF93CDB7DEB7E6970FB6FB
:10B2D000F894DEBF0FBECDBF00913B0510913C0539
:10B2E000F80101900020E9F731976F01C01AD10AE7
:10B2F000F801CF01801B910B8C159D053CF48191C9
:10B300008F32B9F7DF0111971C92F3CF8BE1E1E5A2
:10B31000F4E1DE015C9601900D928A95E1F7F12C43
:10B32000E12CEC14FD040CF05DC0F801EE0DFF1DE6
:10B330008081811103C08FEFE81AF80A5801AE0C22
:10B34000BF1CF5018081882309F44CC0FFEFEF1A80
:10B35000FF0AF801EE0DFF1D7F01E01AF10A81914D
:10B360008111FACFCE014C960E949EB38BE1FE0173
:10B370007C96DE01119601900D928A95E1F7B50158
:10B38000CE0101960E94ACABCE0101960E94932F94
:10B390008FE20E940B3880919F1181113BC085EE96
:10B3A00093E00E940BAF8091311484FF1BC019827F
:10B3B0001C8221E0A501BE01645E7F4FCE01019693
:10B3C0000E94E0B5811129C08AE00E940B380E94DA
:10B3D000174EB50188E297E10E943457CE010196DD
:10B3E0000E94932F8AE00E940B38CE014C960E9457
:10B3F000932FE6960FB6F894DEBF0FBECDBFDF9158
:10B40000CF911F910F91FF90EF90DF90CF90BF9061
:10B41000AF9008958FE991E1C4CFCE014C960E9480
:10B420000DB38BE1FE013196DE015C9601900D9229
:10B430008A95E1F7CE0101960E94932F72CF2F9249
:10B440003F924F925F926F927F928F929F92AF92B4
:10B45000BF92CF92DF92EF92FF920F931F93CF9301
:10B46000DF9300D000D000D01F921F92CDB7DEB77F
:10B47000B82E8091910D843008F0D1C10E940EFD4C
:10B480006B017C018091910D811108C08091A40C09
:10B490009091A50C891B8F7709F4A4C681E6A82E8C
:10B4A00013C08A3019F08D3009F0F6C010928C0D5F
:10B4B00080912A0D90912B0DFC01EA5DF24F1682CE
:10B4C000892BF1F40E940EC28091910D843008F016
:10B4D000ECC08091A40C9091A50C891B8F7709F486
:10B4E000E4C00E94115697FFDCCF0E94134E85EBFB
:10B4F00095E00E9444388091A40C8093A50CE4CF81
:10B5000010922B0D10922A0D0CE21DE0F801819192
:10B51000803209F446C08E3409F0A9C060EB75E0B2
:10B52000C8010F94B2244C01892B41F06EE470E005
:10B53000C80104960F94532F009709F4C8014AE0FC
:10B5400050E070E060E001960F9422222B013C0154
:10B550008091260D9091270DA091280DB091290D75
:10B560000196A11DB11D481659066A067B0629F0F1
:10B5700060E08DE795E0892851F16AE270E0C8014A
:10B580000F94822F9C01009729F1982F901B912CEA
:10B59000992349F09150F801E90FF11D8081982617
:10B5A000F7CF8F01B3CF4AE050E070E060E0C9010F
:10B5B00001960F942222292D30E050E040E06217DE
:10B5C00073078407950751F060E08EE595E00E94CF
:10B5D00063E77ACF60E084E395E0F9CF4092260DEF
:10B5E0005092270D6092280D7092290D8091E906E6
:10B5F0008130E1F067E470E0C8010F94532F0097A9
:10B60000A9F04AE050E070E060E001960F94222239
:10B61000643071058105910548F483E994E00E9446
:10B62000443860E089E894E00E94B23FC092880705
:10B63000D0928907E0928A07F0928B0780912C0DB7
:10B640008B3309F441CF8091910D843008F03CCFC9
:10B650008091930D8A9DC00111246CE27DE08C568F
:10B66000924F0F945E2F80E00E941DE72DCF8091B6
:10B67000311480FFBBCF63E87DE2C8010F94B22490
:10B68000009731F0FC01838180538A3008F0AECFFF
:10B6900060E08AE095E09BCF2AE23DE04CE25DE08D
:10B6A0006CE87DE00E94141D0FCF8091311482FF61
:10B6B000B6C01A82198271E6F72EE0E1EE2EF9E6A5
:10B6C000DF2E8091910D843008F0A9C00E944C1D9E
:10B6D0008111A5C041E050E0BE016B5F7F4F85E95D
:10B6E00095E10E9460B10D8110E0019711F00FEF1C
:10B6F0001FEF80919D1590919E15A0919F15B0917F
:10B70000A01580932D1490932E14A0932F14B09312
:10B7100030140E944C1D0F3F100749F4811107C0DF
:10B720000E94134E83ED95E00E944438CACF4091A9
:10B73000930D242F30E00A3061F00D3051F0882352
:10B7400009F45FC089819A81009719F001969A8364
:10B75000898310929E0489819A81F29EF001F39E62
:10B76000F00D1124EF56F24FE80FF91F1382892BC9
:10B7700069F50E940EC20E944C1D882309F4A1CFD6
:10B780000E94836185E995E10E940DB380912814A0
:10B79000882391F18150809328148D9DC00111243C
:10B7A00062E08F5D994F0E9462B8E091281424E016
:10B7B000E29FF0011124E35EF94F60817181828183
:10B7C00093810E9465220E9415AB7BCF1A82198259
:10B7D00081E00E941DE780912D1490912E14A0917C
:10B7E0002F14B091301480938D0D90938E0DA093F3
:10B7F0008F0DB093900DBFCF0E9416B3E092E90673
:10B8000060CF4F9DA00111244C56524F9E012F5FD7
:10B810003F4F6EE974E0802F0E94141D52CF0E94AA
:10B820000EFD6B017C01B11004C0809123118823AF
:10B8300051F0C0927611D0927711E0927811F09287
:10B840007911BB24B3948091130590911405A091B4
:10B850001505B09116050097A105B105B1F040910D
:10B860007611509177116091781170917911840F50
:10B87000951FA61FB71FA7019601281B390B4A0B5E
:10B880005B0BDA01C901B7FF92C18091130290915D
:10B890001402A0911502B0911602892B8A2B8B2BD2
:10B8A00009F099C10E940EFD4B015C018091270CAB
:10B8B000811108C02091891290918A1281E0291388
:10B8C00001C080E02091EB113091EC1191E08927CB
:10B8D0002A3A31050CF480E091E04091A3045091A4
:10B8E000A4046091A5047091A604452B462B472B18
:10B8F00009F490E0981789F0882309F4BDC1D501B7
:10B90000C40180569444A24FBF4F8093A3049093E8
:10B91000A404A093A504B093A6044090340C5090C6
:10B92000350C6090360C7090370C20919F0430914C
:10B93000A0044091A1045091A204C301B2010F944C
:10B940003525882319F18091A3049091A404A09136
:10B95000A504B091A60440929F045092A004609266
:10B96000A1047092A204892B8A2B8B2B09F449C065
:10B97000D501C40180569444A24FBF4F8093A304C5
:10B980009093A404A093A504B093A6048091A3046B
:10B990009091A404A091A504B091A6040097A105DC
:10B9A000B10579F1881A990AAA0ABB0AB7FC29C01D
:10B9B0001092A3041092A4041092A5041092A6045D
:10B9C00083E396E00E94443860E08FE196E00E94B5
:10B9D000B23F8091ED119091EE111816190624F4E2
:10B9E00090E080E00E941C1F809182119091831151
:10B9F0001816190634F410928311109282110E94C5
:10BA000094BE8091AB049091AC04A091AD04B09130
:10BA1000AE0446015701881A990AAA0ABB0AD50141
:10BA2000C401B7FDB9C12091891290918A12409149
:10BA30002D0280912C02291323C190910109899F25
:10BA4000C0011124880F892F881F990B91958D8330
:10BA500080910209489FC0011124880F892F881FF7
:10BA6000990B91958E830E940EFD69837A838B8357
:10BA70009C8340E0BE016F5F7F4FCE0105960E9420
:10BA8000661C6D8170E089E00E9405FC41E0BE010A
:10BA90006F5F7F4FCE0105960E94661C6E8170E03D
:10BAA00087E00E9405FC80911C06882309F467C189
:10BAB0000091200210912102C80102972091ED11FE
:10BAC0003091EE11281739070CF459C180908A1271
:10BAD0008F82188619861A861B86809189129F800C
:10BAE000891509F4E7C0892D90E03CE5A32EA89EB6
:10BAF000F001A99EF00D1124EA5FF64F45895689A1
:10BB00006789708D452B462B472B81F4418D528DD3
:10BB1000638D748D452B462B472B41F4458D568DF7
:10BB2000678D70A1452B462B472BE1F12CE5B22EFA
:10BB3000B89E9001B99E300D1124A9014A5F564F5D
:10BB40001A01FA0161817281838194810F94B32E6D
:10BB50004B015C01F10161A172A183A194A10F9439
:10BB60003A252B013C01F10165A176A187A190A5A1
:10BB70000F943A259B01AC01C301B2010F94FF2C35
:10BB8000A50194010F949B254B015C012885398503
:10BB90004A855B850F94652E181624F4888699864D
:10BBA000AA86BB868F818F5F87708F8396CF0E9416
:10BBB000134E609186077091870782EE95E00E9490
:10BBC00034578AE00E940B3840E070E060E090E07B
:10BBD00080E00E9446559091891280918A129817B0
:10BBE00049F0C0927611D0927711E0927811F092DC
:10BBF000791158CEBB2019F01092AF0453CE0E9499
:10BC00000EFD0091761110917711209178113091ED
:10BC100079118090130290901402A0901502B090B8
:10BC20001602080D191D2A1D3B1D601B710B820B8E
:10BC3000930B97FDE1CF8091AF04811133CE81E06A
:10BC40008093AF045F9A8091380C8E7F8093380C7C
:10BC50008A9A8091380C8D7F8093380C80910801EE
:10BC600080958170809306018091380C8B7F809342
:10BC7000380C0E94FE1E16CE80E090E0DC0145CE1E
:10BC800020918A125CE5259F900111242A5F364F8E
:10BC9000F901EA5AFF4F9081899FC0011124880F52
:10BCA000892F881F990B91958D83295A3F4FF90150
:10BCB0008081D0CE20911A0230911B0240911C024B
:10BCC00050911D02688579858A859B850F949B25F7
:10BCD0004B015C01B801012E000C880B990B0F94ED
:10BCE0003C259B01AC01C501B4010F94052C69836F
:10BCF0007A838B839C8340911E0250911F02B8016E
:10BD0000CE0101960E94CCC189809A80AB80BC8014
:10BD10004090A7045090A8046090A9047090AA04D1
:10BD2000A3019201C501B4010F94352587FF16C008
:10BD300028E431EE4AE75FE3C301B2010F949B258B
:10BD400020E037ED43EA5CE30F94052CA501940154
:10BD50000F949B2569837A838B839C8369817A8185
:10BD60008B819C816093A7047093A8048093A9049D
:10BD70009093AA040F94712DCB010E941C1FF4E62E
:10BD8000CF0ED11CE11CF11CC092AB04D092AC04CC
:10BD9000E092AD04F092AE040E940EC28091E906DA
:10BDA000882309F4E0C180912602882309F4A3C006
:10BDB0008091ED0481119FC080912311811108C0F1
:10BDC00080912411813021F08091311482FF93C041
:10BDD000F894649B10C08091220290912302A0915C
:10BDE0002402B09125028093EA059093EB05A0937D
:10BDF000EC05B093ED056091EA057091EB0580913B
:10BE0000EC059091ED05789420E030E0A9010F94C5
:10BE1000352587FF70C001E00093ED048091231168
:10BE2000811167C088E496E00E9444388AE00E944D
:10BE30000B3884E08093A10C82E080938D0C81E02C
:10BE40009AE59093C8138093C7138EE490E0909383
:10BE5000CA138093C91387E08093BB1382E8809351
:10BE6000BE1384E890E0A0E0B0E08093BF1390930D
:10BE7000C013A093C113B093C2138BE693E10E9449
:10BE800087340E942F400093911140E36CE876E0E4
:10BE900084E799E00E94344061E088E699E00E94DE
:10BEA00016401091170560E010278CE399E069F4C3
:10BEB0008AE796E00E947F3F80E30E940B388AE089
:10BEC0000E940B3860E08DE596E00E947F3F88E697
:10BED00096E00E94443880E30E940B388AE00E947A
:10BEE0000B38112331F083E696E09093870C809312
:10BEF000860C0E94836190910901892F8095817041
:10BF0000109100021817C9F020913114206220937B
:10BF100031148093000290FD3FC164EF71E080E036
:10BF200090E00E9408260E9438B38091311483FD6E
:10BF30007CC1111133C10E94D9350E940EFD6B01E5
:10BF40007C01109117021123F1F0809118058823CC
:10BF5000D1F04091B0045091B1046091B20470915D
:10BF6000B30446015701841A950AA60AB70AB50117
:10BF7000A40177FD1AC0833009F42FC10CF01EC153
:10BF800081300CF023C1212F30E0A8EEB3E00F94F4
:10BF9000CD2BC60ED71EE81EF91EC092B004D0925B
:10BFA000B104E092B204F092B30480912411813084
:10BFB00009F073C00E940EFD6B017C018091B804F2
:10BFC0009091B904A091BA04B091BB04A701960165
:10BFD000281B390B4A0B5B0BDA01C901B7FD3AC0CC
:10BFE000D701C601805F984DAF4FBF4F8093B80413
:10BFF0009093B904A093BA04B093BB048090B305A6
:10C000009090B405A090B505B090B6050E947C2B29
:10C01000AB01BC014093B3055093B4056093B505E3
:10C020007093B6058091980690919906A0919A0612
:10C03000B0919B0688199909AA09BB09840F951F1D
:10C04000A61FB71F8093980690939906A0939A060F
:10C05000B0939B068091B4049091B504A091B6046E
:10C06000B091B70446015701881A990AAA0ABB0A77
:10C07000D501C401B7FD11C020E8C20E2EEED21EBC
:10C0800026E3E21EF11CC092B404D092B504E09203
:10C09000B604F092B7040E94C8530E9482390E94ED
:10C0A0004C4180911205882379F10E940EFD6B01AD
:10C0B0007C0180910E0590910F05A0911005B09123
:10C0C000110546015701881A990AAA0ABB0AD50127
:10C0D000C401B7FD19C02091120530E0A8EEB3E00D
:10C0E0000F94CD2BC60ED71EE81EF91EC0920E056A
:10C0F000D0920F05E0921005F092110580E00E94A9
:10C10000F2BA8AE00E940B3880910D05882359F11C
:10C110000E940EFD6B017C018091090590910A053A
:10C12000A0910B05B0910C05A7019601281B390BB6
:10C130004A0B5B0BDA01C901B7FD15C020910D0553
:10C1400030E0A8EEB3E00F94CD2BC60ED71EE81E4C
:10C15000F91EC0920905D0920A05E0920B05F092F3
:10C160000C050E94D3AA2B960FB6F894DEBF0FBE23
:10C17000CDBFDF91CF911F910F91FF90EF90DF9096
:10C18000CF90BF90AF909F908F907F906F905F9077
:10C190004F903F902F9008950E9427B3123008F0DF
:10C1A000CCCE0E94D93560E085EC96E050C083ED9E
:10C1B00096E09093870C8093860CBFCE843009F074
:10C1C000E2CE0E94174E8AED96E004C00E94174E00
:10C1D00089E097E00E944438D6CE0E94174E82EF45
:10C1E00096E0F8CF8091880790918907A0918A07FF
:10C1F000B0918B07A7019601281B390B4A0B5B0BEB
:10C20000DA01C901885E9340A109B109B7FD46C9A9
:10C210008DEC95E00E944438C0928807D09289073F
:10C22000E0928A07F0928B0739C9123098F48DE9B1
:10C2300096E00E9444388AE00E940B380E94AA2CA3
:10C2400090E080E00E943E5760E086EB96E00E941E
:10C25000B23F73CE123009F070CE0E9492B788239D
:10C2600079F081E00E9468B742EB50E062E178E04B
:10C2700086E394E10E9460B186E394E10E940DB3ED
:10C280000E94812F811193CF0E946B2F0E940EB8C4
:10C290000E9463B752CECF93DF9380918912909121
:10C2A0008A12891B8095877019F40E941F5AF5CF56
:10C2B000809189128F5F8770A09189129CE5A99F58
:10C2C000D0011124FD01EA5FF64FEF0119929A9512
:10C2D000E9F798E09083A55EB64F90E1EBE8F2E1D4
:10C2E00001900D929A95E1F72091891290918A120E
:10C2F000291303C094E69093861280938912DF91EC
:10C30000CF910C94992F9091891280918A12981351
:10C3100006C08091040990910509892B21F080E0E5
:10C320000E941F5AF0CF0895FC0120813181428183
:10C33000538160915E0C70915F0C8091600C9091C4
:10C34000610C0F949B250F94722E6093971270933B
:10C3500098128093991290939A12909189128091D9
:10C360008A1298130C944B610E9483610E94082AE0
:10C3700040919712509198126091991270919A126F
:10C3800040930C0650930D0660930E0670930F06B3
:10C3900081110C94992F08954F925F926F927F9222
:10C3A0008F929F92AF92BF92CF92DF92EF92FF92C5
:10C3B0000F931F93CF93DF93EC018B015A01F90187
:10C3C00020915E0C30915F0C4091600C5091610C9B
:10C3D00060817181828193810F949B250F94722ECD
:10C3E0006B017C0120915A0C30915B0C40915C0CEC
:10C3F00050915D0CF50160817181828193810F9470
:10C400009B250F94722E4B015C012091560C3091AC
:10C41000570C4091580C5091590CF8016081718172
:10C42000828193810F949B250F94722E2B013C01E6
:10C430002091520C3091530C4091540C5091550C5A
:10C44000688179818A819B810F949B250F94722E3C
:10C4500060938B1270938C1280938D1290938E1236
:10C4600040928F125092901260929112709292129A
:10C470008092931290929412A0929512B09296127A
:10C48000C0929712D0929812E0929912F0929A125A
:10C490009091891280918A12981791F0DF91CF9133
:10C4A0001F910F91FF90EF90DF90CF90BF90AF90D2
:10C4B0009F908F907F906F905F904F900C944B6106
:10C4C0000E9483610E94082A409193125091941215
:10C4D000609195127091961200918F1210919012A6
:10C4E0002091911230919212C0908B12D0908C12A8
:10C4F000E0908D12F0908E12C0920006D09201064C
:10C50000E0920206F09203060093040610930506DB
:10C5100020930606309307064093080650930906B9
:10C5200060930A0670930B064091971250919812EF
:10C530006091991270919A1240930C0650930D06D7
:10C5400060930E0670930F06882391F0DF91CF91D0
:10C550001F910F91FF90EF90DF90CF90BF90AF9021
:10C560009F908F907F906F905F904F900C94992F39
:10C57000DF91CF911F910F91FF90EF90DF90CF90BF
:10C58000BF90AF909F908F907F906F905F904F90F3
:10C5900008953F924F925F926F927F928F929F92F7
:10C5A000AF92BF92CF92DF92EF92FF920F931F93C1
:10C5B000CF93DF93CDB7DEB768970FB6F894DEBFA1
:10C5C0000FBECDBFD82E2A013B01480159013E2C98
:10C5D00020E030E0A901C501B8010F943525811193
:10C5E00010C081E08D1508F0B6C060E070E080E713
:10C5F00093E420E030E040E752E40F94FF2C4B013D
:10C600005C018D8A9E8AAF8AB88E0D2D10E0F801EC
:10C61000E256F64EE491BB24B3941E160CF4B12CF2
:10C62000CC24C39420E030E0A901C301B2010F94EF
:10C63000652E18160CF0C12CBC1471F092E0D912C2
:10C640000BC0332049F081E00E94DDF869E170E021
:10C6500080E090E00E94082680E00E949F2F69837E
:10C660007A838B839C8381E00E949F2F6D837E83DE
:10C670008F83988782E00E949F2F69877A878B87B4
:10C680009C8783E00E949F2F6D877E878F87988B82
:10C69000000F111F000F111FE1E0F0E0EC0FFD1F74
:10C6A0000E0F1F1FF80110821182128213829E0149
:10C6B000235F3F4FAE01475F5F4FBE016B5F7F4F10
:10C6C000CE0101960E94CC61F801408251826282C3
:10C6D0007382198A1A8A1B8A1C8A80910409909194
:10C6E0000509892B91F4CE0141967C018E010B5EE8
:10C6F0001F4F9E01235F3F4FAE01475F5F4FBE015B
:10C700006B5F7F4F40970E9487E70E948361BC1454
:10C7100051F092E0D91205C0332019F080E00E9458
:10C72000DDF80E94035668960FB6F894DEBF0FBE80
:10C73000CDBFDF91CF911F910F91FF90EF90DF90D0
:10C74000CF90BF90AF909F908F907F906F905F90B1
:10C750004F903F90089560E070E88BE395E449CFF7
:10C760004F925F926F927F928F929F92AF92BF9201
:10C77000CF92DF92EF92FF920F931F93CF93DF93AD
:10C78000CDB7DEB72C970FB6F894DEBF0FBECDBF86
:10C790002B013C0129873A874B875C874701580169
:10C7A000F601E080F1800281138120E030E0A901F0
:10C7B000B701C8010F943525882309F488C05E2D80
:10C7C0004F2D302F212F852F942FA32FB22F898308
:10C7D0009A83AB83BC8320E030E0A901B701C80194
:10C7E0000F943525811108C0E0903D02F0903E0283
:10C7F00000913F0210914002C701D8018D839E83B2
:10C80000AF83B887A50194016091300C7091310C11
:10C810008091320C9091330C0F94352587FF0CC01A
:10C820008092300C9092310CA092320CB092330C6A
:10C83000CE0101960E94E32A4092280C5092290CC6
:10C8400060922A0C70922B0C89859A85AB85BC85E9
:10C8500080932C0C90932D0CA0932E0CB0932F0C46
:10C86000CE0105960E94E32AA50194016091300C47
:10C870007091310C8091320C9091330C0F94652E95
:10C88000181664F48092300C9092310CA092320C05
:10C89000B092330CCE0101960E94E32A0E9483617C
:10C8A0002C960FB6F894DEBF0FBECDBFDF91CF91AF
:10C8B0001F910F91FF90EF90DF90CF90BF90AF90BE
:10C8C0009F908F907F906F905F904F90089550E071
:10C8D00040E030E820E477CFCF92DF92EF92FF92F2
:10C8E0000F931F936A01E090300CF090310C00918F
:10C8F000320C1091330CFB01208131814281538134
:10C90000FC0160817181828193810E94B0631F91DB
:10C910000F91FF90EF90DF90CF900895CF92DF922C
:10C92000EF92FF920F931F936B01FC01E080F18067
:10C9300002811381E8E2FCE0248135814681578140
:10C9400060817181828193810E94B0631F910F91F8
:10C95000FF90EF90DF90CF9008950F931F93CF93A8
:10C96000DF93EC018B0181E00E94DDF869E170E06A
:10C9700080E090E00E940826B801CE010E948E64FB
:10C98000C091E80680E00E94DDF81092E80682E09F
:10C990000E94C92F0E94FE2AC2FBCC27C0F981E069
:10C9A0008C27DF91CF911F910F910895AF92BF9285
:10C9B000CF92DF92EF92FF920F931F93CF93DF936B
:10C9C00000D01F92CDB7DEB7FC01E080F18002817C
:10C9D0001381611112C0A090300CB090310CC09046
:10C9E000320CD090330C9501A601B701C8010F9409
:10C9F000352587FF02C07501860120E030E048EC54
:10CA000053E4B701C8010F94352587FD04C0E12C1C
:10CA1000F12C08EC13E4C701D80189839A83AB8316
:10CA2000BC8362EE72E0CE0101960E948E640F908C
:10CA30000F900F900F90DF91CF911F910F91FF906A
:10CA4000EF90DF90CF90BF90AF9008953F924F92BC
:10CA50005F926F927F928F929F92AF92BF92CF928E
:10CA6000DF92EF92FF920F931F93CF93DF9300D04B
:10CA70001F92CDB7DEB7382E80E090E0A0E2B1E49F
:10CA800089839A83AB83BC83C0908012D09081123B
:10CA9000E0908212F090831220E030E0A901C701FB
:10CAA000B6010F94352587FF0CC0A701960160E001
:10CAB00070E080E291E40F94042C69837A838B8385
:10CAC0009C8360E0CE0101960E94D6644090280CC1
:10CAD0005090290C60902A0C70902B0C80902C0C9C
:10CAE00090902D0CA0902E0CB0902F0C332089F13B
:10CAF0000E94CE5419821A821B821C82E090300C54
:10CB0000F090310C0091320C1091330CCE01019653
:10CB10006C01A5019401C301B2010E94B06330927F
:10CB200084070E946D2B0F900F900F900F90DF9154
:10CB3000CF911F910F91FF90EF90DF90CF90BF901A
:10CB4000AF909F908F907F906F905F904F903F90AD
:10CB500008950E948B54CECF80918407882319F0CA
:10CB600080E00E94266580E008952F923F924F92C8
:10CB70005F926F927F928F929F92AF92BF92CF926D
:10CB8000DF92EF92FF920F931F93CF93DF93CDB776
:10CB9000DEB766970FB6F894DEBF0FBECDBFF82E96
:10CBA000282E312CF101E256F64ED49022E0821369
:10CBB00035C080918407811103C081E00E94266501
:10CBC0000E94CE54811139C18AE999E10E94851DE4
:10CBD00020E030E0A9010F9435258823F9F06D2D70
:10CBE000DD0C770B880B990B0F943C252B013C0136
:10CBF0008AE999E10E94851D4B015C0120E030E04B
:10CC000040EA50E40F94352511E087FF1CC0812CC9
:10CC1000912C90EAA92E90E4B92E15C06D2DDD0C53
:10CC2000770B880B990B0F943C252B013C01C1011C
:10CC3000880F991F880F991F8E56964E0E94851D4A
:10CC40004B015C0110E0A3019201C501B4010F94F6
:10CC50009B254B015C016101CC0CDD1CCC0CDD1C67
:10CC6000C6018A57964E0E94851DEE24E394E12664
:10CC700020E030E040EC5FE30F949B25A30192019C
:10CC80000F949B25AB01BC0100E010E098018F2DB3
:10CC90000E94C96220E030E0A901C501B4010F94EF
:10CCA0003525F601E658F64EFA8BE98B882309F410
:10CCB0004DC0F2E000E010E020E431E4FF1619F08E
:10CCC00000E010E09801B501A4017058E12C8F2D0F
:10CCD0000E94C962A5019401C501B4010F94052CFD
:10CCE0006B8B7C8B8D8B9E8B22E0F216E9F0F10131
:10CCF000E958F64E6491611107C00E94174E85E510
:10CD000099E10E9444386AE070E090E080E00F947E
:10CD10003A259B01AC0160E070E088E492E40F9456
:10CD2000FF2C8B019C0104C000E010E020EC30E4FB
:10CD3000EE24E3944B895C896D897E898F2D0E9456
:10CD4000C96232E0F312D0C00E948B5481E090E0BF
:10CD5000A0E0B0E00F2C04C0880F991FAA1FBB1FD2
:10CD60000A94D2F72091380C282B2093380C20916C
:10CD70009E05822B80939E0589899A890E94851D34
:10CD8000F601E85DF34F608371838283938382E0D1
:10CD9000F8121AC0209180123091811240918212B3
:10CDA000509183126091300C7091310C8091320C53
:10CDB0009091330C0F94042C6093300C7093310CD1
:10CDC0008093320C9093330CF601E650F84F1082AA
:10CDD0001182128213828F2D0E94A21C0E94FE2AB1
:10CDE000F601E85DF34F80819181A281B381F60164
:10CDF000EC58F84F80839183A283B38392E0F916B5
:10CE0000A9F18CE0EEEAF2E0DE01119601900D92BC
:10CE10008A95E1F7E1E0F0E0EC0FFD1FEC0DFD1D60
:10CE200080809180A280B38020E030E0A901C5011C
:10CE3000B4010F94352581111EC066960FB6F89483
:10CE4000DEBF0FBECDBFDF91CF911F910F91FF903D
:10CE5000EF90DF90CF90BF90AF909F908F907F909A
:10CE60006F905F904F903F902F9008950E94AC6517
:10CE70008111E3CFC6CF20E030E0A901C501B401A4
:10CE80000F94652E87FF04C0B7FAB094B7F8B0943A
:10CE9000F601E85DF34F6F01A3019201C501B401F2
:10CEA0000F949B259B01AC01F60160817181828109
:10CEB00093810F94042CF6016083718382839383A2
:10CEC000F2E080E090E0A0E4B1E4FF1621F080E021
:10CED00090E0A8E4B2E48D879E87AF87B88BCE013F
:10CEE0000D960E94E32AA9CF81E090E0A0E0B0E097
:10CEF0000F2C04C0880F991FAA1FBB1F0A94D2F7DA
:10CF00002091380C282B2093380C20919E05822BE1
:10CF100080939E0589899A890E94851DF601E85DA6
:10CF2000F34F60837183828393834ECFCF93DF93DC
:10CF300000D01F92CDB7DEB780E090E0A0EAB0E469
:10CF400089839A83AB83BC8361E0CE0101960E9402
:10CF5000D6640F900F900F900F90DF91CF910895AE
:10CF60008F929F92AF92BF92CF92DF92EF92FF92F9
:10CF70000F931F93CF93DF93CDB7DEB72C970FB6E8
:10CF8000F894DEBF0FBECDBF8B0140E050E068E4F7
:10CF900072E44D835E836F83788740E050E060EAFF
:10CFA00070E449875A876B877C878130B9F182307A
:10CFB00009F459C020E030E040E050E46091300CCA
:10CFC0007091310C8091320C9091330C0F94052CA0
:10CFD0004B017C0120E030E048EC53E40F94652ED7
:10CFE000181634F4812C912C88ECE82E93E4F92E59
:10CFF000F801A084B184C284D3849401A701B5014F
:10D00000C6010F94652E181614F054016701C5016E
:10D01000D60189839A83AB83BC8348C0BE01675F16
:10D020007F4FC80108960E948E64B8016C5F7F4FE5
:10D03000AE014B5F5F4FC8010E946C640E94993043
:10D040002C960FB6F894DEBF0FBECDBFDF91CF9107
:10D050001F910F91FF90EF90DF90CF90BF90AF9016
:10D060009F908F900895F8012085318542855385E2
:10D070006091300C7091310C8091320C9091330C96
:10D080000F94052C6B017C0120E030E048EC53E468
:10D090000F94352587FD06C0C12CD12C28ECE22E3B
:10D0A00023E4F22EC982DA82EB82FC82BE01675F42
:10D0B0007F4FCE010196B7CFEF92FF920F931F9350
:10D0C000CF93DF937C018B010E949331C8E2DCE0B7
:10D0D000209161023091620240916302509164029A
:10D0E000F70160817181828193810F94FF2C2C85DF
:10D0F0003D854E855F850F94052C6C877D878E87D7
:10D100009F87C8010E94E32ADF91CF911F910F9161
:10D11000FF90EF900C9483614F925F926F927F9299
:10D12000AF92BF92CF92DF92EF92FF920F931F9335
:10D13000CF93DF9300D000D01F921F92CDB7DEB700
:10D140005C0180E090E0A0E7B2E489839A83AB833E
:10D15000BC8380E090E0A0E8B0EC8D839E83AF8339
:10D16000B887BE016F5F7F4FCE0105960E945C6855
:10D1700068E873E180E090E00E940826C12CD12C81
:10D1800088ECE82E81E4F82EC982DA82EB82FC82F8
:10D1900080E090E0A0E8B0E48D839E83AF83B88701
:10D1A000BE016F5F7F4FCE0105960E945C680EE363
:10D1B0001CE0F80140AC51AC62AC73ACC0AED1AE77
:10D1C000E2AEF3AE80E090E0A0EAB1E489839A8316
:10D1D000AB83BC83F50180819181A281B3818D8372
:10D1E0009E83AF83B887BE016F5F7F4FCE010596E8
:10D1F0000E945C68F80140AE51AE62AE73AE129A06
:10D2000064E670E080E090E00E94082681E02896C5
:10D210000FB6F894DEBF0FBECDBFDF91CF911F9147
:10D220000F91FF90EF90DF90CF90BF90AF907F90E5
:10D230006F905F904F9008951F93CF93DF93CDB77A
:10D24000DEB72C970FB6F894DEBF0FBECDBF182FF8
:10D25000882379F020E030E0A9016091D605709133
:10D26000D7058091D8059091D9050F94352588234D
:10D27000F9F08091390C8117D9F00E9483618CE01C
:10D28000EAEBF2E0DE01119601900D928A95E1F74A
:10D29000CE0101960E94311F8091390C882391F0B4
:10D2A00088E29CE00E940A271092390C0E94FE2A14
:10D2B0002C960FB6F894DEBF0FBECDBFDF91CF9195
:10D2C0001F91089581E08093390C88E29CE00E94D0
:10D2D0001E21ECCF2F923F924F925F926F927F92DE
:10D2E0008F929F92AF92BF92CF92DF92EF92FF9276
:10D2F0000F931F93CF93DF93CDB7DEB7CB54D109F4
:10D300000FB6F894DEBF0FBECDBF2DB73EB739AF15
:10D3100028AF87E00E94274E81110BC061E086E5AF
:10D320000E9456248DA3853060F087E39EE00E9422
:10D330004438A8ADB9AD0FB6F894BEBF0FBEADBFAF
:10D3400040C33DA1332321F087E19EE00E94443891
:10D350006AE080E50E945624182F8CEF810F8F32EF
:10D3600018F083EF9DE0E3CF60E085E40E94722433
:10D37000882309F448C081E08FABE0908412F090DC
:10D380008512D7012D913D914D915C916091280CB2
:10D390007091290C80912A0C90912B0C0F94052CE4
:10D3A000AB01BC0188E50E94C42469877A878B871A
:10D3B0009C87F701248135814681578160912C0C2F
:10D3C00070912D0C80912E0C90912F0C0F94052CA8
:10D3D000AB01BC0189E50E94C4246D877E878F87DD
:10D3E000988BBE01635F7F4FCE0109960E94382E55
:10D3F000382E81110BC063E68FED9DE00E94B23F95
:10D4000087EC9DE094CF92E09FABB7CF8CE40E9475
:10D41000461E082F882309F431C10E9442248EA39E
:10D42000803118F080EA9DE082CFFEA1F13009F44E
:10D4300027C160E083E50E9472248AAF882321F02F
:10D44000011102C037E03EA38DA1833020F086E8B1
:10D450009DE00E9444389091390C9DAF80E00E947D
:10D460001C690E94DB1C1D8A1E8A1F8A188E198E59
:10D470001A8E1B8E1C8E83EF9FE4A3ECB7E48D8F76
:10D480009E8FAF8FB8A383EF9FE4A3ECB7EC89A383
:10D490009AA3ABA3BCA3A12FB0E0BCA7ABA7EDB7E9
:10D4A000FEB724E0129FE019F10911240FB6F89499
:10D4B000FEBF0FBEEDBF8DB79EB701969CAF8BAF81
:10D4C0002DA14FA9BE01635F7F4FCE0109960E9437
:10D4D0006CF99B01AC010F94F72E811162C20E947E
:10D4E0000EFD611571058105910511F00F94BB20AA
:10D4F000212C1BAA1CAA1DAA1EAAAEA1A150BB0BBF
:10D500002C96BFAFAEAF2C97E22DF0E0F8A7EFA3BB
:10D510002BA53CA5E217F3070CF074C23196FEA7C9
:10D52000EDA73F932F93FF93EF9382E79DE09F93A7
:10D530008F938CE79DE09F938F931F920E94FBF83F
:10D540008DB79EB709960FB6F8949EBF0FBE8DBFDC
:10D550009EA1992309F458C10F946C202AE030E071
:10D5600040E050E00F949B2B0F943C2520E030E0EE
:10D5700040EA50E40F94652E0FEF1FEF181614F0D9
:10D5800001E010E00F946C2028E631E040E050E02C
:10D590000F949B2B0F943C252B013C010F946C2086
:10D5A00020E230E040E050E00F949B2B6B5F7F4F18
:10D5B0008F4F9F4F0F943C254B015C01ADA1A430D0
:10D5C000D1F4BC01A40184E69DE00E942041B30196
:10D5D000A2018CE59DE00E94204186E59DE00E942D
:10D5E00044380130110519F483E40E940B3882E5B8
:10D5F0009DE00E944438312CC801110FAA0BBB0BCF
:10D600002A968CAF9DAFAEAFBFAF2A972C96AEAD2A
:10D61000BFAD2C973A161B060CF0F6C02A966CADDF
:10D620007DAD8EAD9FAD2A970F943C256B017C019B
:10D63000BAADBB2341F1AC019B010F94052C20E056
:10D6400030E040E952E40F949B259B01AC01C301FB
:10D65000B2010F94052C2B013C0120E030E044EB9B
:10D6600053E40F94652E1816FCF420E030E044EBF0
:10D6700053E4C301B2010F94042CEDCF1EA2D9CE06
:10D6800022E02EA3D6CE0F946C2024E130E040E0BF
:10D6900050E00F949B2B675E7F4F8F4F9F4F0F94EF
:10D6A0003C25A7019601CFCF20E030E0A901C301BE
:10D6B000B2010F94352587FF0BC020E030E044EB2A
:10D6C00053E4C301B2010F94052C2B013C01ECCFB4
:10D6D0000091841210918512F801248135814681D0
:10D6E00057816D857E858F8598890F94042C2296AD
:10D6F0006CAF7DAF8EAF9FAF22972BED3FE049E43B
:10D7000050E4C301B2010F949B2520E030E044E3D4
:10D7100053E40F94FF2C6B017C010F94FA2C6FA73C
:10D7200078AB89AB9AABD8012D913D914D915C912D
:10D7300069857A858B859C850F94042C26966CAF21
:10D740007DAF8EAF9FAF2697A50194016FA578A9F5
:10D7500089A99AA90F949B259B01AC0126966CADD3
:10D760007DAD8EAD9FAD26970F94052C69837A838E
:10D770008B839C83C701B6010F94A52EA50194014C
:10D780000F949B2522962CAD3DAD4EAD5FAD2297FB
:10D790000F94052C6D837E838F8398874BE351E034
:10D7A00070E060E0CE0101960E94CCC146E351E0FA
:10D7B00070E060E0CE0105960E94CCC1BDA1B430FE
:10D7C00099F449815A816B817C8186E49DE00E94B5
:10D7D00020414D815E816F81788580E69FE20E94C5
:10D7E00020418AE00E940B38198A1A8A1B8A1C8AF7
:10D7F000AE014F5E5F4FBE016B5F7F4FCE01019662
:10D800000E946C64339402CF20E04FA9BE01635F95
:10D810007F4FCE0109960E946CF94B015C01312CBF
:10D82000AC019B010F94F72E811102C03324339475
:10D83000A5019401C501B4010F94F72E8111E2C036
:10D84000EFA1F8A5EE0FFF1FEE0FFF1F2BAD3CADB4
:10D85000E20FF31F80829182A282B382A50194011C
:10D860006D8D7E8D8F8D98A10F94652E181624F4E2
:10D870008D8E9E8EAF8EB8A2A501940169A17AA16A
:10D880008BA19CA10F94352587FF04C089A29AA281
:10D89000ABA2BCA2A50194016BA97CA98DA99EA9EC
:10D8A0000F94052C6BAB7CAB8DAB9EABADA5BEA531
:10D8B000BD01BB0F880B990B0F943C256FA378A774
:10D8C00089A79AA79B01AC016BA97CA98DA99EA9E8
:10D8D0000F94FF2C2B013C014D8A5E8A6F8A788E53
:10D8E000EBADFCADF8ABEFA710E0C12CD12C76016D
:10D8F000AFA5B8A96D917D918D919D91B8ABAFA762
:10D90000A30192010F94042C9B01AC010F949B2561
:10D910009B01AC01C701B6010F94052C6B017C0182
:10D920001F5F211628F72FA138A549A55AA50F94E6
:10D93000FF2C0F94B32E698F7A8F8B8F9C8FBDA194
:10D94000B23068F18DA59EA50E942BE16BA57CA548
:10D9500081E49DE00E9442418BE39DE00E944438B7
:10D9600043E0C501B4010E944EBA80E20E940B3828
:10D9700081E0EDA1E3300CF480E0E12C8E010F5D3D
:10D980001F4F9E01235E3F4FAE01475E5F4FBE01BA
:10D990006B5E7F4F0E94013F8AE00E940B38239408
:10D9A000B3CD0E94AC650E94C21C8DAD0E941C6963
:10D9B0000E94993088AD99AD0FB6F8949EBF0FBE06
:10D9C0008DBFE8ADF9AD0FB6F894FEBF0FBEEDBF49
:10D9D000C55BDF4F0FB6F894DEBF0FBECDBFDF9142
:10D9E000CF911F910F91FF90EF90DF90CF90BF905C
:10D9F000AF909F908F907F906F905F904F903F90EF
:10DA00002F9008950E94AC65332069F280E39DE079
:10DA10000E94443881E0FDA11F160CF080E0EE2446
:10DA2000E3948E010F5D1F4F9E01235E3F4FAE01B9
:10DA3000475E5F4FBE016B5E7F4F0E94013F698D65
:10DA40007A8D8B8D9C8D0052110926E042E00F9457
:10DA500002209F938F938FE19DE09F938F9389E2A4
:10DA60009DE09F938F931F920E94FBF82DB73EB7C6
:10DA7000295F3F4F0FB6F8943EBF0FBE2DBF93CF27
:10DA80002F923F924F925F926F927F928F929F92CE
:10DA9000AF92BF92CF92DF92EF92FF920F931F93BC
:10DAA000CF93DF93CDB7DEB76A970FB6F894DEBF9A
:10DAB0000FBECDBF83E50E94461E182F3090390C53
:10DAC000882319F00E946224382E4090280C509030
:10DAD000290C60902A0C70902B0C80912C0C90914A
:10DAE0002D0CA0912E0CB0912F0C8B8B9C8BAD8BA1
:10DAF000BE8B8091300C9091310CA091320CB09182
:10DB0000330C8F8B988FA98FBA8F112329F0311086
:10DB100003C080E00E941C6986E50E94461E8A8B35
:10DB200020E030E0A9016091D6057091D705809181
:10DB3000D8059091D9050F943525882309F4C9C0DB
:10DB400083E40E94461E882309F49DC00E949A2403
:10DB50006B017C01A0E9B7E0B987A887BF83AE83DA
:10DB6000F5E0FD831D861E8628EC2F8702EC1A86C1
:10DB7000212C88EC8B8792E49C87AE81BF81B98B86
:10DB8000A88B15E0E889F98981909190A190B190D6
:10DB9000F98BE88B2A85322D4B855C85C501B40154
:10DBA0000F94352587FF04C08A86292CAB86BC8656
:10DBB0002D853E854F85502FC501B4010F94652EEC
:10DBC000181624F48D869E86AF860B2D1150D1F643
:10DBD000FD81F150FD838E819F8144969F838E83CA
:10DBE000F111CBCF2D853E854F85502F6A85722D43
:10DBF0008B859C850F94052C20E030E040E05FE3AE
:10DC00000F949B25A70196010F94052C4B015C01F5
:10DC10002DEB37E346E855EB0F94652E87FD0AC0E0
:10DC20002DEB37E346E855E3C501B4010F943525E4
:10DC300018164CF580E00E941C6910E0E884F98415
:10DC400000E0D7016D917D918D919D917D016D01D8
:10DC5000B4E0CB1AD108A50194010F94042CF6016D
:10DC60006083718382839383602F812F0E94D0F71A
:10DC70000F5F053031F71F5F888599854496998736
:10DC800088871530D9F6AA89AA2381F020E030E0F0
:10DC9000A9016091D6057091D7058091D805909122
:10DCA000D9050F94352581110E9489408AE50E948B
:10DCB000461E882351F00E949A2469837A838B83BD
:10DCC0009C83CE0101960E9498F6832D0E941C69C8
:10DCD0000BC0311003C09A89992341F30E94174E5B
:10DCE00080E69CE00E944438332051F08091390C4A
:10DCF000811106C00E94134E81E49CE00E944438CA
:10DD00000E94174E83E39CE00E9444388091390CB6
:10DD10000E9402410E94174E86E29CE00E94443815
:10DD2000C090CC08D090CD08E090CE08F090CF08FD
:10DD300020E030E0A901C701B6010F94652E181646
:10DD40000CF053C042E0C701B6010E944EBA8DE00C
:10DD50000E940B388AE00E940B38A3019201609167
:10DD6000280C7091290C80912A0C90912B0C0F9407
:10DD7000352581111FC02B893C894D895E896091B1
:10DD80002C0C70912D0C80912E0C90912F0C0F94D7
:10DD9000352581110FC02F89388D498D5A8D60919D
:10DDA000300C7091310C8091320C9091330C0F94A7
:10DDB000352581110E9499306A960FB6F894DEBF1E
:10DDC0000FBECDBFDF91CF911F910F91FF90EF90CC
:10DDD000DF90CF90BF90AF909F908F907F906F908B
:10DDE0005F904F903F902F90089581E29CE00E94B9
:10DDF0004438B3CF8F929F92AF92BF92EF92FF922F
:10DE00000F931F93CF93DF9380E00E941C691092C1
:10DE1000D2051092D3051092D4051092D505109218
:10DE2000CE051092CF051092D0051092D105109218
:10DE3000DA051092DB051092DC051092DD051092D8
:10DE4000D6051092D7051092D8051092D90500E991
:10DE500017E0C0E0812C912C80ECA82E8FE7B82E23
:10DE60007801D0E0F70181929192A192B1927F0165
:10DE70006D2F8C2F0E94D0F7DF5FD53099F7CF5FE1
:10DE80000C5E1F4FC53061F7DF91CF911F910F914D
:10DE9000FF90EF90BF90AF909F908F9008959091DA
:10DEA000891280918A12981308C080910409909178
:10DEB0000509892B11F40C94001F80E00E941F5A61
:10DEC000EECF83E50E94941E8823E9F00E940EFDA8
:10DED00060937611709377118093781190937911F4
:10DEE0000E949A2420E030E04AE754E40F949B25F6
:10DEF0000F94782D6093130270931402809315028F
:10DF00009093160208958091370584FD0AC0809190
:10DF1000390587FD06C080913A05837011F40C9491
:10DF20004F6F0E94836188E50E94461E882331F06E
:10DF30005F9A8091380C8E7F8093380C89E50E941F
:10DF4000461E882331F08A9A8091380C8D7F809309
:10DF5000380C8AE50E94461E882359F080910801FA
:10DF600080958170809306018091380C8B7F80931F
:10DF7000380C85E40E94461E81110C94FE1E089503
:10DF80002F923F924F925F926F927F928F929F92C9
:10DF9000AF92BF92CF92DF92EF92FF920F931F93B7
:10DFA000CF93DF93CDB7DEB7A6970FB6F894DEBF59
:10DFB0000FBECDBF84E797E00E942B2A8091E60B2D
:10DFC00083FD7EC02091340C3091350C4091360C8D
:10DFD0005091370C60918007709181078091820782
:10DFE000909183070F943525882309F469C0109117
:10DFF0000309111161C080915F0290916002019745
:10E000002091EB113091EC11281739073CF40E9454
:10E01000174E88E299E10E94443811E02091340CB7
:10E020003091350C4091360C5091370C609180073F
:10E030007091810780918207909183070F94042C3F
:10E040006B017C0120E030E0A9010F94652E87FF71
:10E0500004C0F7FAF094F7F8F0942091610230913F
:10E0600062024091630250916402C701B6010F94AD
:10E070009B2520E030E84BE354E40F94652E1816FE
:10E08000ECF40E94174E89E099E10E944438809197
:10E09000800790918107A0918207B09183078093B8
:10E0A000340C9093350CA093360CB093370C80E869
:10E0B00097E00E94946104C010E0B0CF1111E7CF47
:10E0C0002AE037ED43E25CE3609141027091420245
:10E0D00080914302909144020F949B256B017C0137
:10E0E0006091670270916802072E000C880B990BF3
:10E0F0000F943C259B01AC01C701B6010F949B25F1
:10E10000698B7A8B8B8B9C8B8091390C882309F1DE
:10E110008090CC089090CD08A090CE08B090CF0809
:10E12000C0907C07D0907D07E0907E07F0907F073D
:10E1300020E030E0A901C501B4010F943525882302
:10E14000D1F1A7019601C501B4010F94652E1816EF
:10E1500094F1C12CD12C76018E010F5E1F4F20E867
:10E1600037E04CE757E068E777E084E797E00E9404
:10E1700051F480E1E4E7F7E0A8E2BCE001900D9201
:10E180008A95E1F7A6960FB6F894DEBF0FBECDBF15
:10E19000DF91CF911F910F91FF90EF90DF90CF9083
:10E1A000BF90AF909F908F907F906F905F904F90B7
:10E1B0003F902F9008952091280C3091290C409188
:10E1C0002A0C50912B0C6091740770917507809107
:10E1D0007607909177070F94042C6D8B7E8B8F8B35
:10E1E000988F20912C0C30912D0C40912E0C509139
:10E1F0002F0C609178077091790780917A07909140
:10E200007B070F94042C698F7A8F8B8F9C8F2091C2
:10E21000300C3091310C4091320C5091330CC701CD
:10E22000B6010F94042C6D8F7E8F8F8F98A3209151
:10E23000340C3091350C4091360C5091370C609174
:10E2400080077091810780918207909183070F94D6
:10E25000042C6B017C0120E030E0A9016D897E89EE
:10E260008F89988D0F94352581110CC020E030E006
:10E27000A901698D7A8D8B8D9C8D0F94352588230E
:10E2800009F467CF2D893E894F89588DCA01B9019C
:10E290000F949B254B015C01298D3A8D4B8D5C8D34
:10E2A000CA01B9010F949B259B01AC01C501B401C2
:10E2B0000F94052C4B015C012D8D3E8D4F8D58A187
:10E2C000CA01B9010F949B259B01AC01C501B401A2
:10E2D0000F94052C4B015C01A7019601C701B60103
:10E2E0000F949B259B01AC01C501B4010F94052C33
:10E2F0000F94B32E4B015C012DEB37E346E855E359
:10E300000F94352587FF0FC020E030E0A901C70139
:10E31000B6010F94652E4601570187FF04C0B7FA76
:10E32000B094B7F8B0942DEB37E346E855E3C50158
:10E33000B4010F94352587FD1CCF20E030E040EA82
:10E3400051E4C501B4010F94FF2C0F94782D1B01EB
:10E35000672B19F422242394312CB10190E080E042
:10E360000F943A259B01AC0160E070E080E89FE3E8
:10E370000F94FF2C2B013C01AC019B01C501B401A2
:10E380000F949B254B015C01A30192016D897E894D
:10E390008F89988D0F949B256D8B7E8B8F8B988F9B
:10E3A000A3019201698D7A8D8B8D9C8D0F949B2595
:10E3B000698F7A8F8B8F9C8FA30192016D8D7E8DDB
:10E3C0008F8D98A10F949B256D8F7E8F8F8F98A333
:10E3D000A3019201C701B6010F949B2569A37AA3FB
:10E3E0008BA39CA380E1E8E2FCE08E010F5F1F4F4E
:10E3F000D80101900D928A95E1F70E940EFD2B0144
:10E400003C0128EC420E511C611C711C0DA31EA383
:10E4100081E0281A310809F460C00E940EFD8B01CA
:10E420009C01041915092609370937FD59C02B012C
:10E430003C0128EC420E511C611C711C80E00E94C2
:10E440001F5A2D893E894F89588D69817A818B8128
:10E450009C810F94052C69837A838B839C83298DFF
:10E460003A8D4B8D5C8D6D817E818F8198850F9467
:10E47000052C6D837E838F8398872D8D3E8D4F8DE8
:10E4800058A169857A858B859C850F94052C6987B1
:10E490007A878B879C8729A13AA14BA15CA16D85C6
:10E4A0007E858F8598890F94052C6D877E878F8751
:10E4B000988B750164018E010F5E1F4F9E01235FD3
:10E4C0003F4FAE01475F5F4FBE016B5F7F4F8DA136
:10E4D0009EA10E9451F481119BCF750164013CCE35
:10E4E0000E940EC2AECF8F929F92AF92BF92CF92F8
:10E4F000DF92EF92FF92CF93DF9380904102909052
:10E500004202A0904302B0904402FC01C080D1803E
:10E51000E280F38020E030E0A901C701B6010F944A
:10E520003525882341F0C0924102D0924202E09208
:10E530004302F0924402C0916702D091680284E6DF
:10E5400090E09093680280936702C0906102D0903F
:10E550006202E0906302F090640280E090E0A0E844
:10E56000BFE38093610290936202A0936302B09331
:10E5700064020E94C06F8092410290924202A09277
:10E580004302B0924402D0936802C0936702C092E3
:10E590006102D0926202E0926302F0926402DF9123
:10E5A000CF91FF90EF90DF90CF90BF90AF909F9072
:10E5B0008F9008950F931F93CF93DF9300D01F92F6
:10E5C000CDB7DEB79C0104E717E090E1E8E2FCE09C
:10E5D000D80101900D929A95E1F7F90120813181DE
:10E5E00042815381F80160857185828593850F94FE
:10E5F000052CF801608771878287938780E090E01F
:10E60000A0EAB0E489839A83AB83BC83CE010196F0
:10E610000E9473720F900F900F900F90DF91CF9127
:10E620001F910F9108952F923F924F925F926F9298
:10E630007F928F929F92AF92BF92CF92DF92EF9292
:10E64000FF921F93CF93DF93CDB7DEB72C970FB612
:10E65000F894DEBF0FBECDBF7A011901DC012D9108
:10E660003D914D915C912D833E834F835887FB01F3
:10E6700040805180628073808090280C9090290C9B
:10E68000A0902A0CB0902B0CA50194016D817E8185
:10E690008F8198850F94352581110EC011E0A3015B
:10E6A000920160912C0C70912D0C80912E0C909108
:10E6B0002F0C0F943525811110E0D1012D913D9142
:10E6C0004D915C9129873A874B875C87F701C08021
:10E6D000D180E280F38020910B0230910C024091B6
:10E6E0000D0250910E02C701B6010F943525882303
:10E6F00009F44EC0C0920B02D0920C02E0920D02BF
:10E70000F0920E028091340C9091350CA091360C51
:10E71000B091370C40912C0C50912D0C60912E0C27
:10E7200070912F0C8092740790927507A0927607D3
:10E73000B0927707409378075093790760937A07F0
:10E7400070937B07C0927C07D0927D07E0927E0792
:10E75000F0927F078093800790938107A0938207B0
:10E76000B093830720E030E040E05FE360916A0C03
:10E7700070916B0C80916C0C90916D0C0F949B259B
:10E7800069837A838B839C83CE0101960E94737286
:10E790002D813E814F8158852093740730937507F2
:10E7A0004093760750937707409278075092790705
:10E7B00060927A0770927B07D1012D913D914D9126
:10E7C0005C916091800770918107809182079091A0
:10E7D00083070F94052C60938007709381078093C3
:10E7E00082079093830711112FC020E030E0A90128
:10E7F00069857A858B859C850F943525811133C079
:10E8000060E070E088EC92E469837A838B839C8378
:10E81000CE0101960E9473722C960FB6F894DEBF5B
:10E820000FBECDBFDF91CF911F91FF90EF90DF9092
:10E83000CF90BF90AF909F908F907F906F905F90A0
:10E840004F903F902F9008952AEF3EE74AE25FE312
:10E8500060916E0C70916F0C8091700C9091710CA6
:10E860000F949B25D1CF60E070E080EA91E4CCCF9B
:10E870000F931F93CF93DF9300D000D01F921F926E
:10E88000CDB7DEB78B01FC0123A5211102C00E9488
:10E8900059FB1D821E821F82188620E030E040E076
:10E8A0005FE36091300C7091310C8091320C90914B
:10E8B000330C0F94052C69837A838B839C839E0190
:10E8C0002B5F3F4FAE014F5F5F4F6CE27CE088E211
:10E8D0009CE00E9413731D821E821F82188620E016
:10E8E00030E040E05FE3F8016085718582859385C3
:10E8F0000F94052C69837A838B839C83B8016C5FAA
:10E900007F4F9E012B5F3F4FAE014F5F5F4FC801AE
:10E910000E94137328960FB6F894DEBF0FBECDBFCA
:10E92000DF91CF911F910F9108959B01AC01485F3A
:10E930005F4FBC016C5F7F4F0C9413732F923F921B
:10E940004F925F926F927F928F929F92AF92BF92FF
:10E95000CF92DF92EF92FF920F931F93CF93DF93AB
:10E96000CDB7DEB7A6970FB6F894DEBF0FBECDBF0A
:10E970008C011B015A8749874090280C5090290C24
:10E9800060902A0C70902B0C80902C0C90902D0C89
:10E99000A0902E0CB0902F0CDB018D919D910D90CD
:10E9A000BC91A02D8B8B9C8BAD8BBE8B9C01AD0144
:10E9B000C301B2010F94042C6B017C01D1011496A8
:10E9C0008D919D910D90BC91A02D8F8B988FA98FCB
:10E9D000BA8F9C01AD01C501B4010F94042C6B8F5B
:10E9E0007C8F8D8F9E8FA985BA858D919D910D907D
:10E9F000BC91A02D8B879C87AD87BE879C01AD0104
:10EA0000C301B2010F94042C6F8F78A389A39AA33A
:10EA1000A985BA8514968D919D910D90BC91A02DDC
:10EA20008F87988BA98BBA8B9C01AD01C501B4016E
:10EA30000F94042C6BA37CA38DA39EA3A701960126
:10EA4000C701B6010F949B256B017C012B8D3C8D7A
:10EA50004D8D5E8DCA01B9010F949B259B01AC01C0
:10EA6000C701B6010F94052C4B015C012B893C8931
:10EA70004D895E896B857C858D859E850F94042CE0
:10EA80002B013C012F89388D498D5A8D6F857889EE
:10EA900089899A890F94042C6B017C01A30192014E
:10EAA000C301B2010F949B252B013C01A7019601E4
:10EAB000C701B6010F949B259B01AC01C301B201B4
:10EAC0000F94052C0F94B32E6B017C012F8D38A170
:10EAD00049A15AA1CA01B9010F949B252B013C0100
:10EAE0002BA13CA14DA15EA1CA01B9010F949B25A8
:10EAF0009B01AC01C301B2010F94052C9B01AC0139
:10EB0000C501B4010F94652E1816B4F520E030E06D
:10EB1000A901C701B6010F94652E87FF2AC0C7015E
:10EB2000B601905820E030E040EA50E40F94652EA2
:10EB3000181614F5A10169857A85C8010E949E7492
:10EB4000A6960FB6F894DEBF0FBECDBFDF91CF9172
:10EB50001F910F91FF90EF90DF90CF90BF90AF90FB
:10EB60009F908F907F906F905F904F903F902F90ED
:10EB70000895C701B601D6CF20E030E040E050E470
:10EB8000C501B4010F94652E181624F4B101C80113
:10EB90000E94387419821A821B821C82BE016F5F28
:10EBA0007F4FC1010E9495742DEC3CEC4CEC5CE372
:10EBB000C701B6010F949B259B01AC01F801608150
:10EBC0007181828193810F949B256D837E838F83D6
:10EBD0009887D8019B968C919B978823C9F02AE946
:10EBE00039E949E95FE314966D917D918D919C918E
:10EBF00017970F949B2569837A838B839C83BE012F
:10EC00006F5F7F4F84E797E00E949574F80113A629
:10EC1000BE016B5F7F4F89859A850E94957490CF66
:10EC20003F924F925F926F927F928F929F92AF929C
:10EC3000BF92CF92DF92EF92FF920F931F93CF93E9
:10EC4000DF93CDB7DEB76C970FB6F894DEBF0FBE7B
:10EC5000CDBFDB010C91142F100F153008F067C1E8
:10EC60001196DC90C22ECD0CB4E0BC1508F45FC147
:10EC7000ED2DF0E0E250FB4F8080912CB12CA12CC7
:10EC8000002E04C0B694A794979487940A94D2F760
:10EC900080FE4DC1EC2DF0E0E250FB4F8080912CC6
:10ECA000B12CA12C012E04C0B694A79497948794FC
:10ECB0000A94D2F780FE3BC1322E642F7C01409033
:10ECC000CE055090CF056090D0057090D105809111
:10ECD000D6059091D705A091D805B091D905898F17
:10ECE0009A8FAB8FBC8F660F770B072E000C880BAB
:10ECF000990B0F943C254B015C01602F000F770BA3
:10ED0000880B990B0F943C25298D3A8D4B8D5C8D8A
:10ED10000F949B25A30192010F94052CA50194014A
:10ED20000F94052C6D877E878F87988B612F110F2D
:10ED3000770B880B990B0F943C25298D3A8D4B8DC1
:10ED40005C8D0F949B25A30192010F94052CA501C6
:10ED500094010F94042C69837A838B839C83409065
:10ED6000D2055090D3056090D4057090D505809160
:10ED7000DA059091DB05A091DC05B091DD05898F66
:10ED80009A8FAB8FBC8F632D660F770B072E000C0D
:10ED9000880B990B0F943C254B015C016D2DDD0C0C
:10EDA000770B880B990B0F943C25298D3A8D4B8D51
:10EDB0005C8D0F949B25A30192010F94052CA50156
:10EDC00094010F94052C698B7A8B8B8B9C8B6C2D0B
:10EDD000CC0C770B880B990B0F943C25298D3A8D21
:10EDE0004B8D5C8D0F949B25A30192010F94052CF4
:10EDF000A50194010F94042C6D837E838F839887E3
:10EE0000F70180859185A285B38589879A87AB872D
:10EE1000BC878D8B9E8BAF8BB88F45E351E061E053
:10EE200070E0CE0141960E94CCC145E351E061E023
:10EE300070E0CE0105960E94CCC14AE351E061E04A
:10EE400070E0CE010D960E94CCC14AE351E061E032
:10EE500070E0CE0101960E94CCC189889A88AB8867
:10EE6000BC8827E137EB41ED58EBC501B4010F94A5
:10EE7000652E87FD5CC023E030E04BE953E4C5011B
:10EE8000B4010F94352518160CF451C08D849E845E
:10EE9000AF84B88827E137EB41ED58EBC501B401E9
:10EEA0000F94652E87FD43C023E030E84DE953E41D
:10EEB000C501B4010F9435251816CCF18D809E80C4
:10EEC000AF80B88427E137EB41ED58EBC501B401C1
:10EED0000F94652E87FD2BC023E030E04BE953E40F
:10EEE000C501B4010F94352518160CF189809A805C
:10EEF000AB80BC8027E137EB41ED58EBC501B40195
:10EF00000F94652E87FD13C023E030E84DE953E4EC
:10EF1000C501B4010F94352518164CF0AE014F5FB2
:10EF20005F4FBE01635F7F4FC7010E949E746C9666
:10EF30000FB6F894DEBF0FBECDBFDF91CF911F910A
:10EF40000F91FF90EF90DF90CF90BF90AF909F9088
:10EF50008F907F906F905F904F903F9008952F9289
:10EF60003F924F925F926F927F928F929F92AF9259
:10EF7000BF92CF92DF92EF92FF920F931F93CF93A6
:10EF8000DF93CDB7DEB7CC58D1090FB6F894DEBF0A
:10EF90000FBECDBF80E19CE00E94443887E00E9414
:10EFA000274E81116EC084E50E94941E882329F0AB
:10EFB0000E94872481110E943CBA80E090E0A0E882
:10EFC000BFE389839A83AB83BC838D839E83AF83A6
:10EFD000B8878DEC9CECACE4BEE389879A87AB875D
:10EFE000BC8780E090E0A0E2B1E48D879E87AF8788
:10EFF000B88B8CE390E09A8B898B8DEC90E09C8BA6
:10F000008B8B8DEC9CECACECBEE38D8B9E8BAF8B35
:10F01000B88F80E090E0A0EEBFE3898F9A8FAB8F2E
:10F02000BC8F1BA61CA64AE959E969E97EE38FE477
:10F030000E94C4246D8F7E8F8F8F98A360E083E43D
:10F040000E94722489A360E08BE40E9472248AA348
:10F0500082E40E94941E882381F10E9487240097F5
:10F0600061F19C01285231092536310520F16CE807
:10F0700070E082EE9BE00E9442418DED9BE00E9499
:10F080004438C457DF4F0FB6F894DEBF0FBECDBF74
:10F09000DF91CF911F910F91FF90EF90DF90CF9074
:10F0A000BF90AF909F908F907F906F905F904F90A8
:10F0B0003F902F9008959A8B898B8CE40E94941E28
:10F0C0008823E1F00E949A246B017C01C986DA86CC
:10F0D000EB86FC8620E030E0A9010F94652E87FDC9
:10F0E0000AC020E030E040E050E4C701B6010F94D0
:10F0F000352518161CF485EB9BE0C1CF81E50E94F5
:10F10000461E882331F18091070590910805892BCF
:10F11000E9F00E949A246B017C01CD82DE82EF82AD
:10F12000F8862DEC3CEC4CE45DE30F94652E87FDF6
:10F130000AC020E030E040E751E4C701B6010F9477
:10F140003525181634F484E89BE099CF89E59BE0D7
:10F1500096CF83E50E94941E8823E9F00E949A24AA
:10F160006B017C01CD8ADE8AEF8AF88E2DEC3CECB7
:10F170004CEC5DE30F94652E87FD0AC020E030E083
:10F1800040E050E4C701B6010F94352518161CF471
:10F1900082E39BE074CF80E50E94461E882341F104
:10F1A0008091070590910805892B19F48AEF9AE060
:10F1B00066CF8BA58F5F8BA70E949A246B017C0181
:10F1C000CD86DE86EF86F88A20E030E0A9010F9434
:10F1D000652E87FD0AC020E030E048EC51E4C7010D
:10F1E000B6010F94352518161CF482ED9AE047CF2E
:10F1F00086E40E94941E8823E9F00E949A246B0101
:10F200007C01C98EDA8EEB8EFC8E20E030E040E887
:10F210005FE30F94652E87FD0AC020E030E040E8F0
:10F2200050E4C701B6010F94352518161CF489EA7D
:10F230009AE025CFC98CDA8CEB8CFC8C8D889E886B
:10F24000AF88B88CA7019601C701B6010F949B2522
:10F250009B01AC0160E070E084E490E40F94FF2C2B
:10F2600029813A814B815C810F949B252B013C01C4
:10F27000A5019401C501B4010F949B25A701960136
:10F280000F949B252CEE31E548EB5DE30F94FF2CAA
:10F290009B01AC01C301B2010F949B2569837A8362
:10F2A0008B839C8388E40E94941E882379F00E94BB
:10F2B0008724009759F09C01255A310928383105D7
:10F2C00018F08BE79AE0DBCE9C8B8B8B85E50E9458
:10F2D000461E8823C9F00E940EFD61157105810547
:10F2E000910511F00F94BB208091070590910805BE
:10F2F000892B91F00E949A24609303057093040572
:10F30000809305059093060582E50E94461E8111B3
:10F3100008C087E49AE0B3CE60E070E088E492E44D
:10F32000EBCF8091070590910805892B61F00E9431
:10F330008724AD969FAF8EAFAD97181619064CF087
:10F3400083E19AE09CCE2AE130E0AD963FAF2EAF4C
:10F35000AD9789E50E94941E882381F10E949A242A
:10F360002091D4083091D5084091D6085091D70803
:10F370000F94042C6B017C0188E50E94941E882365
:10F3800031F10E949A242091D0083091D108409107
:10F39000D2085091D3080F94042C6BA37CA38DA3A7
:10F3A0009EA3CFA2D8A6E9A6FAA6CE0183960E9474
:10F3B000051E811115C089EE99E061CEC0902C0C1C
:10F3C000D0902D0CE0902E0CF0902F0CD5CF6091AA
:10F3D000280C7091290C80912A0C90912B0CDDCF78
:10F3E00084E40E94461E91E089270E941C6980E007
:10F3F00090E0A0EAB0E48DA79EA7AFA7B8AB60E00D
:10F40000CE018D960E94D6643091F907CD57DF4F1B
:10F410003883C358D0401092F9070E94FF1B88EC34
:10F4200099E00E94443889899A898A3191050CF0C3
:10F4300044C08B899C890E941C1F61E080E00E946F
:10F44000DCBC811142C06FEF8DED99E00E94B23FAC
:10F450008CA5811104C0CE0101960E9459FB80E069
:10F4600090E0A0EAB0E480937C0790937D07A0939E
:10F470007E07B0937F071DA61EA61FA618AABE0171
:10F48000635D7F4F84E797E00E949574CD57DF4F0F
:10F490005881C358D0405093F9070E94FF1B8AA19E
:10F4A0008111EFCD10928311109282110E9494BEAF
:10F4B00090E080E00E941C1FE4CD0E945A2281E06F
:10F4C0000E9465BB8111B5CFBECF1092340C109253
:10F4D000350C1092360C1092370C84E39CE00E949D
:10F4E00094618BA5882309F452C020E030E040E706
:10F4F00051E460916E0C70916F0C8091700C909142
:10F50000710C0F94FF2C6DA77EA78FA798AB80E19D
:10F51000E8E2FCE0A4E7B7E001900D928A95E1F7FC
:10F520002D853E854F8558896091800770918107B0
:10F5300080918207909183070F94052C6093800738
:10F54000709381078093820790938307CE018D96F5
:10F550000E9473722D853E854F8558896091800782
:10F560007091810780918207909183070F94042CFA
:10F57000609380077093810780938207909383073D
:10F580008CA5811104C0CE0101960E9459FBEEEFBB
:10F59000F4E085E0DF011D928A95E9F780E1E8E279
:10F5A000FCE0A4E7B7E001900D928A95E1F7898528
:10F5B0009A85AB85BC8580937C0790937D07A0934B
:10F5C0007E07B0937F071DA61EA61FA618AABE0120
:10F5D000635D7F4F84E797E00E949574BE01635E90
:10F5E0007F4F84E797E00E94957489A1882309F4EE
:10F5F0001CC42091280C3091290C40912A0C509168
:10F600002B0CE5962CAF3DAF4EAF5FAFE5978091E9
:10F610002C0C90912D0CA0912E0CB0912F0CE196FA
:10F620008CAF9DAFAEAFBFAFE197312C212C9FEFD8
:10F63000A4969FAFA497AFEFA896AFAFA897BFEFE0
:10F64000C158DF4FB883CF57D040EFE4C058DF4FE9
:10F65000E883C058D040F3ECCF57DF4FF883C15850
:10F66000D04027E4CE57DF4F2883C258D04081E0F6
:10F6700090E0A0E0B0E0022C04C0880F991FAA1F00
:10F68000BB1F0A94D2F7CC57DF4F88839983AA8394
:10F69000BB83C458D040AEEFB4E0E796BFAFAEAF87
:10F6A000E79710E000E09101032C000C440B550B90
:10F6B000C857DF4F288339834A835B83C858D040BB
:10F6C000C457DF4F2882CC58D040E796AEADBFADCF
:10F6D000E7978D91E796BFAFAEAFE79790E0B0E0C8
:10F6E000A0E0CC57DF4F288139814A815B81C45823
:10F6F000D04082239323A423B523892B8A2B8B2BE1
:10F7000009F024C1C857DF4F688179818A819B81C4
:10F71000C858D0400F943C252091D6053091D7058C
:10F720004091D8055091D9050F949B252091CE0585
:10F730003091CF054091D0055091D1050F94052C03
:10F74000EB966CAF7DAF8EAF9FAFEB97B801012EFC
:10F75000000C880B990B0F943C252091DA05309111
:10F76000DB054091DC055091DD050F949B25209130
:10F77000D2053091D3054091D4055091D5050F9411
:10F78000052C6B017C01EB962CAD3DAD4EAD5FAD14
:10F79000EB97E5966CAD7DAD8EAD9FADE5970F9483
:10F7A000042C2B013C01A7019601E1966CAD7DADC7
:10F7B0008EAD9FADE1970F94042C4B015C01A3012A
:10F7C0009201C301B2010F949B252B013C01A501BD
:10F7D0009401C501B4010F949B259B01AC01C301A9
:10F7E000B2010F94052C0F94B32E4B015C01EB96E4
:10F7F0002CAD3DAD4EAD5FADEB976BA17CA18DA166
:10F800009EA10F94042C2B013C01A70196016FA12E
:10F8100078A589A59AA50F94042C6B017C01A301FE
:10F820009201C301B2010F949B252B013C01A7015A
:10F830009601C701B6010F949B259B01AC01C30142
:10F84000B2010F94052C0F94B32E20E030E040E776
:10F8500051E40F94FF2CA50194010F94052C6B012A
:10F860007C018090030590900405A0900505B09060
:10F87000060520E030E040E85FE3C501B4010F94E5
:10F88000652E1816F4F4C501B4010F94712D4B01C7
:10F890005C0160E070E0CB01181419041A041B0429
:10F8A00034F40F946C20A50194010F949B2B0F94BA
:10F8B0003C259B01AC01B601C7010F94052C6B01DF
:10F8C0007C01C158DF4F2881CF57D040C058DF4F4F
:10F8D0003881C058D040CF57DF4F4881C158D04001
:10F8E000CE57DF4F5881C258D040B601C7010F94A0
:10F8F000352587FF2BC0A4960FAFA497C457DF4FC1
:10F900003881CC58D040A8963FAFA897EC96CFAEA0
:10F91000EC97ED96DFAEED97EE96EFAEEE97EF96A5
:10F92000FFAEEF97C158DF4FC882CF57D040C058C5
:10F93000DF4FD882C058D040CF57DF4FE882C15840
:10F94000D040CE57DF4FF882C258D0400F5F1F4FD4
:10F950000530110509F0B9CE4FEF241A340A55E0ED
:10F960002516310409F083CEA4968FADA497E82F15
:10F97000F0E0E250FB4F208181E090E0A0E0B0E0B9
:10F98000A8960FACA89704C0880F991FAA1FBB1F89
:10F990000A94D2F7822B8083A8969FADA8976A9687
:10F9A0009FAF6A97A496AFADA4976B96AFAF6B97D6
:10F9B000EC968FADEC97ED969FADED97EE96AFADD3
:10F9C000EE97EF96BFADEF976F968CAF9DAFAEAF52
:10F9D000BFAF6F97A896BFADA897BF3F09F409C204
:10F9E000A496EFADA497EF3F09F403C26B2FBB0FB2
:10F9F000770B880B990B0F943C252091D6053091FD
:10FA0000D7054091D8055091D9050F949B25209199
:10FA1000CE053091CF054091D0055091D1050F947E
:10FA2000052C162F072F382E292E862F902FA32D29
:10FA3000B22D65968CAF9DAFAEAFBFAF6597A49664
:10FA4000FFADA4976F2FFF0F770B880B990B0F94C7
:10FA50003C252091DA053091DB054091DC05509181
:10FA6000DD050F949B252091D2053091D30540915F
:10FA7000D4055091D5050F94052C6B017C01699636
:10FA8000CCAEDDAEEEAEFFAE6997CE018F5A9F4F82
:10FA90000E94051E882309F4B0C120E030E040EA4E
:10FAA00050E4612F702F832D922D0F94052C4B0164
:10FAB0005C01CB01D50121968CAF9DAFAEAFBFAF3E
:10FAC00021972596CCAEDDAEEEAEFFAE2597A8967B
:10FAD0002FADA8972111E3C1A4963FADA497311192
:10FAE000B3C120E030E040EA50E4C701B6010F9412
:10FAF000052C6B017C01A4964FADA497442309F417
:10FB0000C5C1A4968FADA49784300CF0BFC122ED7F
:10FB1000422E23E5522E2BE7622E21E4722E2196EF
:10FB20008CAC9DACAEACBFAC219725968CAD9DAD99
:10FB3000AEADBFAD2597A7968CAF9DAFAEAFBFAFB3
:10FB4000A7979C01AD0169966CAD7DAD8EAD9FAD63
:10FB500069970F94042CAB966CAF7DAF8EAF9FAFBF
:10FB6000AB97A501940165966CAD7DAD8EAD9FAD53
:10FB700065970F94042C2D966CAF7DAF8EAF9FAF21
:10FB80002D97AB962CAD3DAD4EAD5FADAB9761966D
:10FB90002CAF3DAF4EAF5FAF6197A501940160916F
:10FBA000280C7091290C80912A0C90912B0C0F94A9
:10FBB000042C4B015C01A7962CAD3DAD4EAD5FAD65
:10FBC000A79760912C0C70912D0C80912E0C909128
:10FBD0002F0C0F94042CA7966CAF7DAF8EAF9FAF08
:10FBE000A797812F902FA32DB22D8DA79EA7AFA7EA
:10FBF000B8ABC9AADAAAEBAAFCAAC984DA84EB8456
:10FC0000FC84CDAADEAAEFAAF8AE2DEC3CEC4CECBD
:10FC10005CE3C301B2010F949B2529813A814B819A
:10FC20005C810F949B252091340C3091350C4091D0
:10FC3000360C5091370C0F94052C69AF7AAF8BAF0F
:10FC40009CAFA5019401C501B4010F949B254B0104
:10FC50005C01A7962CAD3DAD4EAD5FADA797CA0137
:10FC6000B9010F949B259B01AC01C501B4010F9410
:10FC7000052C20E030E040E050E40F94652E18168B
:10FC8000ACF420E030E040E05FE3C701B6010F9440
:10FC9000052C29966CAF7DAF8EAF9FAF2997BE0123
:10FCA000635C7F4FCE0101960E94387489859A85E6
:10FCB000AB85BC8529968CAF9DAFAEAFBFAF299702
:10FCC000A3961CAE1DAE1EAE1FAEA397BE01615A19
:10FCD0007F4FCE01CD960E9495748CA58823C1F0EC
:10FCE0002AE939E949E95FE36D817E818F81988551
:10FCF0000F949B25A3966CAF7DAF8EAF9FAFA3975C
:10FD0000BE01615A7F4F84E797E00E9495741CA65C
:10FD1000E090660CF090670C0091680C1091690CF3
:10FD2000A090620CB090630CC090640CD090650CF5
:10FD30009501A601B701C8010F94652E181614F499
:10FD4000750186018090410290904202A09043028A
:10FD5000B09044022DEC3CEC4CEC5DE3B701C801E3
:10FD60000F949B256093410270934202809343025B
:10FD70009093440240E0BE01675B7F4FCE018D96B9
:10FD80000F946D1480E1E8E2FCE0A4E7B7E0019095
:10FD90000D928A95E1F78092410290924202A092E0
:10FDA0004302B092440220E04FEFBE01675A7F4FFA
:10FDB000CE0101960E94107620E041E0BE01675A14
:10FDC0007F4FCE0101960E9410762FEF40E0BE01DA
:10FDD000675A7F4FCE0101960E94107621E040E0E5
:10FDE000BE01675A7F4FCE0101960E9410760E9495
:10FDF00083618091A40C8093A50CAD964EAD5FAD50
:10FE0000AD9741505109AD965FAF4EAFAD97452BC1
:10FE100009F419CB6A968FAD6A9787FD14CB6B9660
:10FE20008FAD6B9787FFE1CB0ECB2BA13CA14DA1F2
:10FE30005EA1E5962CAF3DAF4EAF5FAFE5978FA1CA
:10FE400098A5A9A5BAA5EBCB812F902FA32DB22DF4
:10FE500021968CAF9DAFAEAFBFAF219720E030E0D1
:10FE600040EA50E4C701B6010F94042C25966CAF0C
:10FE70007DAF8EAF9FAF2597A4965FADA49754300A
:10FE80000CF42FCE182D092D3A2C2B2C92ED492E47
:10FE900093E5592E9BEF692E90E4792E40CEA896DB
:10FEA0009FADA89794300CF452C0A496AFADA49720
:10FEB000A4300CF120E030E040EA50E4612F702FD4
:10FEC000832D922D0F94042C21966CAF7DAF8EAFB5
:10FED0009FAF219720E030E040EA50E4C701B6012F
:10FEE0000F94042C6B017C01A496EFADA497E43031
:10FEF0000CF40DCECBCF812F902FA32DB22D2196B8
:10FF00008CAF9DAFAEAFBFAF219720E030E040EAAD
:10FF100050E4C701B6010F94052C25966CAF7DAF58
:10FF20008EAF9FAF2597A496BFADA497B111D2CF46
:10FF300020E030E040EA50E4612F702F832D922DB5
:10FF40000F94042C162F072F382E292E9FCFA496FE
:10FF5000FFADA497F1110DC020E030E040E251E484
:10FF6000B401C5010F94042C162F072F382E292E0B
:10FF7000CECDA4962FADA49724309CF020E030E0A5
:10FF800040E251E4B401C5010F94042C21966CAFFA
:10FF90007DAF8EAF9FAF2197182D092D3A2C2B2CBA
:10FFA000B6CD182D092D3A2C2B2C82ED482E83E549
:10FFB000582E8BEF682E81E4782EB1CD2F923F9290
:10FFC0004F925F926F927F928F929F92AF92BF9269
:10FFD000CF92DF92EF92FF920F931F93CF93DF9315
:10FFE000CDB7DEB7EE970FB6F894DEBF0FBECDBF2C
:10FFF0008091390C888B87E50E94461E882309F47E
:020000021000EC
:1000000023C120E030E0A9016091D6057091D705A9
:100010008091D8059091D9050F943525811108C09C
:100020000E94134E8DE09DE00E94443810E01FC1F5
:100030008AE50E94941E882339F10E949A24209117
:10004000D8083091D9084091DA085091DB080F9414
:10005000042C6B017C0120E030E040E251ECC70150
:10006000B6010F94652E87FD0AC020E030E040E223
:1000700051E4C701B6010F943525181674F40E9497
:10008000134E80E09DE0D0CFC090300CD090310C6A
:10009000E090320CF090330CDECF40E050E060ECAA
:1000A0007FE788E50E94C4242091D0083091D108D0
:1000B0004091D2085091D3080F94042C2B013C019D
:1000C00040E050E060EC7FE789E50E94C424209185
:1000D000D4083091D5084091D6085091D7080F9494
:1000E000042C4B015C016FEF89E40E945624182F09
:1000F0006FEF8AE40E945624082FA3019201C301E6
:10010000B2010F94F72E81116EC0A5019401C501B3
:10011000B4010F94F72E811166C08BA19CA1ADA1F3
:10012000BEA18BAB9CABADABBEAB2091CE053091ED
:10013000CF054091D0055091D105C301B2010F9474
:10014000042C2B013C0120E030E040E05FE36BA990
:100150007CA98DA99EA90F949B259B01AC01C3018D
:10016000B2010F94052C2BA93CA94DA95EA90F94AF
:10017000FF2C0F94712D162F4FA058A469A47AA4B8
:100180002091D2053091D3054091D4055091D505E9
:10019000C501B4010F94042C4B015C0120E030E058
:1001A00040E05FE3C301B2010F949B259B01AC01CA
:1001B000C501B4010F94052CA30192010F94FF2CEB
:1001C0000F94712D062F812F012E000C990B97FD96
:1001D00033C005979CF5802F002E000C990B97FDDE
:1001E0002FC005977CF5153008F020CF053008F0BA
:1001F0001DCF80E00E941C6995E01902F0011124D6
:10020000E00FF11D07FDFA95EE0FFF1FEE0FFF1F28
:10021000E057F84FC082D182E282F382602F812FB3
:100220000E94D0F788890E941C698889882309F474
:10023000FDCE0E949930FACE10E0CDCF14E0CBCFA6
:1002400000E0D1CF04E0CFCF8AE40E94461E182FF1
:10025000811127C070E060E086E50E948B249A83BC
:100260008983059708F18BED9CE00E944438812F2B
:10027000EE960FB6F894DEBF0FBECDBFDF91CF91E3
:100280001F910F91FF90EF90DF90CF90BF90AF90B4
:100290009F908F907F906F905F904F903F902F90A6
:1002A00008950E94FA6EC2CE60E084E40E94722437
:1002B0008F8740E050E0BA018AE50E94C4246BA712
:1002C0007CA78DA79EA740E050E86BE376E483E52A
:1002D0000E94C42420E030E040E752E40F94FF2C59
:1002E00060933D0270933E0280933F0290934002E0
:1002F000E0908412F0908512D7018D909D90AD9082
:10030000BC9020E030E0A901C501B4010F94052C98
:100310006BAF7CAF8DAF9EAF20E030E040E450E4A7
:100320000F94352587FF06C01BAE1CAEB0E4BDAFF1
:10033000E0E4EEAF20E030E84DE953E4C501B4015C
:100340000F94052C662E7BAB8FAB98AF20E030E886
:1003500044E953E40F94652E18163CF4612CF0E840
:10036000FBAB24E92FAB33E438AFD70114968D9063
:100370009D90AD90BC90179720E030E0A901C50199
:10038000B4010F94052CD62EE72EF82E092F20E06D
:1003900030E040E551E40F94352587FF05C0D12CAE
:1003A000E12CA0E5FA2E01E420E030E04BE953E433
:1003B000C501B4010F94052CB62EC72E89AF9AAF94
:1003C00020E030E84FE853E40F94652E18163CF413
:1003D000B12CF0E8CF2EBFE8B9AFE3E4EAAF88E490
:1003E0000E94461E882309F416C20E949A240F9484
:1003F000712D1B0177FF02C06F5F7F4F7595679569
:100400007195619571096A567F4F072E000C880B14
:10041000990B0F943C25762E872E982EA92E2D2DE4
:100420003E2D4F2D502F0F94652E18161CF4D72CEF
:1004300074010A2D2BAD3CAD4DAD5EAD672D782D11
:10044000892D9A2D0F94652E181624F07BAC8CAC58
:100450009DACAEAC872D982DA92DBA2D8B8B9C8B86
:10046000AD8BBE8B8D2D9E2DAF2DB02F8F8B988F8A
:10047000A98FBA8FB101330C880B990B0F943C25CF
:100480001B012C01AC019B016D2D7E2D8F2D902F1A
:100490000F94052CD62EE72EF82E092F2B2D3C2D50
:1004A00049AD5AAD0F94352587FF04C0BD2CCE2C25
:1004B000F9AE0AAFA2019101672D782D892D9A2DF1
:1004C0000F94052CD62EE72EF82E092F262D3BA9AA
:1004D0004FA958AD0F94352587FF04C06D2CEBAAAA
:1004E000FFAA08AF862D9BA9AFA9B8AD8B8F9C8FB3
:1004F000AD8FBE8F8B2D9C2DA9ADBAAD8F8F98A3DC
:10050000A9A3BAA3BE01695E7F4FCE0143960E94A4
:10051000382E882309F4B0C1BE01615E7F4FCE0141
:100520004B960E94382EE82E882309F4A5C12F8906
:10053000388D498D5A8D6F8D78A189A19AA10F941C
:10054000042C20E030E040E85EE30F949B254B0153
:100550005C012B893C894D895E896B8D7C8D8D8DED
:100560009E8D0F94042C20E030E040E85EE30F9471
:100570009B256BA37CA38DA39EA38FA298A6A9A65F
:10058000BAA689819A811816190674F489EA9CE042
:100590000E9444388F85882321F08FE99CE00E94D7
:1005A00044388AE00E940B380E9483610E94DB1C61
:1005B00080E00E941C6980E090E0A0E2B1E48FA797
:1005C00098ABA9ABBAAB60E0CE018F960E94D6641F
:1005D0002091D6053091D7054091D8055091D90585
:1005E0006BA17CA18DA19EA10F943525811130C0F6
:1005F0002091DA053091DB054091DC055091DD0555
:100600006FA178A589A59AA50F943525811120C0E1
:100610002091CE053091CF054091D0055091D10564
:100620006B897C898D899E890F943525811110C035
:100630002091D2053091D3054091D4055091D50534
:100640006F89788D898D9A8D0F9435258823A9F02F
:100650000E94FA6E88E0FE01B396A6EDB5E0019027
:100660000D928A95E1F788E0FE017396AEECB5E055
:1006700001900D928A95E1F7188A60E085E40E9466
:100680007224882309F4FBC0F1E0FBAB1B861C86B7
:100690001D861E861A8A9E2C4FE6C42E4CE0D42E50
:1006A0005DE7A52E5CE0B52E1A8915300CF0F7C079
:1006B0006B857C858D859E859B01AC010F94F72E03
:1006C0008111EDC0992009F4DDC031E03FAB35E088
:1006D000232E91E09926F12EFF0CFF0CF10EF394DE
:1006E000898B19896A89121509F4D5C0062E000C68
:1006F000770B880B990B0F943C252FA138A549A5A2
:100700005AA50F949B252F89388D498D5A8D0F94AA
:10071000052C2B013C01612F110F770B880B990BD6
:100720000F943C252BA13CA14DA15EA10F949B25CC
:100730002B893C894D895E890F94052C6B837C83C2
:100740008D839E834F82588669867A8689819A81B5
:10075000892B79F06F2D8BE89CE00E94184169E1AC
:1007600070E089E89CE00E94424186E89CE00E949B
:1007700044381F9299E19F931F92FF92DF92CF928C
:10078000BF92AF921F920E94FBF829814BA9BE0134
:10079000695F7F4FCE0103960E946CF92B013C01EB
:1007A0004B865C866D867E860FB6F894DEBF0FBEE4
:1007B000CDBFAC019B010F94F72E811169C08988D0
:1007C0003A8825E0382D320380011124030D111DD4
:1007D00037FC1A95000F111F000F111F0057184FFB
:1007E000A30192016BA57CA58DA59EA50F94052C58
:1007F000D8016D937D938D939C931397632D882DD2
:100800000E94D0F7188A81E00E941F5AF3948989C8
:10081000BFA98B0F65CF4D2D5E2D6F2D702F86E4F8
:100820000E94C4241B012C014BAD5CAD6DAD7EADAF
:100830008CE40E94C4246B8B7C8B8D8B9E8B2F8AC7
:10084000388E498E5A8E4B2D5C2D69AD7AAD82E47F
:100850000E94C4246B017C01462D5BA96FA978AD71
:1008600082E50E94C4246B8F7C8F8D8F9E8FCF8EEC
:10087000D8A2E9A2FAA246CE8FEB9CE0F6CC22E009
:100880002BAB04CF8FEF8FAB22242A9484E021CFAF
:1008900088890E941C698A898F5F8A8B05CF0E9494
:1008A00066E40E94AC65882359F088890E941C691F
:1008B00080E090E0A0ECBFE78B879C87AD87BE8788
:1008C0006B857C858D859E859B01AC010F94F72EF1
:1008D000811159C08F85811126C082E0F82E02E077
:1008E00094E0C92E12E0DC2CD11A21E041E0612F06
:1008F000802F0E94732221E04FEF612F8F2D0E94E5
:1009000073222FEF41E06D2D802F0E9473222FEF75
:100910004FEF6D2D8F2D0E947322115020F7015043
:10092000F3940F3FF9F60E9489400E94A11E8F8523
:10093000811124C080E39CE00E948B1D4B015C016F
:1009400088E29CE00E94311F9B01AC01C501B4010B
:100950000F949B259B01AC016091300C7091310C80
:100960008091320C9091330C0F94042C6093300CD6
:100970007093310C8093320C9093330C8F858111DE
:10098000E888E092390C0E94C21C8091390C8111D8
:100990000E94FE2A0E9496670E9499306B857C8592
:1009A0008D859E8511E09B01AC010F94F72E81117E
:1009B0005ECC3CCB8F929F92AF92BF92CF92DF9250
:1009C000EF92FF920F931F93CF93DF9300D01F926C
:1009D000CDB7DEB75C016B017A01122F0023E1F184
:1009E0000E94174E88E999E00E94443861E0812F07
:1009F0000E94383A9090180583E08093180581E0B2
:100A00008093270C0E942F4082E08093911140E355
:100A100068E879E084E799E00E94344040E069E1C9
:100A200071E18DE699E00E94344061E088E699E04A
:100A30000E9416408AE799E00E942F228091270C9D
:100A4000882341F060E0812F0E94383A81E00E94C3
:100A50001F5AF4CF9092180520E030E0A901F5016B
:100A600060817181828193810F943525882371F093
:100A700080E090E0A0ECB0E489839A83AB83BC83F0
:100A8000BE016F5F7F4FC5010E945C6820E030E0CF
:100A9000A901F60160817181828193810F943525CE
:100AA000882351F18090760C9090770CA090780C70
:100AB000B090790C80E090E0A0E7B1E48093760CF0
:100AC0009093770CA093780CB093790C80E090E031
:100AD000A0EAB1E489839A83AB83BC83BE016F5FD4
:100AE0007F4FC6010E945C688092760C9092770CD2
:100AF000A092780CB092790C20E030E0A901F701C7
:100B000060817181828193810F94652E181674F42F
:100B100080E090E0A0E4B0E489839A83AB83BC8357
:100B2000BE016F5F7F4FC7010E945C688091ED043A
:100B300029E131E1882311F029E439E047E559E062
:100B400061E679E081E00E9457400E942F4081E0F9
:100B50000F900F900F900F90DF91CF911F910F91F9
:100B6000FF90EF90DF90CF90BF90AF909F908F90CD
:100B70000895CF93C82F8091E60B83FD14C0809118
:100B80000309811110C080915F02909160029C0165
:100B9000215031094091ED115091EE114217530748
:100BA00014F40E941C1FCC2329F061E080E0CF9157
:100BB0000C94DCBC8091030991E0892780933C026E
:100BC00080913C02882389F08091EB119091EC1187
:100BD0002091ED113091EE11821B930B97FF03C012
:100BE000919581959109029744F410923C0280916D
:100BF000E60B83FF06C0C1E01AC080E00E941F5AC6
:100C0000DFCFC0910309C11112C080915F029091A2
:100C1000600201972091ED113091EE1128173907EC
:100C200054F70E94174E8BE299E00E9444388C2FB3
:100C3000CF910895AF92BF92CF92DF92EF92FF9241
:100C40000F931F93CF93DF93CDB7DEB764970FB6A3
:100C5000F894DEBF0FBECDBF0E94164F87FDAFC018
:100C60008AE50E94941E882309F4BAC040E050E04F
:100C7000BA018AE50E94C4247B018C012091300CCA
:100C80003091310C4091320C5091330C60E070E0A7
:100C900088EC93E40F94042C5B016C019701A8018C
:100CA0000F94652E181614F07501860120E030E0CF
:100CB000A901B701C8010F94652E181624F4E12C80
:100CC000F12C00E010E0B701C8010F94712D072E40
:100CD000000C880B990B0F943C25698B7A8B8B8BBE
:100CE0009C8B20E030E0A9010F943525882321F06A
:100CF000CE0141960E94DA7280E090E0A0EAB1E471
:100D00008D879E87AF87B88B19861A861B861C86AF
:100D10008CE40E94461E882309F467C00E949A242E
:100D20006B017C0120E030E0A901C701B6010F94FE
:100D3000652E87FF04C0F7FAF094F7F8F094CD829F
:100D4000DE82EF82F8862091ED113091EE11243091
:100D5000310574F08091EB119091EC11821B930B93
:100D600097FF03C091958195910901E004970CF4D8
:100D700000E080E00E94B985882359F022E0AE01AE
:100D8000435F5F4FBE016B5F7F4FCE0109960E94AC
:100D9000DA8469897A898B899C898B019C01305816
:100DA00009831A832B833C8320E030E0A9010F9450
:100DB0003525882321F0CE0101960E94DA726496CF
:100DC0000FB6F894DEBF0FBECDBFDF91CF911F915C
:100DD0000F91FF90EF90DF90CF90BF90AF9008956C
:100DE000E12CF12C00E211E449CFC090C905D0906C
:100DF000CA05E090CB05F090CC0594CF7F928F92FE
:100E00009F92AF92BF92CF92DF92EF92FF920F9399
:100E10001F93CF93DF9300D000D01F921F92CDB7C6
:100E2000DEB76C015B014A01722E78010091160653
:100E30000E94281F8091ED119091EE118E159F0553
:100E40001CF4C7010E941C1F80E00E94B985882302
:100E500031F0272DA401B501C6010E94DA841E14C9
:100E60001F043CF4C7010E941C1F60E080E00E9448
:100E7000DCBC81E00E94B98580E090E0A0E7B2E4AC
:100E800089839A83AB83BC8380E090E0A0E8B0ECD8
:100E90008D839E83AF83B887BE016F5F7F4FCE0186
:100EA00005960E945C6887E00E94152A811158C04F
:100EB0008091300C9091310CA091320CB091330C98
:100EC0004091F2045091F3046091F4047091F504A0
:100ED000C090EE04D090EF04E090F004F090F104A4
:100EE000C0927407D0927507E0927607F092770768
:100EF000409378075093790760937A0770937B0744
:100F000080937C0790937D07A0937E07B0937F0723
:100F100080E090E0A8E4B2E489839A83AB83BC8349
:100F2000CE0101960E9473728091F6049091F704AD
:100F3000A091F804B091F90480937C0790937D0709
:100F4000A0937E07B0937F0780E090E0A0EAB0E432
:100F500089839A83AB83BC83CE0101960E9473720E
:100F6000C12CD12C80E7E82E82E4F82EC982DA82E7
:100F7000EB82FC8280E090E0A0E8B0E48D839E8369
:100F8000AF83B887BE016F5F7F4FCE0105960E9489
:100F90005C6820E030E0A9016091FA047091FB04E4
:100FA0008091FC049091FD040F94352587FF0BC0C0
:100FB000C982DA82EB82FC82BE016F5F7F4F8AEFCB
:100FC00094E00E945C688091FA049091FB04A091E7
:100FD000FC04B091FD048093340C9093350CA093E5
:100FE000360CB093370C8093800790938107A093C1
:100FF0008207B093830780E897E00E949461809114
:10100000CD0581110E9416F761E087EB99E00E94FF
:101010007F3F809123118150809323114EE658E148
:101020006FEB79E085E00E94EBE280912311882349
:1010300039F00E9415AB80912311815080932311C8
:1010400080E00E94DDF80E9493318091241182306B
:1010500011F40E9452380E9466E428960FB6F89464
:10106000DEBF0FBECDBFDF91CF911F910F91FF90DB
:10107000EF90DF90CF90BF90AF909F908F907F9038
:101080000895CF92DF92EF92FF920F931F93CF9329
:10109000DF9300D01F92CDB7DEB77C016B018A01D0
:1010A00061E08CE399E00E947F3F4EE658E163E403
:1010B00079E085E00E94EBE29091231181E0890FB5
:1010C000809323118091311482FF06C08B7F80931F
:1010D00031149E5F909323110E94443980E1E8E22D
:1010E000FCE0AEEEB4E001900D928A95E1F70E942B
:1010F000836181E00E94DDF820E030E0A901F70182
:1011000060817181828193810F9435258823F1F06C
:101110008091030981110CC080915F02909160025F
:1011200001972091EB113091EC112817390774F0D9
:1011300080E090E0A0E7B2E489839A83AB83BC832C
:10114000BE016F5F7F4FC7010E945C6887E00E940D
:10115000152A811103C0B6010E94B06720E030E07B
:10116000A901F80160817181828193810F943525F5
:10117000882341F080E00E94B985882319F0C801D6
:101180000E948C68129A64E670E080E090E00E9411
:10119000082681E00F900F900F900F90DF91CF9174
:1011A0001F910F91FF90EF90DF90CF900895CF9215
:1011B000DF92EF92FF92CF93DF936B017C01D42FEC
:1011C000C091180583E08093180581E08093270C77
:1011D000C114D104E104F10431F00E940EFDC60EE9
:1011E000D71EE81EF91E8091270C882389F0C114B0
:1011F000D104E104F10421F48D2F0E941F5AF3CF92
:101200000E940EFD6C197D098E099F0997FDF4CF90
:101210001092270CC0931805DF91CF91FF90EF90AB
:10122000DF90CF9008950F931F93CF93DF93C82F34
:10123000162F0E94174EC11194C0CFE8D8E0CE01FE
:101240000E94443861E0812F0E94383A0E940EFDCE
:10125000685370458F4F9F4F60931206709313062B
:1012600080931406909315061092160600911805A7
:1012700083E08093180530E020E049E151E16DE121
:1012800079E082E00E9457408DE199E00E942F2290
:1012900081E08093270C8091270C882309F464C097
:1012A00060E0812F0E94383A80911606882309F465
:1012B00054C00E94174E83E099E00E94443830E009
:1012C00020E04DEE58E064EF78E082E00E94574065
:1012D00084EF98E00E942F2241E060E070E0CB01B3
:1012E0000E94D78830E020E050E040E060EE78E0F7
:1012F00085E00E94574080EE98E00E949A350E9457
:10130000281F80E00E94B9850E94174ECE010E94DE
:1013100044380E940EFD685370458F4F9F4F609375
:10132000120670931306809314069093150610927C
:10133000160630E020E049E151E164ED78E082E01A
:101340000E94574083EC98E00E942F2281E0809316
:10135000270C61E0812F0E94383A81E00E941F5AD9
:101360009ACFC4EAD8E06BCF00931805DF91CF91F4
:101370001F910F910895CF92DF92EF92FF920F93FA
:101380001F93CF93DF93CDB7DEB7A0970FB6F89436
:10139000DEBF0FBECDBF0E94164F87FDCCC085E4D7
:1013A0000E94461E882309F4D5C00E949A246B012E
:1013B0007C0120E030E0A9010F94652E87FF04C076
:1013C000F7FAF094F7F8F094F7FAF094F7F8F0944D
:1013D000CD8EDE8EEF8EF8A28CE0E6ECF2E0DE0140
:1013E000119601900D928A95E1F78AE50E94941E6C
:1013F000882351F040E050E0BA018AE50E94C424FD
:1014000069877A878B879C8788E50E94941E88234A
:1014100051F040E050E0BA0188E50E94C42469839D
:101420007A838B839C8389E50E94941E882351F0E4
:1014300040E050E0BA0189E50E94C4246D837E83B8
:101440008F83988785E50E94461E882309F489C00A
:101450000E949A246B017C0120E030E0A901C701C1
:10146000B6010F94652E87FF04C0F7FAF094F7F8E1
:10147000F094F7FAF094F7F8F094C98EDA8EEB8EC8
:10148000FC8E1D8A1E8A1F8A188E8CE40E94461EBE
:10149000882309F46FC00E949A246B017C0120E02C
:1014A00030E0A901C701B6010F94652E87FF04C083
:1014B000F7FAF094F7F8F094C98ADA8AEB8AFC8A92
:1014C00062E070E082E40E948B24F82E8091231168
:1014D000811131C021E0AE01475E5F4FBE016F5FF9
:1014E0007F4FCE014D960E944188882321F16F2DB8
:1014F00081E00E94138982E50E94941E882309F4EA
:1015000042C00E94872440E050E060EA71E44D87C9
:101510005E876F87788B20912311222361F08C01E5
:101520002F2DAE01435F5F4FBE016F5E7F4FCE0137
:1015300045960E94FE86A0960FB6F894DEBF0FBEB9
:10154000CDBFDF91CF911F910F91FF90EF90DF9072
:10155000CF900895C12CD12C80E8E82E80E4F82E9D
:1015600033CFC090C505D090C605E090C705F09078
:10157000C80572CFC090C905D090CA05E090CB05D0
:10158000F090CC058CCF90E080E0BDCFCF92DF9281
:10159000EF92FF920F931F93CF93DF93CDB7DEB7F8
:1015A0006C970FB6F894DEBF0FBECDBF8CE40E94DF
:1015B000461E882309F4B0C00E949A246B017C0166
:1015C00020E030E0A9010F94652E87FF04C0F7FAF0
:1015D000F094F7F8F094F7FAF094F7F8F094C98ED5
:1015E000DA8EEB8EFC8E8CE0E6ECF2E0DE011196FA
:1015F00001900D928A95E1F788E50E94941E882358
:10160000A1F040E050E0BA0188E50E94C424209196
:10161000D0083091D1084091D2085091D3080F944E
:10162000042C69837A838B839C8389E50E94941EB2
:101630008823A1F040E050E0BA0189E50E94C4246B
:101640002091D0083091D1084091D2085091D30810
:101650000F94042C6D837E838F8398878AE50E9484
:10166000941E882351F040E050E0BA018AE50E94C0
:10167000C42469877A878B879C871D861E861F8670
:10168000188A80912311811138C020E0AE01435F98
:101690005F4FBE016F5F7F4FCE0149960E94418828
:1016A000882359F18091CD0581110E9416F760E0E1
:1016B00080E00E941389898D9A8DAB8DBC8DB058C6
:1016C0008D8B9E8BAF8BB88F198A1A8A1B8A1C8AC6
:1016D0001D861E861F86188A80912311882369F033
:1016E00010E000E020E0AE014B5E5F4FBE016F5E98
:1016F0007F4FCE010D960E94FE866C960FB6F89431
:10170000DEBF0FBECDBFDF91CF911F910F91FF9034
:10171000EF90DF90CF900895C12CD12C80E8E82E77
:1017200080E4F82E58CF2F923F924F925F926F92A3
:101730007F928F929F92AF92BF92CF92DF92EF9261
:10174000FF920F931F93CF93DF93CDB7DEB7E5974B
:101750000FB6F894DEBF0FBECDBF8DAB209118053C
:101760002CAB21E020931805809136058D3409F4C7
:1017700005C6843511F40C94E6A0873409F091C1B4
:1017800080913405909135058B31910509F4DDC1C7
:1017900008F079C18430910508F030C12091E90644
:1017A0008230910508F48EC1213009F091C111E019
:1017B000029709F010E00E94DB2419821A821B8232
:1017C0001C821D821E821F82188682E50E94941E42
:1017D000882309F490C10E949A246B017C0120E0C7
:1017E00030E0A9010F943525882309F4EAC0409020
:1017F000280C5090290C60902A0C70902B0C809132
:101800002C0C90912D0CA0912E0CB0912F0C8CA72C
:101810009DA7AEA7BFA78090740790907507A09072
:101820007607B09077078091780790917907A0911B
:101830007A07B0917B0788AB99ABAAABBBABA5018C
:101840009401C301B2010F94352581110DC028A95F
:1018500039A94AA95BA96CA57DA58EA59FA50F9462
:101860003525882309F4ADC0A3019201C501B40157
:101870000F94042C20E030E040E05FE30F949B25C0
:1018800068A779A78AA79BA72CA53DA54EA55FA50C
:1018900068A979A98AA99BA90F94042C20E030E0BB
:1018A00040E05FE30F949B252B013C0120E030E0FA
:1018B000A901C701B6010F943525881F8827881F05
:1018C000181709F40FC180E090E0A0E8BFEB8CA7E7
:1018D0009DA7AEA7BFA728A539A54AA55BA5CA01A4
:1018E000B9010F949B254B015C01A3019201C30137
:1018F000B2010F949B259B01AC01C501B4010F946B
:10190000052C0F94B32E4B015C01AC019B01C70168
:10191000B6010F94042C68AB79AB8AAB9BABA501E5
:101920009401C701B6010F94052C9B01AC0168A975
:1019300079A98AA99BA90F949B256B017C0120E0C2
:1019400030E0A9010F94652E87FDD1C0C701B60113
:101950000F94B32E6B017C01C301B2019058A50115
:1019600094010F94FF2C2CA53DA54EA55FA50F94C7
:101970009B25A70196010F949B2528A539A54AA56B
:101980005BA50F94052C69837A838B839C83A501C7
:10199000940168A579A58AA59BA50F94FF2C2CA579
:1019A0003DA54EA55FA50F949B25A70196010F9419
:1019B0009B25A30192010F94052C6D837E838F8359
:1019C000988720E030E0A90169817A818B819C8130
:1019D0000F9435258111A3C020E030E0A9016D816D
:1019E0007E818F8198850F943525811198C00E9442
:1019F000134E8BEB9FE00E9444386AC085319105FD
:101A000009F466C08A31910509F49CC0049709F075
:101A100048C080E50E94941EC12CD12C76018823F9
:101A200021F00E9414246B017C0183E50E94941E26
:101A3000882361F00E949A2420E030E04AE754E4D1
:101A40000F949B250F94782D6B017C010E9483617C
:101A500080912511811105C060E081ED9FE00E9419
:101A6000B23F0E940EFDC60ED71EE81EF91E0E9450
:101A70000EFD6C197D098E099F0997FF29C080E032
:101A80000E941F5AF4CF8A32910509F4ECC260F427
:101A90008D31910509F415C208F470C04E9709F410
:101AA00068C20E942FF914C08B35910509F4BEC39A
:101AB0008C35910509F4BEC38A35910591F71092D2
:101AC000F40706C0213021F40E94DB240E94C06F7D
:101AD0003DA9311102C00F941A148CA980931805E6
:101AE0000C94479980E090E0A0E8BFE3F0CEC12CD1
:101AF000D12C760131CF89E40E94941E882331F0E5
:101B00000E949A2469837A838B839C838AE40E944F
:101B1000941E882309F455CF0E949A244ECF412F5A
:101B2000BE016F5F7F4F84E797E00F946D140E94B2
:101B30000EFD6093761170937711809378119093D6
:101B40007911C6CF0E94AF77C3CF87E00E94274E9E
:101B50008111BECF8CE0E2EDF2E0DE011196019042
:101B60000D928A95E1F770E060E080E50E943424F0
:101B7000BE016F5F7F4F0E94B067AACF87E00E94CF
:101B8000152A811106C060E08FE40E947224811141
:101B90009FCF0E948361109246026091390C8CE4C1
:101BA0000E947224E82E80E00E941C690E940EFDB3
:101BB00060937611709377118093781190937911D7
:101BC0000E94DB1C81E08093A5060E946D2B8AE5B4
:101BD0000E94461EF82E882369F081E00E94152A93
:101BE000182F82E00E94152A11110C9409A111E00E
:101BF000811101C010E088E50E94461E81110C94FD
:101C0000FBA0111145C189E50E94461E082F8113D2
